:020000040000FA
:06000000ABEFA8F01200B6
:020006001200E6
:0600080045EF93F0120029
:02000E000202EC
:0100100007E8
:020011000100EC
:020013000000EB
:0600180011EF3DF01200A3
:02001E000B00D5
:100020004A530100000B0000400000003253010061
:10003000E7080000180000002D530100F709000038
:100040000500000001530100C80600002C0000005C
:10005000BC5201005D0A0000450000005F52010033
:10006000000A00005D000000F65101008E0900004A
:100070006900000013000000F30700000200000008
:10008000CB510100C80700002B000000B451010053
:10009000E20A00001700000011000000FE0400004A
:0400A000020000005A
:0C00A40061EC2AF0E8EC25F001340FE2DA
:1000B00000501008270E01540AE2100EF36EFD0ED8
:1000C000F3CFDBFF270EF36EFE0EF3CFDBFF46EC24
:1000D0002BF003E3F36AF46A4ED0DE6ADD6AE8ECE3
:1000E00025F0013430E20050B808240E01542BE210
:1000F000B80E035D240E04590DE2E8EC25F0B80EAD
:10010000005E240E015A026A036A01AE05D002683D
:10011000036802D044EC26F0280E51EC29F02C0E96
:100120000026010EF4EC2BF0580E2B6E020E34EC70
:1001300025F0B80EF36EFD0EF3CFDBFF240EF36E49
:10014000FE0EF3CFDBFF46EC2BF00FE244EC26F083
:10015000B40E51EC29F05C0E0026120EF4EC2BF0DC
:10016000B80E2B6E240E34EC25F090EC24F000C079
:10017000F3FF01C0F4FF020EE15C02E2E16AE55226
:10018000E16E0BEF23F006EC23F00E0EE12606ECF9
:1001900025F05EEC26F0040E02C0DBFF050EA4EC99
:1001A00024F024EC27F0080E02C0DBFF090EBFECA0
:1001B00024F00A0E00C0DBFF0B0E01C0DBFF0C0EAB
:1001C00002C0DBFF0D0E03C0DBFFCDC9E6FFCEC9C9
:1001D000E6FFCFC9E6FFD0C9E6FF380EE66EE40EB3
:1001E000E66E000EF2EC2DF0BDEC74F0D6EC2CF0C7
:1001F00069EC27F0300EE66EE40EE66E000E4EEC73
:100200002BF00FEC26F098EC28F04EEC2BF0A0EC45
:1002100026F046EC2CF0D9C9E6FFDAC9E6FF46EC39
:100220002CF009019F51D8EC2DF00901E051D8ECD8
:100230002DF0E3C900F0016A00BE01686DEC23F007
:1002400098EC28F0D1EC22F00901E951D8EC2DF01E
:100250002BEC27F001AE02D002680368040E80EC9C
:1002600025F0FDE1F9EC2BF098EC28F049EC2CF0AE
:10027000AFEC74F0046E090EBDEC2AF095EC23F09F
:10028000080EDBCF02F0090EDBCF03F09EEC21F06D
:10029000DAEC2CF00AEC28F003EC28F09EEC21F0CC
:1002A000DAEC2CF072EC23F0B6EC2AF027EC24F018
:1002B000DAEC2CF06A0EE66E090EE66E3DEC2DF0DF
:1002C000006E0E0EE15C02E2E16AE552E16E005062
:1002D0000BEF23F0FDEC2BF0010EDB6A020EDB6A64
:1002E000DF6ADF50006E016AFD0EDBCF02F0FE0E0A
:1002F000DBCF03F003500118E8AE02D0013402D086
:1003000023EC26F001E28ED065EC26F0DEEC27F03F
:1003100004BE056836EC2AF024C003F025C004F0C2
:1003200026C005F0C2EC2CF00800F55033E1D20EE7
:10033000066E3B0E076E010E086E010EDBCF09F054
:10034000020EDBCF0AF00B6A0ABE0B68DEEC2CF063
:100350009DEC2BF06DEC84F024C009F025C00AF070
:1003600026C00BF006502424F36E07502520F46EAF
:10037000085026209DEC29F096EC2BF00BE165EC63
:1003800026F0DEEC27F004BE056862EC23F0F550A1
:10039000DF6E41D0DF50006E016AFD0EDB500018A9
:1003A0003AE1FE0EDB50011836E17F0E0601C85D12
:1003B00023E1010EDBCFE6FF020EDBCFE6FF1D0ED1
:1003C000E66EE40EE66E000EF2EC2DF073EC2CF00F
:1003D00011EC28F01B0EE66EE40EE66E000EE66EE3
:1003E000030EDBCFE6FF040EDBCFE6FF41EC22F08D
:1003F00011EC28F07DEC29F0A390A392010EDBCF45
:10040000E2FA020EDBCFE3FA15D85CD90A01E26901
:10041000E369A382A380010EDB2A020E01E261D709
:10042000DB2A5FD7050EE15C02E2E16AE552E16E8C
:100430000BEF23F0FDEC2BF00A01800EE3154DE1EC
:10044000C9EC26F008BE09689CEC23F00EBE0F68CC
:10045000DBEC23F0030E00C0DBFF040E01C0DBFF6A
:10046000D950030FBAEC2CF0550EEE1809E1010E2D
:10047000ED1806E1DF6A51EC2BF004AE04D002D097
:10048000000E16D1056862EC23F0F5CF40FB030E99
:10049000DB6A040EDB6A030EDBCF00F0040EDBCF59
:1004A00001F0080E0DEC26F030E2D5EC26F007BE88
:1004B000086898EC25F0030EDBCF09F0040E42EC3F
:1004C00025F0030EDBCFE9FF040E55EC27F0030EF9
:1004D000DB2A040EE0E3DB2ADED7010E6014DF6EB8
:1004E0000F0E65140B01406F66CF41FB67CF42FBD7
:1004F00068CF43FB69CF44FB6ACF45FB6BCF46FB1C
:100500006CCF47FB6DCF48FB609EDF5001E0CFD042
:10051000540E0B01445D01E0CAD045CB03F0026AE2
:10052000465163EC25F02CE232EC27F0026A0234EB
:10053000000E021807E6D880400E00549C0E0154AD
:10054000000E02541DE3010EDBCF03F9020EDBCFD8
:1005500004F90901D89004330333D89004330333EA
:100560000351095D04510A5904E203C909F904C998
:100570000AF90551035D0651045902E272EC27F0B5
:100580000F0E0B014215036E026A435163EC25F016
:1005900001E38DD032EC27F0000E005C0F0E015805
:1005A00001E385D0010EDBCF15F9020EDBCF16F982
:1005B0000901D00ED8801557070E16573E51135D0E
:1005C0003F51145907E33E51135D006E14513F55DE
:1005D000016E21D018EC28F0086A096A010E0A6E33
:1005E0000B6A3EC90CF03FC90DF00E6A0F6A0C5041
:1005F000085C046E0D500958056E0E500A58066EC0
:100600000F500B58076E045000260550012206506B
:10061000022207500322A4EC2BF013C93EF914C99F
:100620003FF932EC27F0026A036AD9EC25F0E9ECD5
:1006300024F0163521E215510008000E16551CE273
:100640002BEC27F001AE02D002680368D9EC25F04C
:10065000040EB9EC29F0E9EC24F02BEC27F001AE04
:1006600002D00268036800506227015063230250E1
:100670006423035065231BD019EC27F001AE02D090
:1006800002680368D9EC25F0080EB9EC29F0E9EC12
:1006900024F019EC27F001AE02D002680368005084
:1006A0006627015067230250682303506923010E17
:1006B000006E050EE15C02E2E16AE552E16E005077
:1006C0000BEF23F006EC23F00E0EE1260A01800E5C
:1006D000E31570E1C9EC26F008BE09689CEC23F034
:1006E0000EBE0F68DBEC23F063EC24F0F0EC22F09C
:1006F000900E0016050E0116900E001805E1050E6D
:10070000011802E1020E1BD0F0EC22F0900E001650
:10071000060E0116900E001805E1060E011802E102
:10072000030E0DD0F0EC22F0500E0016050E01164F
:10073000500E001816E1050E011813E1040EDF6ECD
:100740000F0EE76E040EDBCF00F0050EE75000162B
:10075000016A010E00C0DBFF51EC2BF004AE04D0A7
:1007600002D0000E03D3056862EC23F0F5CF40FB06
:10077000040EDB6A050EDB6AF0EC22F0080E0DECCD
:1007800026F041E2D5EC26F007BE086898EC25F08B
:10079000040EDBCF09F0050E42EC25F0040EDBCF92
:1007A000E9FF050E55EC27F0040EDB2A050EE4E305
:1007B000DB2AE2D7070E0F015015DF6EE00E52154F
:1007C000E00BE838E840006E010E5115080DF350BB
:1007D0000024E76E010EE7CFDBFF0F0E55150B016E
:1007E000406F56CF41FB57CF42FB58CF43FB59CF09
:1007F00044FB5ACF45FB5BCF46FB5CCF47FB5DCF4D
:1008000048FB0F01509F020EDF5C01E0A4D0010EF7
:10081000DB500E0A01E185D0070A31E00E0A01E043
:10082000A4D20B0141AB08D0E60E09018E6F8F6B8D
:1008300009010A0E906F05D009018E6B8F6B0901BB
:10084000906B42CB17F9100E090117150AE0090148
:100850009951800B06E1000E09013E6F3F6B136F4B
:10086000146B0B014851000801E37FD2F00E485D84
:1008700001E37BD2280E485D0901C06F76D2600E7D
:10088000090117150BE1FF0E0B01465D07E046510C
:10089000000804E2465109010B6F0C6B47CB03F0D3
:1008A000026A0B014851C1EC2AF05EEC26F0D950E7
:1008B000020FBAEC2CF0FF0EEE1802E1FF0EED185D
:1008C00001E153D2020EDBCF28F0030EDBCF29F07B
:1008D00009010D51285C006E0E512958016E24EC5F
:1008E00027F095EC23F0D890015004E60A0E005C46
:1008F000000E015802E3010E0AD095EC23F00134FA
:1009000008E30050F608FF0E015403E3020E3D6FAA
:1009100001D03D6B020EDBCF0DF9030EDBCF0EF9DC
:1009200024D241CB01F0006A0B014251090100249D
:10093000136F000E0120146F0B014651280808E2C6
:10094000F00E465D05E2280E465D0901C16F0DD22D
:100950000901C16B0AD2030EDF5C35E1010EDB50E9
:100960000F0A01E002D20901B55101E1FED10F0EDB
:100970000B014415300F0901AE6F0B0144390F0B09
:10098000300F0901AF6F0F0E0B014315300F090136
:10099000B06F0B0143390F0B300F0901B16F0F0E10
:1009A0000B014215300F0901B26F0B0142390F0BD9
:1009B000300F0901B36F0F0E0B014115300F090104
:1009C000B46FB56BD2D1040EDF5C01E078D1090EB3
:1009D000FEC0DBFF010EDB500F0A01E125D1010A49
:1009E00001E1E5D0090A01E19BD0030A6CE0020AAB
:1009F00001E0BBD1FF0E0B01415D01E1B6D194ECEA
:100A000028F001E1B2D15FEC28F0C7EC25F0FDE160
:100A10000B0142390F0B000100108E6F01C08FF0E7
:100A200039EC27F000010010966F01C097F09CECA4
:100A300027F0C7EC25F0FDE10B0145390F0B000154
:100A400000109E6F01C09FF040EC27F000010010E5
:100A5000A66F01C0A7F00B014751006E016A040E9A
:100A6000C7EC25F0FDE10B0148390F0B0001001028
:100A7000AE6F01C0AFF0090EDB50FC0B3C0803E188
:100A80003F0EFE6F72D1090EDB50FC0B01E16DD100
:100A9000090EDB50030B010FE76E080EE7CFDBFFFB
:100AA000DB50030803E1090EDB6A06D1080EDBCF39
:100AB000E6FF090EDB50FC0BE552E710E76E090E6E
:100AC000E7CFDBFFF9D0FF0E0B01415D01E14DD116
:100AD00094EC28F001E149D1080EDB6A070EF36EB1
:100AE000080EDBCFF4FFF350F45C13E2080EDB508A
:100AF000EA6A410FE96E0B0EEA22EF50E66E080E2D
:100B0000DB50FAEC22F0E552E750EF6E080EDB2ADC
:100B1000E5D7090EDB84F5EC26F001E283D07DD029
:100B2000FF0E0B01415D01E120D194EC28F001E1C1
:100B30001CD15FEC28F0C7EC25F0FDE10B01423938
:100B40000F0B00010010B66F01C0B7F039EC27F0B1
:100B500000010010BE6F01C0BFF09CEC27F0C7EC95
:100B600025F0FDE10B0145390F0B00010010C66FA8
:100B700001C0C7F040EC27F000010010CE6F01C0AB
:100B8000CFF00B014751006E016A040EC7EC25F04F
:100B9000FDE10B0148390F0B00010010D66F01C0B9
:100BA000D7F0090EDB86F5EC26F03CE336D0FF0EDD
:100BB0000B01415D01E1D9D094EC28F001E1D5D0E1
:100BC0005FEC28F0C7EC25F0FDE10B0142390F0B7B
:100BD00000010010DE6F01C0DFF039EC27F00001EA
:100BE0000010E66F01C0E7F09CEC27F0C7EC25F0A1
:100BF000FDE10B0145390F0B00010010EE6F01C044
:100C0000EFF040EC27F000010010F66F01C0F7F0A4
:100C1000090EDB88F5EC26F005E33F0EF36E090EB6
:100C2000F3CFDBFF090E48D0FF0E0B01465D01E15B
:100C30009CD094EC28F001E198D04651026E036AF2
:100C4000040ED89002360336E804FBE10B01473965
:100C50000F0B00010210006E0A0E00C0DBFF0B0E2E
:100C600003C0DBFF0F0E0B014715036E026A4851EC
:100C700000010210006E0C0E00C0DBFF0D0E03C061
:100C8000DBFF1FEC28F00A0EDB5000240001606F30
:100C90000B0EDB50000101200001616FD890613321
:100CA0006033090EDB8AF5EC26F005E33F0EF36EA8
:100CB000090EF3CFDBFF090EDBCFFEF056D0050E99
:100CC000DF5C53E1010EDB50070A4FE146CB00F039
:100CD000016A026A036A040E26EC28F0FDE145CBA6
:100CE00004F0056A066A076A040E1F0B03E0ECECC9
:100CF00024F0FDE1045000120550011206500212CA
:100D00000750031244CB08F0096A0A6A0B6A0C0EFA
:100D10001F0B07E0D890083609360A360B36E8066E
:100D2000F9E108500012095001120A5002120B504A
:100D3000031243CB0CF00D6A0E6A0F6A140E1F0BE0
:100D400007E0D8900C360D360E360F36E806F9E17E
:100D500000500C1009010F6F01500D10106F025060
:100D60000E10116F03500F10126F010E006E0E0E59
:100D7000E15C02E2E16AE552E16E00500BEF23F024
:100D8000FDEC2BF002EC2CF07F0E0601C85D04E0B8
:100D9000200EC85D01E0B0D0030EE66ECEEC27F069
:100DA00063EC2CF0170EE66EE40EE66E000EEFEC30
:100DB00025F005E0010EF36E020EF3CFDBFF140EFB
:100DC000E66EE40EE66E000EEFEC25F005E0010E97
:100DD000F36E030EF3CFDBFF090118A11ED0030E43
:100DE000DB500CE00A015D5109E00A015E5106E1A9
:100DF0008FEC2BF0CD0EABEC2BF01891020EDB50EC
:100E00000CE05DEC27F0BFEC1CF001EC2EF00009CB
:100E100002E0D1EC58F009011891090118A322D081
:100E2000030EDB5010E00A015D510DE00A015E5136
:100E30000AE18FEC2BF0CF0E9CEC26F07AEC0EF052
:100E4000A2EC27F01893020EDB500CE05DEC27F0CB
:100E50004FEC0EF001EC2EF0000902E0D1EC58F05E
:100E600009011893090118A90CD00A015D0509E1CF
:100E70000A015E5106E18FEC2BF0CE0EABEC2BF0AD
:100E80001899090118A524D00A015D0521E10A017C
:100E90005E511EE1020EF36E040EF3CFDBFFD00EA7
:100EA000E66EE66A040EDBCFE6FFA5EC27F064EC05
:100EB00028F0DBCFE6FFC3EC00F0E55264EC28F04D
:100EC000DB50020802E02AEC2EF00901189518897F
:100ED000090118A711D00A015D050EE10A015E5152
:100EE0000BE1020EE66EC3EC00F0E552020802E0F0
:100EF0002AEC2EF009011897050EE15C02E2E16A86
:100F0000E552E16E0BEF23F03BDF010C06EC23F022
:100F1000070EE1260501EF51DE6EDD6AF051E66E47
:100F2000D950020F71EC25F0F151E66ED950040F43
:100F300071EC25F04B0E0701CB5D38E172EC23F02C
:100F4000013418E288EC26F015E247EC27F0033470
:100F500002E2BFEC27F003E3006A016A09D072ECF9
:100F600023F0A3EC29F08DEC26F0FDE192EC26F0C5
:100F70005EEC26F0F0EC22F0013418E288EC26F06A
:100F800015E2B6EC2AF0033402E2BFEC27F003E3EB
:100F9000006A016A09D0F0EC22F0A3EC29F08DEC94
:100FA00026F0FDE192EC26F063EC24F00901A52B7C
:100FB000000EA623A723A823320E0901016A0325E8
:100FC000006E04510122640EDFEC29F028C0A0F964
:100FD0007BEC27F059EC2BF0D880000E2654000E45
:100FE0002754000E2854000E295406E30901CD6B46
:100FF000CE6BCF6BD06B2AD00FC900F010C901F0B7
:1010000011C902F012C903F0A5EC2CF07BEC27F01B
:10101000E3EC2DF0A5EC2CF0E2EC22F0050E005EE6
:10102000000E015A025A035A040E26EC28F0FDE184
:1010300000C0CDF901C0CEF902C0CFF903C0D0F98C
:101040000901CD2B000ECE23CF23D023D2EC27F0E5
:1010500027E1320E0901036A0D25026E0E510322AB
:10106000640E2D6E2E6A02C028F003C029F066ECD3
:10107000A8F028C002F029C003F0000ED880285440
:10108000000E295403E3006A016A0CD0CCEC2CF06A
:10109000A3EC29F08DEC26F0FDE192EC26F002D0D5
:1010A000CCEC2CF000C09FF90901000ED8808E55C1
:1010B000000E8F5505E20901998709019D8904D029
:1010C0000901999709019D99600E090117152008DA
:1010D00004E109019985998902D0090199990901C9
:1010E00017A910D0090199BF2ED0998F0901A96BBA
:1010F000AA6BAB6BAC6B010EF3EC24F0F2EC14F0CA
:1011000087D921D0090199AF1ED0999FA5C9A9F906
:10111000A6C9AAF9A7C9ABF9A8C9ACF90901A907D9
:10112000000EAA5BAB5BAC5B010EF3EC24F0D88045
:10113000E40E09011D55570E1E55000E1F55000ED9
:10114000205501E2188381EC15F06ED9090199A9A7
:10115000E0D0640E006E016A07EC2CF02D6E01C029
:101160002EF066ECA8F0060E28C0DBFF0901000E89
:10117000D8800755000E08553FE2000ED880035571
:10118000000E045539E2000ED8800555000E0655B4
:1011900033E2C1EC22F007EC2CF027EC82F05BECA0
:1011A00029F041EC83F0DDEC84F028C00BF929C074
:1011B0000CF90901000ED8802854000E29540EE2C3
:1011C000FBEC26F004E30901A36BA46B07D066ECEB
:1011D0002DF08DEC26F0FDE1E6EC27F0F0EC22F0AE
:1011E000013406E288EC26F003E214EC23F004D08C
:1011F000A3C9A1F9A4C9A2F9150E0901945D03E1DF
:10120000040EF3EC24F009019451020808E2010EE7
:10121000946F03C909F904C90AF9FAD861D0090120
:10122000000ED8800355000E04552CE290EC24F0FB
:10123000013428E288EC26F025E2060EDB50026E2F
:10124000036ADECF04F0DDCF05F003500518E8AEE9
:1012500002D0053404D00450025C0550035812E358
:101260000051066E076ADECF08F0DDCF09F00750A7
:101270000918E8AE02D0093404D00850065C0950C1
:10128000075828E3FBEC26F02DE2020EDBCF0AF034
:10129000030EDBCF0BF00B3425E20A500008000EE2
:1012A0000B5420E2020EDBCF0CF0030EDBCF0DF06F
:1012B00009010C50A15D0D50A25914E3020EDBCFC1
:1012C0000EF0030EDBCF0FF009010E50015D0F5041
:1012D000025908E20901020E946F040EF3EC24F0A7
:1012E000020E0DD0020E0901945D0BE00901B80E4B
:1012F000035D240E045905E30901020E946FF3EC1B
:1013000024F0060EDBCF00F9A1C901F9A2C902F948
:1013100047D00901FBEC26F01CE2FBEC26F004E3CD
:101320000901A36BA46B07D066EC2DF08DEC26F0C1
:10133000FDE1E6EC27F0F0EC22F0013406E288EC67
:1013400026F003E214EC23F004D0A3C9A1F9A4C948
:10135000A2F909019451020813E30901100E095D75
:10136000270E0A5903E30901040E02D00901150EE4
:10137000946F040EF3EC24F0020EF3EC24F010D082
:1013800009019951800B0CE09951100B09E1995119
:10139000040B06E099950901040E946F72EC27F096
:1013A0000901000ED8800D55000E0E5516E20501FC
:1013B000ED51000812E2C8C700F0C9C701F0050EE0
:1013C0002D6E2E6AC8C728F0C9C729F066ECA8F0B0
:1013D0002450251002E109011887000E006E070E47
:1013E000E15C02E2E16AE552E16E00500BEF23F0AE
:1013F000090117BF08D0400E176F09018E6B8F6B64
:101400000901906B000C179F000C09011885000C56
:10141000A3908CEC2AF013C93EF914C93FF9ACEC47
:1014200025F0A38096EF2AF006EC23F0100EE126BB
:10143000090117A9EFD00901E35103E1BDEC26F042
:10144000E9D009015C515D115E115F1107E1A7EC64
:1014500026F0A390ACEC25F0A380DCD05C0EE96E06
:10146000090EEA6EEE500F5D266EEE501059276E93
:10147000EE501159286EEE501259296EA5EC2CF041
:1014800089ECA7F022C0DEFF23C0DEFF24C0DEFF10
:1014900025C0DDFFDD52DD528EEC2CF0D890030E1E
:1014A000EB50000A08E6640EEE5C000EEE58000EEB
:1014B000EE58000EEE5801E2ADD0A390080E62C9BE
:1014C000DBFF090E63C9DBFF0A0E64C9DBFF0B0EED
:1014D00065C9DBFF0C0E66C9DBFF0D0E67C9DBFFBC
:1014E0000E0E68C9DBFF0F0E69C9DBFF0901ACEC0A
:1014F00025F0A38060510901DB5D006EDC5109011C
:101500006155016E63EC24F0F0EC22F0026A036A8C
:1015100001AE02D002680368640E51EC29F0ACEC15
:1015200029F0EEEC83F0060E26C0DBFF070E27C085
:10153000DBFFA7EC26F095EC23F0D890015002E6F3
:1015400069EC28F02BE3DF5009014027010EDB5046
:101550004123020EDB504223030EDB504323B1EC48
:101560002BF02850442729504523080EDB504627EE
:10157000090EDB5047230A0EDB5048230B0EDB50CD
:1015800049230C0EDB504A270D0EDB504B230E0E69
:10159000DB504C230F0EDB504D233CD095EC23F059
:1015A000013438E30050FF08FF0E015433E3DF50ED
:1015B00009014E27010EDB504F23020EDB50502352
:1015C000030EDB50512328682968040EDBCF2DF071
:1015D000050EDBCF2EF022EC84F0265009015227B5
:1015E00027505323080EDB505427090EDB50552398
:1015F0000A0EDB5056230B0EDB5057230C0EDB502C
:1016000058270D0EDB5059230E0EDB505A230F0EB8
:10161000DB505B23100EE15C02E2E16AE552E16E11
:101620000BEF23F006EC23F0190EE1260C0EDB6A1B
:101630000D0EDB6A0E0EDB6A06EC25F000C0DFFF44
:10164000010E01C0DBFF020E02C0DBFF030EA4ECA3
:1016500024F063EC24F0060E02C0DBFF070EBFECA3
:1016600024F0080E00C0DBFF090E01C0DBFF0A0EEC
:1016700002C0DBFF0B0E03C0DBFFD9CFE9FF8FEC0D
:1016800029F045E219C900F01AC901F01BC902F09E
:101690001CC903F097EC2CF019C926F01AC927F0E1
:1016A0001BC928F01CC929F00CEC2CF00C0E26C02C
:1016B000DBFF25C900F026C901F027C902F028C9BF
:1016C00003F097EC2CF025C926F026C927F027C98E
:1016D00028F028C929F00CEC2CF00D0E26C0DBFFF9
:1016E00031C900F032C901F033C902F034C903F046
:1016F00097EC2CF031C926F032C927F033C928F015
:1017000034C929F00CEC2CF00E0E26C0DBFF1AECCD
:101710002BF077EC2CF0F0EC22F06CEC26F0005083
:1017200001100210031007E08EEC2CF0D8800A0E96
:1017300044EC2DF003E313EC2AF0B5D0FE0EDB50A1
:10174000740801E0B8D013EC2AF0F6EC28F0010E92
:10175000E66EE66A8EEC2CF0EECF00F0EECF01F0F4
:10176000EECF02F0EFCF03F0E80E2B6E030E2C6EDF
:10177000ABEC28F0ABEC2CF0000EE66EE40EE66E5F
:10178000000E5BEC2CF0B1EC2DF001EC2BF00C0E0C
:10179000BEEC2CF0F40EE66EE30EE66E000EB5EC39
:1017A00028F01DC900F01EC901F01FC902F020C9B0
:1017B00003F0FDEC29F0F8EC2CF0F6EC28F00D0E1F
:1017C000BEEC2CF0E40EE66EE30EE66E000EB5EC19
:1017D00028F029C900F02AC901F02BC902F02CC950
:1017E00003F0FDEC29F02DC900F02EC901F02FC93E
:1017F00002F030C903F0F6EC28F00E0EBEEC2CF02F
:10180000D80EE66EE30EE66E000EB5EC28F035C994
:1018100000F036C901F037C902F038C903F0FDEC19
:1018200029F039C900F03AC901F03BC902F03CC9BE
:1018300003F0F6EC28F09FEC2AF0CF0EE66EE30EF4
:10184000E66E000E2EEC22F046C900F047C901F00A
:1018500048C902F049C903F0EFEC2AF04AC900F088
:101860004BC901F04CC902F04DC903F0F6EC28F069
:10187000A8EC2AF0C00EE66EE30EE66E000E2EEC2B
:1018800022F054C900F055C901F056C902F057C9F9
:1018900003F0EFEC2AF058C900F059C901F05AC919
:1018A00002F05BC903F0F6EC28F0050EE66EE40EDC
:1018B000E66E000E28D18EEC2CF0150EEECFDBFF7D
:1018C000160EEECFDBFF170EEECFDBFF180EEECFBE
:1018D000DBFF01EC22F013E25DEC23F010E2D7EC29
:1018E00028F0100E2B6E270E36EC29F0B40EE66EA3
:1018F000E30EE66E000EABEC21F0B0EC28F0040E27
:101900001DC9DBFF050E1EC9DBFF060E1FC9DBFF6D
:10191000070E20C9DBFF080E21C9DBFF090E22C913
:10192000DBFF0A0E23C9DBFF0B0E24C9DBFF150EFC
:1019300019C9DBFF160E1AC9DBFF170E1BC9DBFF27
:10194000180E1CC9DBFF01EC22F00DE25DEC23F068
:101950000AE20C0EBEEC2CF09F0EE66EE30EE66E75
:10196000000E4CEC2CF0040E29C9DBFF050E2AC931
:10197000DBFF060E2BC9DBFF070E2CC9DBFF080EB1
:101980002DC9DBFF090E2EC9DBFF0A0E2FC9DBFFB5
:101990000B0E30C9DBFF150E25C9DBFF160E26C95D
:1019A000DBFF170E27C9DBFF180E28C9DBFF01EC90
:1019B00022F00DE25DEC23F00AE20D0EBEEC2CF0FD
:1019C000930EE66EE30EE66E000E4CEC2CF0040E69
:1019D00035C9DBFF050E36C9DBFF060E37C9DBFF55
:1019E000070E38C9DBFF080E39C9DBFF090E3AC9FB
:1019F000DBFF0A0E3BC9DBFF0B0E3CC9DBFF150EFC
:101A000031C9DBFF160E32C9DBFF170E33C9DBFF0E
:101A1000180E34C9DBFF01EC22F00DE25DEC23F07F
:101A20000AE20E0EBEEC2CF08A0EE66EE30EE66EB7
:101A3000000E4CEC2CF0040E46C9DBFF050E47C926
:101A4000DBFF060E48C9DBFF070E49C9DBFF080EA6
:101A50004AC9DBFF090E4BC9DBFF0A0E4CC9DBFF8D
:101A60000B0E4DC9DBFF150E40C9DBFF160E41C939
:101A7000DBFF170E42C9DBFF180E43C9DBFF01EC89
:101A800022F00EE25DEC23F00BE26CEC28F0840E09
:101A9000E66EE30EE66E000EE7EC2CF0B0EC28F0FC
:101AA000040E54C9DBFF050E55C9DBFF060E56C9EF
:101AB000DBFF070E57C9DBFF080E58C9DBFF090E15
:101AC00059C9DBFF0A0E5AC9DBFF0B0E5BC9DBFFEE
:101AD000150E4EC9DBFF160E4FC9DBFF170E50C99E
:101AE000DBFF180E51C9DBFF01EC22F00EE25DECCA
:101AF00023F00BE271EC28F0790EE66EE30EE66E51
:101B0000000EE7EC2CF0B0EC28F0190EE15C02E2DC
:101B1000E16AE552E16E0BEF23F006EC23F0020ED2
:101B2000C5EC26F0D00EEE1801E0AED0ED5001E08D
:101B3000ABD0590EE66EE30EE66E000EFFEC28F019
:101B400019C9E6FF1AC9E6FF1BC9E6FF1CC9E6FF73
:101B5000FBEC21F01DC9E6FF1EC9E6FF1FC9E6FF29
:101B600020C9E6FFFBEC21F021C9E6FF22C9E6FF10
:101B700023C9E6FF24C9E6FFFBEC21F025C9E6FFF7
:101B800026C9E6FF27C9E6FF28C9E6FFFBEC21F0DE
:101B900029C9E6FF2AC9E6FF2BC9E6FF2CC9E6FFE3
:101BA000FBEC21F02DC9E6FF2EC9E6FF2FC9E6FFA9
:101BB00030C9E6FFFBEC21F031C9E6FF32C9E6FF90
:101BC00033C9E6FF34C9E6FFFBEC21F035C9E6FF77
:101BD00036C9E6FF37C9E6FF38C9E6FFFBEC21F05E
:101BE00039C9E6FF3AC9E6FF3BC9E6FF3CC9E6FF53
:101BF000FBEC21F040C9E6FF41C9E6FF42C9E6FF20
:101C000043C9E6FFFBEC21F09FEC2AF0DAEC2CF064
:101C100046C9E6FF47C9E6FF48C9E6FF49C9E6FFEE
:101C2000FBEC21F04AC9E6FF4BC9E6FF4CC9E6FFD1
:101C30004DC9E6FFFBEC21F04EC9E6FF4FC9E6FFB8
:101C400050C9E6FF51C9E6FFFBEC21F0A8EC2AF0F1
:101C5000DAEC2CF054C9E6FF55C9E6FF56C9E6FF99
:101C600057C9E6FFFBEC21F058C9E6FF59C9E6FF6A
:101C70005AC9E6FF5BC9E6FFFBEC21F06C0EE66E8D
:101C8000090EE66E57EC24F0FE0EDB50D6EC27F082
:101C900002E2E16AE552E16E00500BEF23F006EC40
:101CA00023F0E652FE0EDB500FE00501F3B50CD039
:101CB000A8EC29F003E079EC23F008E1B9EC28F076
:101CC00003E079EC23F002E1000E11D0E3EC2AF0FE
:101CD00004E078EC25F0200901D0650EDF6E0601E6
:101CE000006BDFCFE6FF9EDCE55201EC2DF0E55204
:101CF0000BEF23F006EC23F0030EC5EC26F0D00E1C
:101D0000EE1811E1ED500FE1FE0EDB5005E07CEC2A
:101D100025F0A5EC27F020D084EC27F0A5EC27F0E7
:101D2000020829E026D0E7EC2AF005E087EC25F050
:101D3000EF50200901D0650EE76E020EE7CFDBFF02
:101D4000D0EC29F0020EDBCFE6FF6CDCE552FE0E94
:101D5000DB500BE03AEC2EF0E5EC29F007EC2DF02F
:101D60006CEC2DF0EFEC2CF006D00DEC2EF03AECF4
:101D70002EF02AEC2EF0010E006E030EE15C02E262
:101D8000E16AE552E16E00500BEF23F061EC2AF0BE
:101D9000FE0EDBCFE6FF76EC31F0E552E76EFE0E8D
:101DA000E7CFDBFF86EC2CF003E073EC26F003D0EA
:101DB000C80E006E016A06EC2AF00901175159ECB1
:101DC0002AF0A2EC22F00901995172EC2DF00901E0
:101DD0009D5172EC2DF009019451D8EC2DF00DC9F4
:101DE000E6FF0EC9E6FF46EC2CF015C9E6FF16C962
:101DF000E6FF46EC2CF088EC27F0FBEC21F07BECC6
:101E000028F046EC2CF080EC28F046EC2CF085EC29
:101E100028F046EC2CF00BC9E6FF0CC9E6FF46ECB7
:101E20002CF007C9E6FF08C9E6FF46EC2CF0A3C971
:101E3000E6FFA4C9E6FF46EC2CF0A1C9E6FFA2C963
:101E4000E6FF46EC2CF00701CA51D8EC2DF0ADECC2
:101E500027F002E1010E02D0FE0EDB50D6EC27F097
:101E600002E2E16AE552E16E00500BEF23F006EC6E
:101E700023F0E150FA0FBAEC22F00AE087EC25F0EB
:101E8000EF5006E0ECEC29F0B5EC25F091EC27F0F2
:101E9000FE0EDB5006E07CEC25F078DFE552E552E3
:101EA000E552010E0BEF23F061EC2AF0E3EC2AF08F
:101EB00009E078EC25F006E0FAEC24F0B5EC25F02A
:101EC00091EC27F00501F3B50CD0A8EC29F003E064
:101ED00079EC23F008E1B9EC28F003E079EC23F089
:101EE00002E1000ECFD0FE0EDB5002E08EEC23F0BC
:101EF0008AEC28F009011751E66EE66A350EE66EA7
:101F0000E30EE66E000EA2EC22F088EC27F02F0E16
:101F1000E66EE30EE66E000EFAEC29F0D6EC2CF03D
:101F200018EC28F0F9EC2BF02A0EE66EE30EE66EC4
:101F3000000ED7EC22F03EC900F03FC901F0026A62
:101F4000036AF9EC2BF0250EE66EE30EE66E000E4A
:101F5000D7EC22F00901E951E66EE66A200EE66E42
:101F6000E30EE66E000E33EC29F07DEC29F07F0ED7
:101F70000601C85D35E18AEC28F00901E051E66E02
:101F8000E66A180EE66EE30EE66E000E33EC29F0FC
:101F900069EC27F0120EE66EE30EE66E000E63ECBF
:101FA0002BF00FEC26F00C0EE66EE30EE66E000E44
:101FB00063EC2BF0A0EC26F0060EE66EE30EE66E68
:101FC000000E33EC29F0D9C9E6FFDAC9E6FF000EAE
:101FD000E66EE30EE66E000E33EC29F07DEC29F0A0
:101FE0008AEC28F066C0E6FF67C0E6FFF90EE66EF1
:101FF000E20EE66E000EA2EC22F068C0E6FF69C0B9
:10200000E6FFF40EE66EE20EE66E000EA2EC22F0A3
:102010006AC0E6FF6BC0E6FFEE0EE66EE20EE66E0D
:10202000000EA2EC22F000016C51E66EE66AE90EA9
:10203000E66EE20EE66E000EA2EC22F000016D519B
:10204000E66EE66AE40EE66EE20EE66E000EA2ECC6
:1020500022F000016E51E66EE66ADE0EE66EE20EDA
:10206000E66E000EA2EC22F00001FE51E66EE66A7A
:10207000D90EE66EE20EE66E000EA2EC22F07DECCA
:1020800029F0010ED6EC27F002E2E16AE552E16E9A
:1020900000500BEF23F061EC2AF01AEC2BF063EC0C
:1020A0002CF0090199A53FD009019451040A10E0D0
:1020B000060A08E0030A12E1D00EE66EE20EE66EB2
:1020C000000E11D0BA0EE66EE20EE66E000E0BD0D8
:1020D000AC0EE66EE20EE66E000E05D09B0EE66ECE
:1020E000E20EE66E000E9EEC28F0F8EC2CF09EEC72
:1020F00021F0930EE66EE20EE66E000ED7EC22F0B3
:10210000050EE66EE40EE66E000E9EEC28F0040E60
:102110000901945D1EE0C8EC23F08A0EE66EE20E23
:10212000E66E000E14D0770EE66EE20EE66E000E3E
:102130009EEC28F00901100E035D270E045909E2F8
:10214000C8EC23F0670EE66EE20EE66E000E78EC49
:102150002DF0D2EC27F01CE1A3C9E6FFA4C9E6FFED
:102160005D0EE66EE20EE66E000E33EC29F0A1C9BC
:10217000E6FFA2C9E6FF590EE66EE20EE66E000E1D
:1021800033EC29F0550EE66EE20EE66E000E27D017
:10219000A3C900F0A4C901F0040EC7EC25F0FDE1CD
:1021A000ECEC2DF05D0EE66EE20EE66E000ED1EC6C
:1021B00022F0A1C900F0A2C901F0040EC7EC25F07D
:1021C000FDE1ECEC2DF0590EE66EE20EE66E000E2F
:1021D000D1EC22F0510EE66EE20EE66E000E9EECA1
:1021E00028F0020EE66EE66A03C900F004C901F0A9
:1021F000026A036A7BEC28F02FEC25F0490EE66EAC
:10220000E20EE66E000E7DEC24F0020EE66EE66A4B
:1022100005C900F006C901F0026A036A80EC28F0E3
:102220002FEC25F0450EE66EE20EE66E000E7DEC1C
:1022300024F0020EE66EE66A09C900F00AC901F050
:10224000026A036A85EC28F02FEC25F0410EE66E59
:10225000E20EE66E000E7DEC24F03E0EE66EE20E1F
:10226000E66E000E9EEC28F0D2EC27F01DE1CDC901
:1022700000F0CEC901F0CFC902F0D0C903F028ECBC
:1022800026F03DEC2CF0B6EC2DF0ABEC2CF0360E3D
:10229000E66EE20EE66E000ED7EC22F0550EE66E0C
:1022A000E20EE66E000E2FD0CDC904F0CEC905F0C7
:1022B000CFC906F0D0C907F028EC26F026C004F0FC
:1022C00027C005F028C006F029C007F0040E1F0B38
:1022D0003DEC2CF003E080EC25F0FDE1050E27EC51
:1022E00024F0360EE66EE20EE66E000EFAEC29F0F1
:1022F000086E090EE15E085063EC2CF0510EE66E9C
:10230000E20EE66E000E9EEC28F0020EE15C02E2A8
:10231000E16AE552E16E0BEF23F006EC23F0FE0ECE
:10232000DB500FE00501F3B50CD0A8EC29F003E079
:1023300079EC23F008E1B9EC28F003E079EC23F024
:1023400002E1000E05D00601006BA5DE01EC2DF0C8
:102350000BEF23F006EC23F0D0EC29F09CDE3AECF6
:102360002EF0010E0BEF23F061EC2AF086EC2CF03E
:1023700003E073EC26F003D0C90E006E016A06EC90
:102380002AF00501F15159EC2AF033EC29F0ADECBB
:1023900027F002E1010E02D0FE0EDB50D6EC27F052
:1023A00002E2E16AE552E16E00500BEF23F006EC29
:1023B00023F0E1501FEC2BF0CA0EEE1815E1ED50A2
:1023C00013E1E7EC2AF009E087EC25F0EF5005E097
:1023D000ECEC29F02DEC28F002D00501F16BECECCF
:1023E00029F01C0E8EEC25F0FE0EDB5006E07CEC96
:1023F00025F0BADFE552E552E552010E0BEF23F06E
:102400001DEC2CF028E0A8EC29F003E079EC23F097
:1024100006E1B9EC28F01FE079EC23F01CE0E7ECD2
:102420002AF016E0050E66EC2BF012E0E3EC2AF041
:1024300008E078EC25F005E0FAEC24F02DEC28F02B
:1024400002D00501F16BFAEC24F01C0E8EEC25F0A5
:102450000501F3A502D0000E31D08EEC23F0240E3E
:10246000E66EE20EE66E000EFFEC28F00501F1517B
:102470000AE11E0EE66EE20EE66E000E49EC2CF04E
:1024800041EC22F016D0F151C8EC2AF0D2EC27F042
:1024900006E1550E006EE20E016E000E05D0510EE3
:1024A000006EE20E016E000E026E6DEC23F0E1ECA8
:1024B00026F063EC2CF07DEC29F0010ED6EC27F031
:1024C00002E2E16AE552E16E00500BEF23F006EC08
:1024D00023F0080EE126020EDB6A34EC28F0050139
:1024E00053EC26F021EC2CF00501F151000807E235
:1024F000F151E66ED950060F71EC25F02AD0090192
:10250000055106110AE00751081107E0C1EC22F05D
:10251000EAEC26F0CEEC2AF004D0060EDB6A070EB9
:10252000DB6AD2EC27F015E16CEC26F0033402E212
:10253000BFEC27F003E3006A016A09D095EC23F0B1
:10254000A3EC29F08DEC26F0FDE192EC26F024ECD2
:1025500027F0D950060F25EC2AF00FE0060EDBCF4E
:1025600008F0070EDBCF09F00A6A0B6A09AE02D049
:102570000A680B683EEC23F002D0006A016A63EC43
:1025800024F086EC2CF003E073EC26F003D0CB0EA5
:10259000006E016A06EC2AF00501F05159EC2AF0B0
:1025A00033EC29F00501EF51D8EC2DF0040EDBCF10
:1025B000E6FF050EDBCFE6FF46EC2CF02EEC24F018
:1025C00046EC2CF0C8EC23F098EC28F0D1EC22F08B
:1025D000ADEC27F002E1010E02D0FE0EDB50006EE2
:1025E000080EE15C02E2E16AE552E16E00500BEF99
:1025F00023F006EC23F0040EC5EC26F0CC0EEE180A
:1026000045E1ED5043E1DE6ADD6A02EC2CF0E7ECD7
:102610002AF016E087EC25F0EF5012E098EC28F055
:10262000E66EECEC29F03BEC28F063EC2CF098EC37
:1026300028F0E66E8FEC2BF03BEC28F021EC2CF030
:102640008EEC2CF0EE50ED1005E0E7EC2DF0B5EC43
:1026500025F002D0006A016A00C0F0F5D950020FDF
:1026600025EC2AF005E02EEC24F0B5EC25F002D0A4
:10267000006A016A00C0EFF5E7EC2DF01B0E8EEC4E
:1026800025F02EEC24F01A0E8EEC25F0FE0EDB5019
:1026900006E07CEC25F01BDFE552E552E552010E29
:1026A000006E040EE15C02E2E16AE552E16E005068
:1026B0000BEF23F006EC23F0100EE126FE0EDB50AC
:1026C00068E0A8EC29F003E079EC23F006E1B9EC2E
:1026D00028F05FE079EC23F05CE0E7EC2AF056E0CC
:1026E000020E66EC2BF052E0060EDB6A3FEC28F09F
:1026F0000501EF6BF06BE3EC2AF03EE078EC25F09F
:102700003BE0FAEC24F078EC89F0E552E55221EC5C
:102710002CF0FAEC24F03CEC98F021EC2AF00006C6
:10272000000E015AF80EDB500024E96EF90EDB5062
:102730000120EA6E040EEFCFDBFFDB50250808E135
:1027400046EC28F0CEEC2AF0020EDBCFEFF507D0F6
:1027500046EC28F04DEC28F0020EDBCFF0F5FAEC59
:1027600024F022EC5AF0E552E552F80EF3CFDBFFED
:10277000F90EF4CFDBFFBFD7B8EC2BF01A0E8EECBE
:1027800025F0D5EC2AF01B0E8EEC25F00501F3A503
:1027900002D0000EFED08EEC23F00F0EE66EE20E9D
:1027A000E66E000EFFEC28F00501EF5108E1F05154
:1027B00006E10B0EE66EE20EE66E000EDCD005ECD6
:1027C0002BF0EF51000813E253EC26F00A0EF3CF82
:1027D000DBFF0B0EF4CFDBFF0501EF51C8EC2AF055
:1027E000A80EE66EE30EE66E000E9EEC28F00501E4
:1027F000F051000801E384D0F151000807E2F151E3
:10280000E66ED9500E0F71EC25F03AD00901055152
:1028100006110EE0075108110BE0C1EC22F0EAECC2
:1028200026F00E0E28C0DBFF0F0E29C0DBFF04D000
:102830000E0EDB6A0F0EDB6AD2EC27F021E10E0EE2
:10284000DBCF02F00F0EDBCF03F0033402E2BFEC6C
:1028500027F003E3006A016A0DD00E0EDBCF00F013
:102860000F0EDBCF01F0A3EC29F08DEC26F0FDE19B
:1028700092EC26F00E0E00C0DBFF0F0E01C0DBFF56
:10288000D9500E0F25EC2AF00FE00E0EDBCF08F02A
:102890000F0EDBCF09F00A6A0B6A09AE02D00A6894
:1028A0000B683EEC23F002D0006A016A0C0E00C0F7
:1028B000DBFF0D0E01C0DBFF0501EF51000807E251
:1028C000060EE66EE20EE66E000E9EEC28F00501A6
:1028D000F051C8EC2AF0D2EC27F006E1550E006E5C
:1028E000E20E016E000E05D0510E006EE20E016E7A
:1028F000000E026E6DEC23F0E1EC26F063EC2CF0A0
:102900001FEC28F0013420E288EC26F01DE2D950BB
:102910000A0F25EC2AF013E003EC28F00A0EDBCFB7
:1029200004F00B0EDBCF05F003500518E8AE02D023
:10293000053404D00450025C0550035805E20C0E27
:10294000DBCFE6FF0D0E0BD00AEC28F0013411E2CC
:1029500088EC26F00EE20A0EDBCFE6FF0B0EDBCF93
:10296000E6FFFD0EE66EE10EE66E000EE66EE9ECA9
:1029700021F0B3EC27F09EEC28F0C8EC23F0ED0E2C
:10298000E66EE10EE66E000E78EC2DF07DEC29F09F
:10299000010E006E100EE15C02E2E16AE552E16EAA
:1029A00000500BEF23F006EC23F0E652090117ADBF
:1029B00002D0010E14D00B0EDF6E3F0E0001FE5D43
:1029C00008E0DF50000805E2010EC4EC27F0DF0646
:1029D000F4D73F0EFE5D02E0000E01D0010EE5527D
:1029E0000BEF23F061EC2AF0DEDFDE6ADD6A66ECD5
:1029F0002AF002E626EC2CF02EE245EC22F0030E43
:102A0000DDEC22F0FDE181EC2CF0DDEC22F0FDE1CB
:102A10000FEC23F0040E95EC24F045EC22F0030EAD
:102A2000DDEC22F0FDE181EC2CF0DDEC22F0FDE1AB
:102A3000D4EC2DF095EC24F045EC22F0030EDDEC07
:102A400022F0FDE1E3EC2CF07EEC26F0DF2A010E13
:102A5000CEE3DB2ACCD7DE6ADD6A66EC2AF002E63A
:102A60003FEC2BF013E20EEC2DF0F0EC26F00EEC28
:102A70002DF098EC27F009EC29F062EC2DF052ECE7
:102A800027F0DF2A010EE9E3DB2AE7D7DE6ADD6AF9
:102A900066EC2AF002E669EC28F029E2F5EC2DF06C
:102AA000020E95EC24F0F5EC2DF0040E95EC24F0DC
:102AB00005EC29F00F0EBBEC2DF0110E2DEC2DF0D6
:102AC0000C0E2DEC2DF00D0E2DEC2DF0060EBBECAA
:102AD0002DF0080EBBEC2DF00E0E2DEC2DF00A0E95
:102AE0007EEC26F0DF2A010ED3E3DB2AD1D70001EA
:102AF000FE6B020EE15C02E2E16AE552E16E0BEF71
:102B000023F006EC23F0180EE1263F0E0001FE5DD7
:102B100001E0E6D3CCEC25F090EC24F0070E0DECB0
:102B200026F001E397D045EC22F0020EDDEC22F016
:102B3000FDE1CDEC28F0EF5001E18CD045EC22F026
:102B4000020EDDEC22F0FDE17AEC26F0F00E005CE6
:102B500001E380D045EC22F0020EDDEC22F0FDE135
:102B6000CDEC28F0EE52EF5014E045EC22F0020ECE
:102B7000DDEC22F0FDE17AEC26F045EC22F0020ECD
:102B8000DDEC22F0FDE1CDEC28F0EE52EF50005CE0
:102B90000DE245EC22F0020EDDEC22F0FDE14CEC02
:102BA0002DF0DDEC22F0FDE198EC27F045EC22F071
:102BB000020EDDEC22F0FDE1CDEC28F0020EF9EC86
:102BC00023F016E045EC22F0020EDDEC22F0FDE1F0
:102BD0007AEC26F045EC22F0020EDDEC22F0FDE16D
:102BE000CDEC28F0020EF9EC23F0D88000540DE271
:102BF00045EC22F0020EDDEC22F0FDE14CEC2DF074
:102C0000DDEC22F0FDE1F0EC26F045EC22F0020EC6
:102C1000DDEC22F0FDE17AEC26F0016A74EC2AF09A
:102C2000020EDDEC22F0FDE154EC28F0096A0A6A9C
:102C30000B6A45EC22F0020EDDEC22F0FDE1CDEC5A
:102C400028F0EFCF04F0056AFDEC23F001E264D731
:102C5000DB2A62D78EEC2CF0070EEE1801E03FD194
:102C6000ED5001E03CD135EC24F0E00E2E6E400E2C
:102C700034EC26F03FEC2AF0B6EC84F018EC82F04D
:102C80000DEC29F025EC2BF058EC82F0D2EC28F07A
:102C90002C6A2D6A200E2E6E420E2F6E57EC82F09B
:102CA000B6EC84F029C0C2F90901780EE26F40EC5D
:102CB00024F0E00E2E6E400E5CEC22F005E1010ED9
:102CC000F36E97EC26F0DB6A72EC23F00001715191
:102CD000026E036A23EC26F016E2020EDBCF71F0DF
:102CE000DBCF00F0030EDBCF01F00DEC26F003E3A9
:102CF000800E6D6F08D072EC23F0020E0DEC26F002
:102D000002E3800E6C6FDE6ADD6A90EC24F0070E41
:102D10000DEC26F001E3E3D045EC22F0020EDDECF1
:102D200022F0FDE154EC28F008C029F016EC82F006
:102D300066EC27F0DBCF09F0150EDBCF0AF0160E9C
:102D4000DBCF0BF0170EDBCF0CF0DCEC2AF00CC065
:102D50002FF07EEC2DF0020EDDEC22F0FDE1CDEC4B
:102D600028F0EFCF15F015C029F016EC82F027C03F
:102D700011F028C012F029C013F02AC014F0140E6C
:102D8000DBCF16F0150EDBCF17F0160EDBCF18F0E9
:102D9000170EDBCF19F016C02CF017C02DF018C09D
:102DA0002EF019C02FF043EC85F0010A05E00D6A02
:102DB0000E6A0F6A3F0E04D00D6A0E6A0F6ABF0ECC
:102DC000106E0DC02CF00EC02DF00FC02EF0DAECFE
:102DD00024F003E0BFEC2BF002D095EC23F063EC81
:102DE00024F0800E00016D150CE02BEC2BF009E3B4
:102DF000010EDF5211E0DFCFF3FFFBEC27F0FDE126
:102E00000BD02BEC2BF00BE3010EDF5205E0DFCFF4
:102E1000F3FFFBEC27F0FDE100016D131FD0800EE6
:102E20006C150FE0F0EC22F0020E0DEC26F009E339
:102E3000010EDF5211E0DFCFF3FFFBEC27F0FDE1E5
:102E40000BD0C6EC2BF00AE2010EDF5205E0DFCF1B
:102E5000F3FFFBEC27F0FDE100016C13F0EC22F036
:102E600045EC22F0020EDDEC22F0FDE162EC2DF0EB
:102E7000B9EC29F0EFCF04F004340DE345EC22F077
:102E8000020EDDEC22F0FDE162EC2DF0F9EC23F016
:102E9000FF0DF3500AD045EC22F0020EDDEC22F0DB
:102EA000FDE162EC2DF0F9EC23F0026E036A02BE44
:102EB000036823EC26F00DE245EC22F0020EDDEC77
:102EC00022F0FDE162EC2DF0B9EC29F0060EDBCF2B
:102ED000EFFFDF2A010E01E218D7DB2A16D7000127
:102EE0006251631105E06251605D6351615904E212
:102EF00060C062F061C063F06451651105E060512B
:102F0000645D6151655904E260C064F061C065F0C0
:102F1000CCEC25F090EC24F00E0E0DEC26F001E345
:102F200099D045EC22F0030EDDEC22F0FDE10FEC30
:102F300023F0EE50ED1001E18DD045EC22F0030EB0
:102F4000DDEC22F0FDE1F2EC28F0000E005C0F0E4B
:102F5000015801E37FD045EC22F0030EDDEC22F0B6
:102F6000FDE1D4EC2DF0BFEC25F012E045EC22F0B1
:102F7000030EDDEC22F0FDE181EC2CF0DDEC22F023
:102F8000FDE1D4EC2DF0FCEC25F0C9EC27F00FE2CC
:102F900045EC22F0030EDDEC22F0FDE181EC2CF09B
:102FA000DDEC22F0FDE1D4EC2DF095EC24F045ECC5
:102FB00022F0030EDDEC22F0FDE10FEC23F0040E15
:102FC000BFEC25F013E045EC22F0030EDDEC22F01F
:102FD000FDE181EC2CF0DDEC22F0FDE10FEC23F0C3
:102FE000040EFCEC25F023EC26F010E245EC22F078
:102FF000030EDDEC22F0FDE181EC2CF0DDEC22F0A3
:10300000FDE10FEC23F0040E95EC24F045EC22F0EA
:10301000030EDDEC22F0FDE1F2EC28F074EC2AF076
:10302000030EDDEC22F0FDE1CCEC2BF00A6A0B6A1A
:1030300045EC22F0030EDDEC22F0FDE10FEC23F075
:10304000EECF04F0EFCF05F0FDEC23F001E262D704
:10305000DB2A60D78EEC2CF00E0EEE1801E031D199
:10306000ED5001E02ED135EC24F0600E2E6E410EB5
:1030700034EC26F040EC24F0600E2E6E410E5CEC39
:1030800022F005E1010EF36E97EC26F0DB6A72EC9C
:1030900023F0000100506F5D0150705918E2020EDC
:1030A000DBCF6FF0030EDBCF70F072EC23F0050E78
:1030B0000DEC26F004E3686B800E696F08D072ECAB
:1030C00023F00DEC26F003E3666B800E676FDE6A7B
:1030D000DD6A90EC24F00E0E0DEC26F001E3F1D049
:1030E00045EC22F0030EDDEC22F0FDE1CCEC2BF000
:1030F00008C028F009C029F027EC82F066EC27F020
:10310000DBCF0AF0150EDBCF0BF0160EDBCF0CF089
:10311000170EDBCF0DF00AC02CF00BC02DF00CC049
:103120002EF00DC02FF07EEC2DF0030EDDEC22F022
:10313000FDE10FEC23F0EECF16F0EFCF17F016C045
:1031400028F017C029F027EC82F027C012F028C021
:1031500013F029C014F02AC015F0140EDBCF18F0BC
:10316000150EDBCF19F0160EDBCF1AF0170EDBCFE2
:103170001BF018C02CF019C02DF01AC02EF01BC087
:103180002FF043EC85F0010A05E00E6A0F6A106A21
:103190003F0E04D00E6A0F6A106ABF0E116E0EC089
:1031A0002CF00FC02DF010C02EF0DAEC24F003E06C
:1031B000BFEC2BF002D095EC23F063EC24F000017F
:1031C0006951800B0CE0F0EC22F00DEC26F007E3E7
:1031D00002EC26F010E080EC25F0FDE10CD0F0ECE4
:1031E00022F0060E0DEC26F00CE302EC26F003E0D4
:1031F00080EC25F0FDE100500001681301506913D7
:103200001BD06751800B0AE02BEC2BF007E302EC9C
:1032100026F00DE080EC25F0FDE109D0C6EC2BF0A6
:103220000BE202EC26F003E080EC25F0FDE100501B
:103230000001661301506713F0EC22F045EC22F018
:10324000030EDDEC22F0FDE1E3EC2CF0B9EC29F00B
:10325000EECF04F0EFCF05F00001800E05140EE074
:1032600045EC22F0030EDDEC22F0FDE1E3EC2CF066
:10327000FCEC25F0026C031E03220AD045EC22F080
:10328000030EDDEC22F0FDE1E3EC2CF0FCEC25F08C
:1032900023EC26F010E245EC22F0030EDDEC22F0E8
:1032A000FDE1E3EC2CF0B9EC29F0060EDBCFEEFFEC
:1032B000070EDBCFEDFFDF2A010E01E20AD7DB2A82
:1032C00008D700016A51681906E16B51691903E1D9
:1032D0006E516D5D03E0110E090118130001FE6BC4
:1032E000180EE15C02E2E16AE552E16E0BEF23F0B9
:1032F00006EC23F0080EE126D950FB0FBAEC22F0C1
:1033000002E0A00E01D0C70E006E016A63EC24F04B
:103310001AEC2BF0FFEC22F0E50EE66EE10EE66E05
:10332000000EC7EC28F0A3EC28F00F0E29EC2AF0D1
:10333000A3EC28F0080E41EC2BF003E057EC25F04D
:1033400008D0A3EC28F0060E41EC2BF004E05DEC75
:1033500025F0C7EC28F02EEC24F07DEC2AF084EC6C
:103360002DF0A3EC28F0080EBFEC25F00EE1A3EC45
:1033700028F0060EBFEC25F008E1D50EE66EE10E52
:10338000E66E000EC7EC28F05CD0DE6ADD6A66EC03
:103390002AF002E626EC2CF054E228EC2CF00C0E7D
:1033A000B9EC27F0E8AE02D0033402D0C9EC27F024
:1033B00001E399D0A3EC28F0080E6BEC2AF0DF5063
:1033C0001F0B03E0ECEC24F0FDE181EC23F003E0C3
:1033D00057EC25F010D0A3EC28F0060E6BEC2AF089
:1033E000DF501F0B03E0ECEC24F0FDE181EC23F057
:1033F00023E05DEC25F0C7EC28F045EC22F0030E4D
:10340000DDEC22F0FDE1E3EC2CF029EC2AF0D3EC2A
:103410002BF0CF0EE66EE10EE66E000E8AEC2DF07C
:1034200005E12EEC24F007EC27F004D02EEC24F07C
:1034300082EC26F084EC2DF0DF2A010EA8E3DB2AD3
:10344000A6D728EC2CF0140EB9EC27F0E8AE02D089
:10345000033402D0C9EC27F046E2C20EE66EE10E5C
:10346000E66E000EC7EC28F0A3EC28F0110EF9EC84
:1034700023F0E66ED950020F71EC25F028EC2DF008
:10348000800B03E057EC25F006D0BFEC2DF0800B4D
:1034900004E05DEC25F0C7EC28F02EEC24F07DEC88
:1034A0002AF090EC2DF028EC2DF009E1BFEC2DF086
:1034B00006E1D50EE66EE10EE66E000E19D0DE6A6C
:1034C000DD6A66EC2AF002E63FEC2BF05AE228ECCB
:1034D0002CF0080EB9EC27F0E8AE02D0033402D08D
:1034E000C9EC27F008E3D10EE66EE10EE66E000EA1
:1034F000C7EC28F046D0010EDF5205E0DFCFF3FF26
:10350000FBEC27F0FDE1006E28EC2DF0001403E049
:1035100057EC25F00FD0010EDF5205E0DFCFF3FFAF
:10352000FBEC27F0FDE1006EBFEC2DF0001424E071
:103530005DEC25F0C7EC28F009EC29F062EC2DF0E9
:10354000C3EC25F0016A00BE01685EEC26F0D3EC06
:103550002BF0BD0EE66EE10EE66E000E8AEC2DF04D
:1035600005E12EEC24F007EC27F004D02EEC24F03B
:1035700082EC26F090EC2DF0DF2A010EA2E3DB2A8C
:10358000A0D7080EE15C02E2E16AE552E16E0BEFC2
:1035900023F006EC23F00A0EE126D3EC14F0000928
:1035A00005E1FE0EDB50000801E2AED1D9501FEC60
:1035B0002BF0CD0EEE1830E1ED502EE1DF6A010E5A
:1035C000DF5C01E3A1D14AEC22F0080EBFEC25F04C
:1035D00003E130EC2BF013E0D0EC29F08FEC2BF072
:1035E000DFCFE6FFEEEC27F0016ADF34FE0B013699
:1035F000006E6E0E0026090E35EC2BF00BD0EA6A39
:10360000DF34FE0BEA36E96E6E0EE926090EEA2279
:10361000EE6AED6ADF2AD3D7020EDB6834EC28F0BD
:10362000010EDB6A070E58EC28F02DE2EBEC2AF0D5
:10363000EF50006E016AD950040FF4EC27F0EBEC68
:103640002AF0EE52EFCF00F0020EDB50005C06E2F3
:10365000EBEC2AF0EE52020EEFCFDBFFEBEC2AF0A0
:10366000020EC3EC25F0030EDB50D880005408E2B4
:10367000EBEC2AF0020EB9EC29F0030EEFCFDBFFE2
:10368000010EDB2ACFD7040EDBCF28F0050E13EC9A
:1036900024F0040E28C0DBFF050E29C0DBFFDF6A23
:1036A000010EDF5C01E330D14AEC22F0080EBFECE2
:1036B00025F002E0030E09D04AEC22F0060EBFEC22
:1036C00025F002E0020E01D0010EF36E060EF3CFDC
:1036D000DBFF30EC2BF002E0030E08D04AEC22F0C6
:1036E0003AEC2CF002E0020E01D0010E81EC29F040
:1036F000DF28E66EE66AA50EE66EE10EE66E000EC7
:103700003AEC22F00E0EF8EC2AF0010EE66EE66AB4
:103710007EEC2CF0DCEC2DF07BEC28F07EEC2CF039
:1037200080EC28F07EEC2CF085EC28F07EEC2CF080
:103730004AEC22F0B0EC2CF00FEC2AF0B0EC2CF0BC
:103740001BEC29F04AEC22F0020EAAEC22F00FEC5E
:103750002AF0020EAAEC22F01BEC29F04AEC22F02F
:10376000040EAAEC22F00FEC2AF0040EAAEC22F0D0
:103770001BEC29F0F0EC22F0D9EC2BF0E0EC21F07E
:10378000020E83EC2AF0E0EC21F0030E83EC2AF029
:10379000C3EC2DF00F0E16EC29F0C3EC2DF0110E3A
:1037A000F9EC23F0E66EE66A7EEC2CF0016ADF3479
:1037B000FE0B0136006E700E0026090E35EC2BF064
:1037C000010EDB6A0E0E58EC28F001E39BD04AECA8
:1037D00022F0080E6BEC2AF0DB501F0B03E0ECEC40
:1037E00024F0FDE181EC23F002E0030E11D04AEC5D
:1037F00022F0060E6BEC2AF0DB501F0B03E0ECEC22
:1038000024F0FDE181EC23F002E0020E01D0010E74
:10381000F36E060EF3CFDBFFFFEC27F0016E010E17
:10382000015204E0E846FE0B0106FCE1006E30ECBC
:103830002BF0001402E0030E14D0FFEC27F0016E11
:10384000010E015204E0E846FE0B0106FCE1006EA9
:103850004AEC22F03AEC2CF0001402E0020E01D007
:10386000010E81EC29F0010EDB28E66EE66A940E6B
:10387000E66EE10EE66E000E3AEC22F0DF28F8EC80
:103880002AF0DCEC2DF0010EDB50080DB5EC2CF02D
:10389000F2EC28F0050EC7EC2DF095EC29F0020EA5
:1038A00016EC29F095EC29F0040E16EC29F095ECB5
:1038B00029F0060E16EC29F096EC2DF0EF50D9EC1D
:1038C00029F0EE52EF50D9EC29F0020EF9EC23F07A
:1038D000D9EC29F0030EC3EC25F0016A00BE0168A3
:1038E0006DEC23F0E0EC21F0010E016ADB34FE0BFD
:1038F0000136006E720E0026090E35EC2BF0010E1B
:10390000DB2A60D7DF2ACCD6FE0EDB50006E0A0E13
:10391000E15C02E2E16AE552E16E00500BEF23F058
:103920001DEC2CF019E07CEC25F033DE88EC2AF05D
:10393000A8EC29F003E073EC26F003D0CE0E006E65
:10394000016A6DEC23F007EC2DF076EC29F063ECC6
:103950002CF0EFEC2CF009D084EC27F01ADE88EC88
:103960002AF0020802E02AEC2EF0010ED6EC27F035
:1039700002E2E16AE552E16E00500BEF23F006EC43
:1039800023F00D0EE126FE0EDB500FE00501F3B52E
:103990000CD0A8EC29F003E079EC23F008E1B9ECB5
:1039A00028F003E079EC23F002E1000E03D2D3EC1F
:1039B00014F08EEC23F0E3EC2AF004E078EC25F030
:1039C000200901D0000E64EC28F0DB5009E0010E64
:1039D000E76EDFEC2BF0E750F9EC23F0200901D083
:1039E000000EE76E050EE7CFDBFF040EDB50760A14
:1039F00001E1F4D0020A0FE0060A01E0C7D1F2ECBF
:103A000014F009017D0EFC6FE10EFD6F000EFE6FDC
:103A100054EC3EF0CED1060EDB683FEC28F002EC11
:103A20002CF02CEC2CF002E63FEC2BF030E2B4EC66
:103A300022F0EF50006E016AD950080FF4EC27F025
:103A4000B4EC22F0EE52EFCF00F0060EDB50005C3B
:103A500006E2B4EC22F0EE52060EEFCFDBFFB4EC40
:103A600022F0020EC3EC25F0070EDB50D880005484
:103A700008E2B4EC22F0020EB9EC29F0070EEFCF09
:103A8000DBFF020EDB2A030ECCE3DB2ACAD7080ECB
:103A9000DBCF28F0090E13EC24F04DEC28F01AECE3
:103AA00026F0050EDB5064081CE100016DAF03D069
:103AB00057EC25F004D06CAF04D05DEC25F031EC70
:103AC0002DF000017151E66EE66A7DEC2AF0E66E9B
:103AD0009EEC2CF073EC2CF02CEC29F00DEC27F084
:103AE00024D0E6EC2BF0D9EC2BF07A0EE66EE10E4A
:103AF000E66E000E93EC2BF0060E83EC2AF0760EA9
:103B0000E66EE10EE66E000E93EC2BF0070E83ECF2
:103B10002AF0720EE66EE10EE66E000E93EC2BF0CC
:103B20006E0EE66EE10EE66E000E35EC2DF0DB6AF1
:103B3000030EDB6A2CEC2CF002E63FEC2BF001E3E9
:103B400022D1010EF36E020EDB5004E0D890F33662
:103B5000E806FCE1F35000016D1503E057EC25F099
:103B60000FD0010EF36E020EDB5004E0D890F33656
:103B7000E806FCE1F35000016C1504E05DEC25F073
:103B800031EC2DF0BDEC29F015E13AEC2BF00034CE
:103B90000AE23AEC2BF0016A00BE01686DEC23F0FA
:103BA00007EC27F010D03AEC2BF0016A00AE07D0FA
:103BB000016805D0B4EC22F0EF506AEC24F06DEC13
:103BC00023F082EC26F093EC2BF00DEC27F035EC93
:103BD0002DF0DB2A030EAEE3DB2AACD71AEC26F07D
:103BE000DE6ADD6A66EC2AF002E669EC28F001E3A1
:103BF000CAD0050EDB5064081FE105EC29F0080E61
:103C000041EC2BF003E057EC25F008D005EC29F04F
:103C1000060E41EC2BF004E05DEC25F031EC2DF0CC
:103C200005EC29F00F0E16EC29F07DEC2AF093EC50
:103C30002BF001EC27F011D0020EE66EE66A05ECDF
:103C400029F0B0EC2CF00A0E0EEC2BF07A0EE66E9A
:103C5000E10EE66E000E20EC25F035EC2DF0DB6A6F
:103C6000030EDB6A2CEC2CF002E626EC2CF001E3D0
:103C700084D00B0EDBCF00F00C0EDBCF01F0A00EDA
:103C8000026E060E036E0D0E025E000E035A23EC4A
:103C900026F009E27DEC29F0D1EC58F01E0E10EC74
:103CA0002CF01AEC26F005EC29F0080E6BEC2AF04B
:103CB000020EDB501F0B03E0ECEC24F0FDE181EC85
:103CC00023F003E057EC25F011D005EC29F0060EA7
:103CD0006BEC2AF0020EDB501F0B03E0ECEC24F03F
:103CE000FDE181EC23F004E05DEC25F031EC2DF0FA
:103CF000BDEC29F029E1F3EC29F0DDEC22F0FDE147
:103D0000E3EC2CF0AAEC22F00001800E01140CE18F
:103D1000F3EC29F0DDEC22F0FDE1E3EC2CF016EC05
:103D200029F007EC27F00BD0F3EC29F0DDEC22F0C2
:103D3000FDE1E3EC2CF016EC29F082EC26F093EC9C
:103D40002BF001EC27F011D0030EE66EE66AF3ECDF
:103D500029F0DDEC22F0FDE1F2EC28F0050E0EEC8E
:103D60002BF082EC26F020EC25F035EC2DF0DB2A50
:103D7000030E01E277D7DB2A75D7DF2A010E01E2B5
:103D800031D7DB2A2FD77DEC29F013D00601006B49
:103D9000010EE66EE66A000EE66EEEEC27F014EC1D
:103DA0002CF07DEC29F068C06AF069C06BF06DC042
:103DB0006EF0010E006E0D0EE15C02E2E16AE5526A
:103DC000E16E00500BEF23F006EC23F0FC0EDBCF8E
:103DD00028F0FD0EDBCF29F0CF0E281801E1295085
:103DE00040E0D00E281801E129503BE0CD0E281804
:103DF00001E1295033E0CE0E281801E129502EE0D0
:103E0000CB0E281801E1295025E0CC0E281801E13D
:103E1000295020E0C90E281801E1295017E0CA0EE8
:103E2000281801E1295012E0C80E281801E1295094
:103E300009E0060E28181BE1295019E1C9DBAAEC9C
:103E400011F012D0C5DB37EC0FF00ED0C1DBD7EC90
:103E500011F00AD0BDDBF9EC12F006D0B9DB60DD61
:103E600003D0B6DB7AEC0EF06FEC2AF001D0000E36
:103E7000D2D3CCDB030EE126DE6ADD6A71EC24F0DE
:103E800004BE0568040E13EC27F0FDE183EC24F07A
:103E900001E1E4D0B60E066E3D0E076E010E086E0F
:103EA000DECF09F0DDCF0AF00B6A0ABE0B68040E04
:103EB000D89009360A360B36E806FAE1065009248E
:103EC000036E07500A20046E08500B20056E03C0D5
:103ED000E6FF04C0E6FFE66E4AEC98F088EC2AF0B4
:103EE0009CEC2DF00006000E015A025A6DEC23F0F6
:103EF000B60E0F6E3D0E106E010E116EDECF12F07B
:103F0000DDCF13F0146A13BE1468040ED890123675
:103F100013361436E806FAE10F5012240C6E1050D6
:103F200013200D6E115014200E6E0C2A000E0D225F
:103F30000E220CC0E6FF0DC0E6FF0EC0E6FFF90E34
:103F4000DBCFE6FFFA0EDBCFE6FF2AEC97F0156E2B
:103F5000070EE15E1550000901E07AD0FE0EDB503D
:103F600030E0F70EDBCFE6FFF80EDBCFE6FFDBEC51
:103F700059F0E552E552F70EF3CFDBFFF80EDAEC1D
:103F800027F0F70FE66EFF0EDA20E66EFB0EDBCFB2
:103F9000E6FFFC0EDBCFE6FF71EC24F004BE056803
:103FA000040E13EC27F0FDE183EC24F0E66EB7EC91
:103FB00060F0066E050EE15E0650000902E1000E9B
:103FC0004ED0DECFE9FFDDCFEAFF030EEA02F3CFEA
:103FD000EAFFE902F3CFE9FFF450EA26E40EE9260E
:103FE0000A0EEA22EECF00F0EECF01F0EFCF02F0A2
:103FF000F70EDBCFE6FFF80EDBCFE6FFF90EDBCFE7
:10400000E6FFFA0EDBCFE6FFFB0EDBCFE6FFFC0E92
:10401000DBCFE6FFFD0EDBCFE6FF06D002C0FBFFE5
:1040200001C0FAFF0050F96EF9DF036E070EE15E82
:104030000350E76E020EE7CFDBFFFD0EDB5005E01D
:10404000020EDB5002E0D1EC58F0020EDB5007D03C
:10405000DF2A010E01E212D7DB2A10D7000E006E14
:10406000030EE15C02E2E16AE552E16E0050D3D258
:10407000CDDAFAEC24F0ACDAE66A76EF2BF0C6DAA9
:10408000F90EDBCFE6FFA4DA010EE66EE66E76EF00
:104090002BF01DEC2CF003E10501F3A502D0000E7E
:1040A0003DD00901580EFC6FE10EFD6F000EFE6F52
:1040B00054EC3EF0DE6ADD6A71EC24F004BE056863
:1040C000040E13EC27F0FDE183EC24F026E0090157
:1040D000560EFC6FE10EFD6F000EFE6F54EC3EF0CD
:1040E00071EC24F004BE0568040E13EC27F0FDE12A
:1040F000005003240901FC6F01500420FD6F0250A1
:104100000520FE6FFC2B000EFD23FE2354EC3EF039
:10411000DF2A010ED1E3DB2ACFD7010ED6EC27F040
:1041200002E2E16AE552E16E005075D26FDAE652C2
:10413000520E0501C85D06E1540EC95D03E1CA5186
:1041400001E178D0520EC86F540EC96FCA6BCB6BA9
:10415000CC6B0901400E176F880E036F130E046FAE
:10416000100E056F270E066F096B0A6B0901320EE0
:10417000A06F0901006B0B6F0C6B640E076F086B6F
:10418000016B026B0D6B0E6B156B166B0F6B106B6F
:10419000116B126B136B146B120E9CEC26F0600EFD
:1041A000E66E000E8BDB0001E80E626F030E636F9C
:1041B0001C0E9CEC26F0720EE66E000E7FDBDF6AB2
:1041C000070EDF5C0BE2DF5015DA280EEF6EDF50D2
:1041D00011DAEE52F00EEF6EDF2AF2D7700E9CEC81
:1041E00026F08E0EE66E000E69DBDF6A0E0EDF5CD7
:1041F0000EE2DF50080DB5EC2CF0D4EC2DF0B9EC4C
:1042000029F0D00EEE6E070EED6EDF2AEFD78CECA4
:104210002AF03E6B3F6B96EC2AF0ACEC25F0186B65
:104220000901A56BA66BA76BA86B0901A96BAA6B0B
:10423000AB6BAC6B0001FE6B900E6F6E6EAEFED77B
:10424000606A0F011869E00E196F2A0E006FA00E48
:10425000016F046B056B506BFE0E1C6F1D6BB20E75
:10426000086F096BD20E0C6F0D6BAA0E106F116BDD
:10427000BA0E146F156B706ABF0E716E020E726EFD
:10428000200E736E0501F451000802E26F6A02D03D
:10429000600E6F6E0701C00ECC6F3B0ECD6F010E2E
:1042A000CE6F0701C60ECF6F3B0ED06F010ED16FE0
:1042B0000701340ED56F040ED66F000ED76F0701BD
:1042C000C40ED86F060ED96F000EDA6F0701080E04
:1042D000F06F0F0EF16F000EF26F07010C0EDB6F27
:1042E0000F0EDC6F000EDD6F0701F00EDE6F130E98
:1042F000DF6F000EE06F07010A0EE16F140EE26F30
:10430000000EE36F0B01700E4C6F400E4D6F000EF0
:104310004E6F0B017E0E4F6F400E506F000E516FAF
:104320000B01C80E496F3D0E4A6F000E4B6F060120
:10433000EE81EE83EE85010EE5526DD1F20E002680
:104340002B0EF4EC2BF0E40E2B6E570E2C6EABEC18
:1043500028F0ABEF2CF05BEC2CF0AFEC74F0086EB7
:10436000090E16EC2BF04CEC2AF097EC2CF004C064
:1043700026F068EC29F0040EDBCF2BF0050EDBCF26
:104380002CF0060EDBCF2DF0070EDBCF2EF0E3EC8A
:104390002DF018EC2CF054EC2DF0AA0EE66EE30E86
:1043A000E66E000E5BEC2CF0A0EC74F0086E070ECD
:1043B00016EC2BF0A80EE66EE30EE66E000E120071
:1043C00098EC28F0E66ED5EC2AF076EC29F07EEF3A
:1043D0002BF0E7EC2DF06CEF2DF0120EEA02F3CF8C
:1043E000EAFFE902F3CFE9FFF450EA26600EE9267E
:1043F000000EEA22120098EC28F0FAEC29F0D6EF31
:104400002CF0040EDBCF04F0050EDBCF05F0060E1A
:10441000DBCF06F0070EDBCF07F0D950080FBAEC60
:104420002CF0EE50045C006EEE500558016EEE501C
:104430000658026EEE500758036E110E00C0DBFFE7
:10444000120E01C0DBFF130E02C0DBFF140E03C00F
:10445000DBFFD950040FE96E8FEF29F05BEC2CF0F5
:10446000BDEC74F0046E090E01EF2BF0B5EC28F0F2
:10447000D7EF28F0E66ED5EC2AF073EC2CF07EEF47
:104480002BF071EC74F06FEF2AF0DECFE9FFDDCF97
:10449000EAFF1200DF50120DB5EC2CF0600EE92699
:1044A000000EEA2212000102F3CF01F00002F3CF66
:1044B00000F0F450012612002F6ECBEC2DF03FECF3
:1044C0002AF0140EDBCF2CF0150EDBCF2DF0160EDC
:1044D000DBCF2EF0170EDBCF2FF041EC83F05BEC3F
:1044E00029F057EC82F0100E27C0DBFF110E28C018
:1044F000DBFF120E29C0DBFF130E2AC0DBFFD950F1
:10450000100FBAEC2CF0EECFE6FFEECFE6FFEECFC9
:10451000E6FFEFCFE6FF09EC95F088EC2AF0E552D4
:104520003DEC2CF025EC2BF026C027F0B1EC2AF066
:10453000020E28C0DBFF030E29C0DBFFD950020F9B
:1045400025EF2AF049EC2CF000EC75F0006E070E18
:1045500028EF29F0B9EC29F0B0EF2CF09EEC2CF00C
:1045600076EC29F02CEF29F0F3EC29F0A3EC2DF0F8
:10457000CDEF28F0E96EFF0EDA20EA6EEE50ED1076
:10458000120007C928F008C929F027EC82F00DECC9
:1045900029F005C928F006C929F03DEC29F0CBEF38
:1045A0002DF049EC2CF076EC29F063EF2CF0FAECCE
:1045B00029F0046E090EBDEF2AF0D890E936EA36EC
:1045C000E806120089ECA7F022C000F0EDEF2BF016
:1045D000ECEC29F0E5EC29F0FE0EDBCFE6FF120053
:1045E000040EDBCF00F0050EDBCF01F01200E66E0B
:1045F000B8EF2BF0040DB5EC2CF0CDEF28F0060E43
:10460000F3CFDBFF070EF4CFDBFF1200D9CFE6FFBD
:10461000E1CFD9FF1200E552E7CFD9FF12008E0E8D
:10462000E926000EEA221200B1EC2BF029EC82F010
:104630000DEC29F007EC2CF03DEC29F041EC83F077
:10464000D2EC28F07FEC2BF0EEEC82F0DDEC84F085
:1046500028C0A1F929C0A2F91200ACEC29F0F1ECB4
:10466000A7F0050E2626000E27222822292259EF20
:104670002BF0000EE66E060EE66E1200F0C504F09A
:10468000056A066A076A100E2B6E270E2C6E2D6ABD
:104690002E6AF0C526F068EC29F008C02BF0DCEC9F
:1046A0002AF0EEEC83F026C002F027C003F0B6EC4F
:1046B0002DF052EC00F021EF2AF0D950150FE96EE1
:1046C0008FEF29F036EC2AF0C2EC2CF0020EF62621
:1046D000000EF722F8220800120000C0E6FF01C019
:1046E000E6FF1200020EDBCF00F0030EDBCF01F07D
:1046F0001200FC0EDBCFE9FFFD0EDBCFEAFFEF502F
:1047000012000450001605500116065002160750FC
:10471000031600500110021003101200E5EC29F0FE
:10472000AAEC58F0E552E5521200060EDBCF00F07D
:10473000070EDBCF01F01200DEEC2CF007C027F0F3
:1047400008C028F009C029F06DEC84F024C007F0FF
:1047500025C008F026C009F004502424F36E05504B
:104760002520F46E065026209DEC29F00800F5CF98
:1047700002F002C003F0026AD20E0A6E3B0E0B6E0C
:10478000010E0C6EE2CA0DF0E3CA0EF00F6A1200C1
:10479000100EE66E270EE66E52EC00F021EC2AF0C9
:1047A00031EF2CF001C029F066ECA8F028C000F031
:1047B00029C001F01200DEEC2CF00DC027F00EC075
:1047C00028F00FC029F06DEC84F024C00DF025C056
:1047D0000EF026C00FF00A502424F36E0B50252053
:1047E000F46E0C5026209DEC29F096EC2BF0C1EFD6
:1047F0002AF0B9EC29F0EF501200066A076A93EC30
:104800002CF008C02BF0DCEC2AF089ECA7F0EDECE2
:104810002BF0D9500C0FBAEC2CF0225087EC2BF077
:10482000DF2A010E1200DBCF29F029EC82F00DEC1B
:1048300029F02C6A2D6AE00E2E6E400E2F6ECBEC06
:104840002DF025EC2BF058EC82F0DDEF84F0002603
:10485000000E012254EC2DF0ABEF2CF0020EDBCF5A
:10486000E6FF030EDBCFE6FF12004CEC2AF093ECE0
:104870002CF03CEC82F0D2EC28F02C6A2D6A12006D
:104880000C0EDBCF08F00D0EDBCF09F00E0EDBCFE8
:104890000AF00F0EDBCF0BF008C026F09DEC2BF0DA
:1048A0003CEC82F00DEC29F02C6A2D6A12003DECF4
:1048B0002DF0E76EFE0EE7CFDBFF1200E66E74EC24
:1048C00097F06FEF2AF0040E00C0DBFF050E01C069
:1048D000DBFF1200006E016A280E005E000E015A16
:1048E0001200B60E006E3D0E016E010E026EDECF9E
:1048F00003F0DDCF04F0056A120049EC2CF0B1ECB6
:104900002DF0BDEF2AF000500324F36E0150042077
:10491000F46E025005209DEC29F00800F5501200BD
:10492000DECF00F0DDCF01F01200B9EC29F000C0BD
:10493000EEFF01C0EDFF1200026A036A010E046E71
:10494000056A066A076A120003C0DBFF290EE96EDA
:10495000090EEA6E1D51EE24006E1E51EE20016E0E
:104960001F51EE20026E2051EE20036E35510026BD
:10497000365101223751022238510322120003C05E
:10498000DBFF2D0EE96E090EEA6E2151EE24006E5A
:104990002251EE20016E2351EE20026E2451EE20B2
:1049A000036E395100263A5101223B5102223C51FB
:1049B000032212002F6E00C027F0B1EC2AF0CEECDB
:1049C0002AF0060E070EDBCF03F00001800E031461
:1049D0001200005087EF2BF0D890043605360636CB
:1049E0000736E8061200E66EE66AFEEC3EF0E55297
:1049F000E5521200F80EDBCFE6FFF90EDBCFE6FF43
:104A00001200F3CFE6FF01C0E6FF1200250EE96EAB
:104A1000090EEA6E09011951EE24006E1A51EE20BA
:104A2000016E1B51EE20026E1C51EE20036E3151BF
:104A30000026325101223351022234510322120046
:104A4000E66E9EEC2CF0B1EC2DF0E15E04502CEC07
:104A500029F06B0EE66EE10EE66E000E120002C04B
:104A6000E6FF03C0E6FF12002C6E68EC2CF0EEECC3
:104A700083F027C001F08EEC2CF02650EE2601507A
:104A8000ED221200DBCF0AF0030E0926000E0A22E7
:104A90000B6A00500924F36E01500A20F46E025094
:104AA0000B209DEC29F00800F550E66E1200E30E95
:104AB000E66EE10EE66E000E1200E10EE66EE10E0D
:104AC000E66E000E1200C1EC2AF0A4EC2BF0D950D7
:104AD000010FBAEC2CF0000ED880EE54000EED540D
:104AE0001200BAEC2CF0E552E750EE6EED6A1200BF
:104AF000DFEC2BF0EF501200E5EC29F0E66A120033
:104B0000D8900036013602360336E8061200FA0E57
:104B1000DBCFE9FFFB0EDBCFEAFF1200E66E63ECB2
:104B20009FF088EF2AF0A3EC3EF0E552E552120028
:104B3000DEEC2CF006C027F007C028F008C029F0F2
:104B40006DEC84F003502424006E04502520016E87
:104B500005502620026E1200626B636B646B656BFE
:104B6000666B676B686B696B120078EC89F021EFFC
:104B70002AF0050E005E000E015A040E1200F9DB49
:104B8000EE50ED101200F5DBEFCF00F01200D890E0
:104B900000360136E8041200080EDB6A090EDB6AF3
:104BA00005EC2BF00E0EDB6A0F0EDB6ADE6ADD6AA7
:104BB00012003D510C0DB5EC2CF0190EE926090E32
:104BC000EA221200000E005E060E015AB6EF2AF02D
:104BD000FD0EDBCF00F0FE0EDBCF01F0120049EC42
:104BE0002CF0C8EC98F0026E050EE15E0250CFEC9E
:104BF0002DF0F350F4101200BCDBEECF02F0EFCF3B
:104C000003F01200010E006E016A026A036ADF50AF
:104C10001F0B120021DB020E120039EF2DF0D6EC33
:104C20002CF0D5C9E6FFD6C9E6FFD7C9E6FFD8C93B
:104C3000E6FF1200D9500B0FBAEC2CF0000EEE6E0E
:104C4000060EED6E12000050025C01500358120077
:104C5000A5EC2CF0CDC926F0CEC927F0CFC928F09D
:104C6000D0C929F0F1EFA7F02F6EEEEC82F0140E10
:104C700027C0DBFF150E28C0DBFF160E29C0DBFFA7
:104C8000170E2AC0DBFF1200FD0EDBCF28F0FE0E50
:104C9000DBCF29F00351285C006E04512958016EC6
:104CA000026A036A1200EF51640DCFEC2DF031EC73
:104CB0002CF052EC00F0E552E5521200020E00C05A
:104CC000DBFF030E01C0DBFF1200D20E006E3B0EB5
:104CD000016E010E026E1200060EDBCF02F0070E0F
:104CE000DBCF03F01200FC0EDBCF00F0FD0EDBCFBC
:104CF00001F0120052DAEFCF00F012003ADBEE6A58
:104D0000ED6A1200CA0EE66EE10EE66E000E1200AB
:104D100000500008000E01541200D89001320032F9
:104D2000E8041200010E0026000E01221200020EFD
:104D3000F3CFDBFF030E1200E66EE66AE66A1200AE
:104D4000D6EC2CF0DBC9E6FFDCC9E6FF12000FC988
:104D50005CF910C95DF911C95EF912C95FF9DBC9C7
:104D600060F9DCC961F91200E6EC2BF00A0EDBCF2A
:104D700002F00B0EDBCF03F0120009015C6B5D6BE0
:104D80005E6B5F6B606B616B1200E126D9501FEFA9
:104D90002BF0D20E046E3B0E056E010E066EE2CABB
:104DA00007F0E3CA08F0096A1200D20E036E3B0E48
:104DB000046E010E056EE2CA06F0E3CA07F0086A47
:104DC000120049EC2CF071EC74F0036E050EE15EFC
:104DD000035012007FEC2BF041EC83F0DDEF84F008
:104DE000DCD9020EC6DA36EF2CF0DB503F0B006E3A
:104DF0003D0E005C1200000ED8800B55000E0C55C5
:104E00001200D90EE66EE10EE66E000E1200CC0E18
:104E1000E66EE10EE66E000E1200BF0EE66EE10ECB
:104E2000E66E000E1200D890033604360536E8060A
:104E3000120015C900F016C901F0006C011E000E29
:104E40000122026A036A1200060E00C0DBFF070E91
:104E500001C0DBFF120015C900F016C901F0026A9B
:104E6000036A1200010EDBCF00F0020EDBCF01F06F
:104E700012000F0E0B014215016E006A4351120021
:104E80000F0E0B014515016E006A46511200020E0D
:104E9000DBCF02F0030EDBCF03F0120023EC98F01F
:104EA0006FEF2AF066DAEF6A1200DBCFEAFF410EFD
:104EB000E9260B0EEA2236EF2CF08FEC2BF0E66E93
:104EC000E66AE66EE66A010EE66E1200A6D9140ED8
:104ED0001200D1C9E6FFD2C9E6FFD3C9E6FFD4C9A3
:104EE000E6FF120003C905F904C906F90BC907F961
:104EF0000CC908F912000FC926F010C927F011C912
:104F000028F012C929F0120060DA020EE66E1200D3
:104F10000FC9E6FF10C9E6FF11C9E6FF12C9E6FF97
:104F2000120031EC2CF06AEC01F0E552E55212006F
:104F300034D9EE5236EF2CF00B014451006E016A69
:104F4000040E1200CCDA090112008DEC0DF088EF8E
:104F50002AF0CEEC97F088EF2AF03AEC2EF0FE0E15
:104F6000DB5002081200840EE66EE20EE66E000EC2
:104F70001200025E000E035A015003181200025084
:104F80000008000E03541200E66E58EC72F0E55271
:104F900012000250005C0350015812001CEC9FF0FC
:104FA000E55212004D0E0701CB5D1200006E020E9D
:104FB000E15C1200F4CFDBFFD9501200010EDBCF11
:104FC00003F0020EDBCF04F0056A1200010E0901A6
:104FD0000024A36F000E0120A46F1200E66A78EC93
:104FE00019F096DAE5521200BAEC2CF00050EE26D9
:104FF0000150ED221200E846FE0BF3061200010EEE
:10500000DB407F0B12000C0EDBCF02F00D0EDBCF6E
:1050100003F012000A0EDBCF00F00B0EDBCF01F025
:105020001200030EF3CFDBFF040EF4CFDBFF120000
:1050300013C900F014C901F0026A036A12000C0ED1
:10504000DBCF00F00D0EDBCF01F01200D890033261
:10505000023201320032E806120078EC89F0E552A3
:10506000E552F3CFF1F51200030EDB6A040EDB6AA2
:10507000050EDB6A1200E3ECA3F06FEF2AF0070ED7
:10508000DB6A080EDB6A090EDB6A1200F80EDBCF62
:1050900028F0F90EDBCF29F01200080E28C0DBFF44
:1050A000090E29C0DBFF120078D8EFCF08F01200FC
:1050B000F36E010EDBCFF4FFF350F45C12004151AC
:1050C000006E016A040E1200E76E040EE7CFDBFFEC
:1050D0001200010E39EF2DF044C9E6FF45C9E6FF85
:1050E000120052C9E6FF53C9E6FF12005FEC74F0EC
:1050F000E552E552120003C9E6FF04C9E6FF1200BB
:1051000005C9E6FF06C9E6FF120009C9E6FF0AC99C
:10511000E6FF1200000EDE6E060EDD6E1200020EBD
:10512000E126FE0EDB501200090EDB503F08120094
:105130002E0EE66EE40EE66E000E1200AADB41ECC7
:1051400022F063EF2CF0FD0EDBCFE9FFFE0EDBCF8C
:10515000EAFFEDEF21F0BCDBE3EC2DF0B6EF2DF034
:10516000AADB41EC22F077EF2CF0A5DBBCDB77EF7C
:105170002CF0E66A13DFFC0EF3CFDBFFFD0E1ADF27
:10518000FC0FBAEF22F0E66ED9DB41EF22F0F7EC2C
:1051900022F041EC22F0FFEF22F0720EE926000E21
:1051A000EA2212009CEC2DF02AC003F01200110E2E
:1051B000DBCF04F0120EDBCF05F0130EDBCF06F0D1
:1051C000140EDBCF07F0AFDB150EDBCF2BF0160E86
:1051D000DBCF2CF0170EDBCF2DF0180EDBCF2EF02F
:1051E000E3EF2DF00FEC23F0B0EF2CF09EEC21F06C
:1051F000090EE66EE40EE66E000E2EEF22F0F2ECE3
:105200002DF041EC22F063EF2CF045EC22F0EDEFB5
:1052100021F045EC22F0A3EF2DF027C004F028C0C8
:1052200005F029C006F02AC007F01200AAEC22F00F
:10523000050EC7EF2DF00A0E53EC22F00E0E2D6E68
:105240002E6AF3CF28F0D2EC23F085DBE0EF21F0DB
:10525000E15E005063EF2CF00B0EF3CFDBFF0C0E82
:10526000F4CFDBFF1200E66EE9EF21F02C6E2D6A21
:105270002E6AE2EC22F09EEF21F027EC82F027C0AC
:1052800008F028C009F029C00AF02AC00BF0CEDBD4
:1052900004C027F005C028F006C029F007C02AF096
:1052A00012002B6E2C6A14DBE2EF22F0F7EC22F0F6
:1052B0001ADBFFEF22F027C00CF028C00DF029C048
:1052C0000EF02AC00FF0B2DB00C027F0AAEF2DF0DD
:1052D000FAEC2DF089ECA7F022C004F023C005F011
:1052E00024C006F025C007F01FEF2DF0A0EC74F0ED
:1052F000026E070EE15E0250120039EC23F093EFCC
:1053000025F0F36E070EF3CFDBFFB60EE66EE10E6F
:10531000E66E000EF2EC2DF041EC22F0CCD3DACFA9
:10532000EAFFD880000E44EF2DF0E0EC21F0010EF2
:10533000DB50080D1ADB0FEF23F0F86EF4CFF7FF08
:10534000F3CFF6FF12000A0E53EC22F0B9EF25F06E
:10535000D950FC0FBAEF22F072DBDFCF2BF0010E39
:10536000DBCF2CF0020EDBCF2DF0030EDBCF2EF0C7
:105370001200E926000EEA221200010EE76E72EC1E
:1053800023F0E7500026000E01226DEC23F0E66AC0
:10539000E66AE66AAEEC22F0050EDB506408120005
:1053A000470EE66EE30EE66E000EF2EC2DF04EEFC9
:1053B00027F06AEC24F06DEC23F096EF2DF02D6EC3
:1053C0002E6A00C028F0D2EF23F0FC0EDBCFE6FF00
:1053D000FD0EDBCFE6FF1200FA0EDBCFE6FFFB0E81
:1053E000DBCFE6FF1200020EDBCFE9FF030EDBCFBF
:1053F000EAFF12004EDABDEF74F09EEC21F0F00EE1
:10540000E66EE30EE66E000E2EEF22F06DEC23F05A
:105410003F0EE66EE30EE66E000ED1EF22F00A0EAE
:10542000B6DBC3EF2DF0F0EC22F056DC9EEC21F061
:105430000C0EE66EE40EE66E000E2EEC22F0B4EFDB
:1054400026F0E552E552CFEF2DF094DAEE50ED1054
:105450001200AAEC22F0050E0102F3CF01F00002C7
:10546000F450012664DC01C0DBFF1200A7DA03C0A0
:1054700027F004C028F005C029F06DEF84F0140E69
:10548000DBCF27F0150EDBCF28F0160EDBCF29F08F
:10549000170EDBCF2AF01200080EDBCF04F0090E46
:1054A000DBCF05F00A0EDBCF06F00B0EDBCF07F0EB
:1054B0001200E66EE66A3B0EE66EE30EE66E000E46
:1054C000120006EC23F0020EE126120090EC24F00C
:1054D000D89001501200AAEC22F09CEF24F0006E4C
:1054E000050EE15E00501200026A036AD950080FEF
:1054F00041DAE9EC24F045EF22F0DD0EE66EE10E34
:10550000E66E000E1200DB506AEC24F06DEF23F023
:10551000E552E552E5521200240E0EDC190EE66E3D
:10552000090E5EEC24F009013D6B12001C0E04DC38
:10553000400EE66E090E5EEC24F0BDEF26F044C985
:1055400000F045C901F0026A036AC6DD2FEF25F0BD
:1055500052C900F053C901F0026A036AC2DD2FEF9D
:1055600025F0F8DA58EC82F0DDEF84F0040EDBCFA2
:1055700002F0050EDBCF03F01200E15E045063EF92
:105580002CF000010224006E000E0320016E1200B8
:105590009CEC26F0E66AE66AE9EF21F0060E28C0E8
:1055A000DBFF070E29C0DBFF1200080EDBCFE6FF92
:1055B000090EDBCFE6FF120009C02CF00AC02DF067
:1055C0000BC02EF01200D950F80FBAEF22F0D950CC
:1055D000FA0FBAEF22F0010EDB50FAEF22F09EEC48
:1055E00021F0CB0EE66EE30EE66E000E2EEF22F0FB
:1055F000E66EE66A300EE66EE40EE66E000E3AEFF8
:1056000022F0E15E045077EF2CF00A0EDB6A0B0EFD
:10561000DB6A0C0EDB6A0D0EDB6A120053EC22F023
:10562000026A036A01EC25F02FEF25F0E15E0850D5
:1056300077EF2CF0E66A39EC23F0A9EF27F0FC0FA6
:10564000E96EFF0EDA20EA6E12002C6A2D6A2E6ACD
:105650003F0E2F6E1200F0EC22F0030E0DEF26F03D
:105660004AEC22F00D0EF9EF23F001226DEC23F04D
:1056700057EF24F0B4EC22F0030EC3EF25F0070E31
:10568000F8D1AAEC22F00150800B1200E8EC25F0D2
:1056900009010050035D015004591200FAD8F9EFD6
:1056A00075F065EC26F0E2CA03F0E3CA04F0056A7F
:1056B00012004BD9F1EFA7F0810EE66EE30EE66E15
:1056C000000EABEF21F0E5D84CEF75F0E76E87ECFC
:1056D00025F0E750F9EC23F03F081200FFEC22F030
:1056E00072EC23F00001800E0114120039EC1FF05F
:1056F000006E080EE15E00500BEF23F0DCD12C6A47
:10570000400E2D6E1C0E2E6E460E2F6E1200EE26D3
:105710000150EE220250EE220350EE221200000E43
:10572000E66EE66A1200E66EAEEF22F0F62A000E92
:10573000F722F8220800F550120009C027F00AC02D
:1057400028F00BC029F01200010E00C0DBFF020E92
:1057500001C0DBFF12009CEC26F090EC1CF0A2EFE5
:1057600027F0040EDBCF28F0050EDBCF29F0120066
:10577000060EDBCFE6FF070EDBCFE6FF120095EC4F
:1057800023F0006C011E000E01221200F0EC22F04A
:1057900047EC27F023EF26F00FEC23F0EECF08F0D4
:1057A000EFCF09F0120090EC24F092EC26F06DEFB0
:1057B00023F0280E005E000E015A6DEF23F0F80E64
:1057C000DBCFE9FFF90EDBCFEAFF1200080EDBCFDB
:1057D00000F0090EDBCF01F0120023C001F024C05D
:1057E00002F025C003F012000122000E0222032263
:1057F00012006DEC23F02FEF25F006EC23F0050EE0
:10580000E1261200020EDB6A030EDB6A120003C9F6
:1058100028F004C929F01200E2EC22F02DEF23F069
:10582000C4EC27F08EEF23F039EC23F076EF28F06C
:10583000050E0026000E0122120006EC23F08FEF69
:1058400028F097EC26F0F4CFDBFF12000E0E11D1FA
:1058500095EC23F0E2EF25F072EC23F0D8900150A4
:105860001200F3CFE6FFF4CFE6FF1200E552E75057
:10587000EF6E12000C0EF9EF23F026C000F027C0E7
:1058800001F028C002F029C003F0120051DC33EF10
:1058900029F0E66EE7EF2DF036EC22F0100E2B6EBD
:1058A000270EE4DC9C0EE66EE30EE66E000EABEC1B
:1058B00021F0B0EF28F0E66E0F0EDBCFE6FF100E02
:1058C000DBCFE6FF1200F3CFDEFFF4CFDDFF1200E7
:1058D0002D6A2E6A00C026F001C027F002C028F011
:1058E00003C029F01200A0EC74F001EF2EF00F0EAF
:1058F000F3CFDBFF100EF4CFDBFF120019DC3AEF21
:1059000022F070DC45EC22F0030E1200410EE66E30
:10591000E30EE66E000E73DCA8EF29F0D9CFE9FFA5
:10592000DACFEAFF120004C026F0FAEF2DF0E80EFD
:105930002B6E030E2C6E2D6A2E6A12000B0EDBCF1F
:10594000E6FF0C0EDBCFE6FF12000A0E2B6E2C6A70
:105950002D6A2E6A120028C0E6FF29C0E6FF120059
:10596000EECF00F0EFCF01F01200F3CFE9FFF4CF5C
:10597000EAFF1200E96EDACFEAFF1200DBCFE6FFA2
:10598000E66A120000502424F36E01502520F46EC4
:10599000025026209DEF29F0320E0901016A0D25E3
:1059A000006E0E510122640EDFEF29F0006E090E29
:1059B00028EF29F098EC28F0D7EF22F00B0E2C6E90
:1059C0002D6A2E6A12000FEC23F0060E120036EC40
:1059D00022F0E80E2B6E030E49DC5CEF2BF04F0E2D
:1059E000E66EE30EE66E000E9EEC28F03AEF2EF027
:1059F00021C900F022C901F023C902F024C903F033
:105A0000120012DF020E0CDF78DC010E1200520EC3
:105A1000E66EE30EE66E000EF2EF2DF009EC29F0D3
:105A2000CDEC28F0EF50E66E09EF29F027C02CF0FE
:105A300028C02DF029C02EF02AC02FF0120022C05D
:105A400026F023C027F024C028F025C029F012003A
:105A5000A3EC28F00D0EF9EF23F052EC27F005EF40
:105A600029F0C3EC28F02CEF29F0C3EC28F00AEF62
:105A700026F0005C000E01581200FE0EDBCFE6FFA0
:105A800034EC2FF088EF2AF0EE54000EEE54000EA6
:105A9000EE54000EEE541200CDEC28F0EF50E66EFE
:105AA00045EC22F0020E1200022203220A0E2B6E97
:105AB0002C6AABEF28F0080EF3CFDBFF090EF4CF12
:105AC000DBFF1200CDEC28F0030E12000BC900F032
:105AD0000CC901F0A3EF29F0A0EC74F0006E070EE2
:105AE00028EF29F0E66EE66A98EC28F0A2EF22F0A3
:105AF000D1EC22F0B3EC27F09EEF28F057EC82F0C7
:105B0000D2EC28F045EF22F056EC29F001EC27F01A
:105B1000C7EF28F0F7EC22F076EC29F06EEF2BF0CF
:105B200056EC29F00DEC27F0C7EF28F0E0EC21F05F
:105B3000FFEC27F0FAEF22F027C000F028C001F0B8
:105B400029C002F01200D890E936EA36D890E9363A
:105B5000EA36120001C028F002C029F003C02AF082
:105B6000120092EC75F0046E0B0E120026C0E6FFD8
:105B700027C0E6FF12007EEC26F005EF29F0A3EC2B
:105B800028F03AEF2CF0E0EC21F04AEF22F053EC51
:105B900022F001EF25F0EEEC82F0D2EF28F0F3CF07
:105BA00000F0F4CF01F012000FEC23F0020E12000F
:105BB000E66EE66A46EF2CF0060EE0DE9FDE070E8C
:105BC000DDDE7EEF2CF0F1ECA7F03DEF2CF0DECF28
:105BD000E6FFDDCFE6FF12002BDE0A0EDFEC29F038
:105BE000ABEF2CF0E66E39EF23F005EC29F0B8DED0
:105BF00005EF29F005C027F006C028F007C029F0FE
:0C5C00001200006E070EE15E0050120062
:045C0C000A019E6B80
:105C10009F6B12000A015D6B12007F0E0601C85DCA
:105C200008E10901CE0EFC6FDC0EFD6F000EB2EF35
:105C30003AF00A01010E5E6F050EE1EC3BF009013E
:105C4000C20EFC6FDC0EFD6F000EB2EC3AF00A0ED5
:105C5000E1EF3BF07F0E0601C85D04E10901FAECBB
:105C60003AF006D00901BD0EFC6FDC0EFD6F000E90
:105C7000B2EF3AF07DEC3CF07F0E0601C85D05E125
:105C800078EC3BF0A3EC3EF05AD00A018D0549E1D7
:105C9000450E0601055D45E0410E055D42E0610EE1
:105CA000055D3FE0670E055D3CE0500E055D39E0A7
:105CB000020E05C6DBFF060EE66E060EE66E000E51
:105CC000E66E050E14EC3BF0DCEC39F019EC3AF022
:105CD00002E600EC3BF005E2EFEC3BF0F7E3DB2AF9
:105CE000F5D7000EE66E050EE66EEAEC3CF0000E0F
:105CF000E66E050E6CEC39F0B50EE66EDC0EE66E67
:105D0000000E5FEC39F0020EDBCF07F6080EE66EF0
:105D1000060E00EC3DF0000EE66E050EE66E2BEC76
:105D20003BF078EC3BF0EAEC3CF013EC3AF06CEC36
:105D30003BF078EC3BF06FEC90F0E552E552E55229
:105D4000E5520901FAEC3AF0B2EC3AF0030EE15CEC
:105D500002E2E16AE552E16E68EF39F063EC39F096
:105D6000050EE126D650016E006A030E00C0DBFF6F
:105D7000040E01C0DBFFD75092EC3AF0DF6A080E48
:105D8000DF5C0BE2DF50EA6A410FE96E0B0EEA229C
:105D9000EF5092EC3AF0DF2AF2D7030EDBCFE6FFAA
:105DA000040EDBCFE6FF07EC8CF0E552E552DF6A2C
:105DB000160EDF5C11E26EEC39F004BE05682CECC7
:105DC0003AF0DF50EA6A5F0FE96E0A0EEA22E55206
:105DD000E750EF6EDF2AECD70A01756B090E27EC4E
:105DE0003CF0CAEC39F0D80EE66E040EE66ECEEC4E
:105DF00039F0F7EC3CF0CEEC39F0160EE66EE66AC0
:105E000005EC3BF00DECA1F0026E0A0EE15E0250D3
:105E10000901AD0EFC6FDC0EFD6F000EB2EC3AF026
:105E200005EC3BF084EC3AF03DEC3CF024EC3AF02D
:105E30006FEC90F02CEC3CF009013DEC3CF0080ECE
:105E400027EC3CF0CAEC39F0CEEC39F084EC3AF0B7
:105E5000FAEC3AF0B2EC3AF0050EE15C02E2E16AEB
:105E6000E552E16E68EF39F0CEEC3BF078EC3BF0B8
:105E7000F7EC3CF078EC3BF00FEC74F0E552E552B7
:105E8000C6EC39F0FE0EDB50020A11E0030A03E013
:105E9000010A1EE109D07AEC3AF032EC3BF003E162
:105EA000DE52DD50011814E011EC3CF011D07AEC18
:105EB0003AF032EC3BF003E1DE52DD50011808E02D
:105EC000ACDE11EC3CF0010EF36EFE0EF3CFDBFF07
:105ED000FE0EDB50006E020EE15C02E2E16AE5526A
:105EE000E16E005068EF39F081EC3CF0020E27ECD7
:105EF0003CF0E1EC3AF0A40EE66EDC0EE66E000E2D
:105F000025EC39F082EC3BF06CEC3BF066EC3BF0BE
:105F1000E66E020EDBCFE6FF030EE4EC3AF082EC15
:105F20003BF08EC9E6FF8FC9E6FFFCEC38F00901B3
:105F30009051E6EC3BF0090194510F0A20E0020A6F
:105F400018E0090A10E0060A08E0030A1EE1980EAC
:105F5000E66EDC0EE66E000E1DD0900EE66EDC0ED8
:105F6000E66E000E17D08A0EE66EDC0EE66E000EB0
:105F700011D0810EE66EDC0EE66E000E0BD0780EB0
:105F8000E66EDC0EE66E000E05D06F0EE66EDC0EE1
:105F9000E66E000E04EC3AF009019651040A18E08E
:105FA000070A10E0020A08E0010A18E1650EE66E31
:105FB000DC0EE66E000E14D05C0EE66EDC0EE66EB5
:105FC000000E0ED0550EE66EDC0EE66E000E08D00A
:105FD000480EE66EDC0EE66E000E02D066EC3BF07C
:105FE00004EC3AF0FEEC39F04D080FE1A1C9E6FFF0
:105FF000A2C9E6FFFCEC38F0A3C9E6FFA4C9E6FF9E
:10600000B6EC3CF089EC3BF01AD0A1C900F0A2C973
:1060100001F0040E0AEC3BF0FDE12BEC39F041EC11
:1060200039F082EC3BF0A3C900F0A4C901F0040EE2
:106030000AEC3BF0FDE12BEC39F041EC39F082EC5D
:106040003BF009019151E6EC3BF092C9E6FF93C9A0
:10605000E6FFFCEC38F009019751E6EC3BF0090152
:106060009851E6EC3BF009019551E6EC3BF0090153
:106070009451E6EC3BF009019651E6EC3BF0DDC9AA
:1060800000F0016A00BE0168EFEC3CF0DEC9E6FFFB
:10609000DFC9E6FFFCEC38F0E5C900F0016A00BE9C
:1060A0000168EFEC3CF05DEC3AF0B6EC3CF0C0EC93
:1060B0003AF082EC3BF08E0EE66E0A0E48EC39F0B8
:1060C000040EE15C02E2E16AE552E16E005068EF25
:1060D00039F0CEEC3BF0E8EC3AF0410EE66EDC0E27
:1060E000E66E000EBAEC3CF099EC39F09AEC3CF01C
:1060F00000BE016814EC39F0900EE66E0A0E85ECD5
:106100003CF002E2E16AE552E16E005068EF39F0DE
:1061100063EC39F0070EE1263A0EE66EDC0EE66E11
:10612000000EFBEC39F0CAEC39F0DF6A040EDF5CDC
:106130006FE239EC3BF0EFCF00F0000EE76E001895
:10614000E8AE02D0003403D0E750D880005452E2C9
:10615000DF50EA6AC70FE96E090EEA22EFCF04F0BA
:1061600004C029F016EC82F027C000F028C001F02E
:1061700029C002F02AC003F0560E2C6E0E0E2D6EB2
:106180008D0E2E6E3E0E2F6EEEEC82F00CEC85F036
:10619000030E26C0DBFF040E27C0DBFF050E28C060
:1061A000DBFF060E29C0DBFF010EE66EE66AD95062
:1061B000030F9CEC3AF0E66AE66AE66ACEEC39F048
:1061C00092EC75F0006E0B0EE15E0050CAEC39F0F7
:1061D00039EC3BF0EF50D80F006E016A00BE016849
:1061E000EAEC3BF066EC3BF0E66EF3EC3CF066EC80
:1061F0003BF005D0350EE66EDC0EE66E000EE66E68
:10620000CEEC39F0CBEC3BF0CAEC39F0DF2A8ED77C
:10621000E4C900F0016A00BE0168EAEC3BF0E66AFE
:10622000E66AE66AF3EC3CF0920EE66E0A0E48EC83
:1062300039F0070EE15C02E2E16AE552E16E0050DE
:1062400068EF39F07DEC3CF0010EF36E020EF3CFF7
:10625000DBFFF36EDB6EB5EC3AF02E0EE66EDC0E75
:10626000E66E000EDFEC3CF00F0EF66E000EF76EE1
:10627000000ED8EC39F0100EF66E000EF76E000E20
:10628000D8EC39F009EC3AF06CEC3BF040EC3BF028
:106290007DEC3BF0020E19EC3CF000EC3DF0FAEC2A
:1062A0003CF0AE0EE66E090E94EC39F00901E951AE
:1062B000ACEC3BF00501F451ACEC3BF0C80EE66EE3
:1062C000050E94EC39F0EC0EE66E090E94EC39F004
:1062D000940EE66E0A0E48EC39F0030EE15C02E221
:1062E000E16AE552E16E005068EF39F063EC39F095
:1062F000060EE1260901A951AA11AB11AC1109E161
:10630000020EDB6A030EDB6A040EDB6A050EDB6A33
:106310001DD0A90EE96E090EEA6EEE500901A55DC9
:10632000006EEE50A659016EEE50A759026EEE5067
:10633000A859036E020E00C0DBFF030E01C0DBFF95
:10634000040E02C0DBFF050E03C0DBFF09019951FB
:10635000E66EE66A200EE66EDC0EE66E000EDFEC00
:106360003CF009019A51ACEC3BF009019E51ACECB8
:106370003BF0C0C900F0016A00BE016814EC39F0BE
:106380000901C151ACEC3BF0C2C900F0016A00BE8A
:10639000016814EC39F0CBC9E6FFCCC9E6FFF9EC93
:1063A00038F0CDC9E6FFCEC9E6FFCFC9E6FFD0C9B8
:1063B000E6FFF6EC39F009019F51ACEC3BF0D95007
:1063C000020F9CEC3AF0F6EC39F0ADC900F0016A2E
:1063D00000BE016814EC39F009019B51ACEC3BF0B4
:1063E000E2C900F0016A00BE016814EC39F0E1C9AD
:1063F00000F0016A00BE016814EC39F0A9EC39F034
:1064000066EC3BF0B6EC39F009019C51ACEC3BF08A
:106410003DEC3AF066EC3BF0B6EC39F009019D51E9
:10642000ACEC3BF0960EE66E0A0E48EC39F0060E28
:10643000E15C02E2E16AE552E16E005068EF39F09A
:10644000CEEC3BF0190EE66EDC0EE66E000EFBECB9
:1064500039F07DEC3BF00701CF51D011D11116E09E
:10646000CFC7F6FFD0C7F7FFD1C7F8FF0800F55038
:106470000DE0CFC7E6FFD0C7E6FFD1C7E6FF44EC8B
:1064800039F066EC3BF0E66E44EC39F0090EE66E4E
:10649000DC0EE66E000EE66E44EC39F09C0EE66E05
:1064A0000A0E85EC3CF002E2E16AE552E16E005032
:1064B00068EF39F0CEEC3BF047EC3BF0020EE66EB5
:1064C000DC0EE66E000EBAEC3CF0FFEC3BF0E1ECCB
:1064D0003AF0F9EC38F009019F51ACEC3BF09AEC42
:1064E0003CF000BE016814EC39F0E8EC3AF0B0EC96
:1064F0003CF099EC39F0FD0EDB0404E1980EE66EF9
:106500000A0E03D09A0EE66E0A0E85EC3CF002E20B
:10651000E16AE552E16E005068EF39F063EC39F062
:10652000090EE126010EF36E080EF3CFDBFF020E1B
:10653000F36E080EF3CFDBFFC7EC3AF0EE50ED1030
:1065400001E138D1FD0EDBCFDEFFDBCFDDFFFEEC5E
:1065500039F009E0FEEC39F0200805E0DF2A010EF1
:10656000F6E3DB2AF4D7FEEC39F0200801E022D173
:106570004EEC3BF001E3DB2AEF6A1EEC39F005EC50
:106580003BF019EC3BF001E115D1090EE66EE7ECAA
:1065900039F0D80EE66E040E5AEC39F01EEC39F0E4
:1065A000ECEC39F01EEC39F0CEEC3AF078EC3BF044
:1065B00024EC3AF02BEC3BF078EC3BF06CEC3BF04D
:1065C00019EC3BF001E0F6D01EEC39F0000EE66E5F
:1065D000060E14EC3BF005EC3BF0C1EC39F0D80EA4
:1065E000E66E040E5AEC39F078EC3BF0ECEC39F046
:1065F00078EC3BF0CEEC3AF024EC3AF044EC3CF092
:10660000A6EC3AF068EC3AF002E600EC3BF00AE265
:10661000D4EC3CF016EC3AF0060EDB2A070EF2E35F
:10662000DB2AF0D724EC3AF04CEC3CF0A6EC3AF044
:1066300068EC3AF002E600EC3BF00AE2D4EC3CF005
:1066400013EC3AF0060EDB2A070EF2E3DB2AF0D752
:106650000A01010E5D6F0A0EE66EE7EC39F028ECD8
:1066600039F050084EE10A018D5127E1060EDB6A30
:10667000070EDB6A68EC3AF004E6160E005C000ECA
:10668000015819E26EEC39F004BE05682CEC3AF0C2
:10669000060EDBCFE9FF070EDBCFEAFF760EE92619
:1066A0000A0EEA22E552E750EF6E060EDB2A070ECD
:1066B000E1E3DB2ADFD70A018C6B8D6BFA0EE66E05
:1066C000DB0EE66E000E5FEC39F05CEC3BF0C1ECEB
:1066D00039F00DEC2EF04AEC3AF00A01010E8D6F04
:1066E000E66EE7EC39F0E80EE66E040E5AEC39F08F
:1066F0005CEC3BF0ECEC39F05CEC3BF0CEEC3AF0CF
:1067000002D00A018D6B0501F69FB5EC3AF0D80E68
:10671000E66EDB0EE66E000EFDEC3CF00F0EF66E44
:10672000000EF76E000EC0EC3BF019EC39F0100EC5
:10673000F66E000EF76E000EC0EC3BF019EC39F06F
:1067400009EC3AF0DAEC3BF040EC3BF08DEC3BF03E
:106750000701CC51CD11CE110CE0CCC7E6FFCDC75F
:10676000E6FFCEC7E6FFDAEC3BF0CBEC3BF08DEC7E
:106770003BF0080E19EC3CF019EC39F00501F5512D
:10678000ABEC3CF00501F651E66EE66A66EC3BF0D8
:10679000E66EDAEC3BF000EC75F0E2EC3CF08DECF0
:1067A0003BF00501F751ABEC3CF0140ED5EC39F0A1
:1067B0004AEC3AF0090EE15C02E2E16AE552E16E70
:1067C00068EF39F07DEC3CF00A015D511AE1070EEB
:1067D000E66EE66AD00EE66EDB0EE66E000EB3ECF9
:1067E0003CF01EEC3BF001E0B9D0070EB9EC39F0FB
:1067F00095DEE552E5520601060ED06F0E0ED16F02
:10680000ADD0F7EC3BF078EC3BF01EEC39F070ECDF
:106810003CF06CEC3BF016EC3AF0050EE66EE66AE6
:10682000CA0EE66EDB0EE66E000EBAEC3CF01EEC15
:106830003BF006E0400EE66EB7EC3FF0E5528ED03E
:10684000D950FD0F96EC3CF0050EEE6E060EED6E87
:106850001DEC3AF0EF50450835E154EC3CF04D08A2
:1068600031E1C7EC3AF0020EEE26000EED22F7EC15
:106870003BF0010EE66E050EE66E010EB9EC39F046
:1068800070EC3CF0DCEC39F019EC3AF002E600EC8C
:106890003BF005E2EFEC3BF0F7E3DB2AF5D76CECDD
:1068A0003BF0010EE66E050E6CEC39F01DEC3AF093
:1068B000EFCF00F5D950FD0F96EC3CF0000EEE6ED8
:1068C000050EED6E0501F6BF03D00501150EF76F3D
:1068D0001DEC3AF0EF50430A37E0190A11E01B0AA9
:1068E0003DE1C30EE66EDB0EE66E000E5FEC39F0A6
:1068F0000A015E5133E10DEC2EF03AEC2EF01ED081
:1069000054EC3CF030081DE00901010EE86F0A016B
:106910005E5124E10DEC2EF0E66A74EC2FF0E552A6
:10692000E66A69EC30F0E552E66A88EC30F0E55250
:10693000E66A88DCE552E66AD9DCE5522AEC2EF0FC
:106940000DD00901E86B0AD0010EB9EC39F00ED870
:10695000E552E5520A015E5101E1DBD9030EE15C2B
:1069600002E2E16AE552E16E68EF39F081EC3CF059
:10697000FD0EDBCFDEFFDBCFDDFFFEEC39F009E003
:10698000FEEC39F02C0805E0DF2A010EF6E3DB2AE5
:10699000F4D7FEEC39F02C0805E14EEC3BF001E3B6
:1069A000DB2AEF6A1EEC39F078EC89F0E552E5520B
:1069B000F3CF9EFAF4CF9FFADECFA0FADDCFA1FA93
:1069C000040EE15C02E2E16AE552E16E68EF39F043
:1069D00063EC39F0060EE126020EE1EC3BF0310EDD
:1069E0000A019E1901E19F5101E173D1290E9E19FF
:1069F00001E19F5101E15BD1280E9E1901E19F51F8
:106A000001E128D1060E9E1901E19F5101E11ED13D
:106A1000050E9E1901E19F5101E10FD1040E9E194F
:106A200001E19F5101E1C0D0030E9E1901E19F5188
:106A300001E182D0020E9E1901E19F512AE0010E70
:106A40009E1901E19F5102E0000E5AD1DE6ADD6A13
:106A500019EC3AF004E6100E005C000E015801E358
:106A60004ED16CEC3BF0B80EE66EDB0EE66E000E1F
:106A7000FDEC3CF0100EABEC3CF0F1EC3AF0EF50DA
:106A8000ABEC3CF03AEC2EF0DF2A010EE1E3DB2A1E
:106A9000DFD7D5EC3AF0DCDB09E03AEC3CF006E07D
:106AA000020EDB2A030EF7E3DB2AF5D73AEC3CF0C3
:106AB00001E0BCD08AEC3AF001E3DB2A0AEC3CF0BE
:106AC00001E0AED055EC3BF004E6100E025C000E87
:106AD000035801E3A5D071EC3BF078EC89F0E55266
:106AE000E552F350E66EF1EC3AF0E552E750EF6E06
:106AF00019EC3AF004E6080E005C000E015810E3B1
:106B000071EC3BF089EC3CF0080E005E000E015A7F
:106B1000180E0024E66E63EC9FF0E552E552E55254
:106B20000FEC3BF00F0EEE1804E1ED5002E1A0EC8B
:106B300092F0ACEC3AF07FD0DE6ADD6A19EC3AF004
:106B400004E6200E005C000E015801E3D8D0DFCF30
:106B5000E6FFE7EC39F00FEC3BF0090EEE1804E12C
:106B6000ED5002E128EC3BF06CEC3BF0AD0EE66E34
:106B7000DB0EE66E000EFDEC3CF0200EABEC3CF0C4
:106B800071EC3BF066EC3BF0E66E040EDBCFE6FF0B
:106B9000050EE4EC3AF08DEC3BF03AEC2EF0DF2AF7
:106BA000010ECCE3DB2ACAD7D5EC3AF051DB09E081
:106BB0003AEC3CF006E0020EDB2A030EF7E3DB2A98
:106BC000F5D73AEC3CF032E18AEC3AF001E3DB2A0B
:106BD0000AEC3CF025E155EC3BF004E6180E025CB3
:106BE000000E03581DE271EC3BF0DFCFE6FF63ECD3
:106BF0009FF0E552E552E552ACEC3AF001DB0FECC8
:106C00003BF0020EEE1801E1ED5007E00FEC3BF017
:106C10000E0EEE181CE1ED501AE1A0EC92F017D028
:106C20006F0EE66E4D0EE66E010E05D0430EE66E5B
:106C30004D0EE66E010EE4DA0AD0ACEC3AF08EECC2
:106C40003CF0040EE66EB7EC3FF058D063DA3AEC55
:106C50002EF055D0D5EC3AF0FBDA09E03AEC3CF0F6
:106C600006E0020EDB2A030EF7E3DB2AF5D73AEC47
:106C70003CF015E18AEC3AF001E3DB2AEF6ADCEC48
:106C80003AF0AAEC58F0E552E55271EC3BF084EC96
:106C90003AF0BD0EFC6FDC0EFD6F000E23D00DEC44
:106CA0002EF0430EE66E4D0EE66E010E21D0090168
:106CB000A10EFC6FDB0EFD6F000EB2EC3AF0DCECC7
:106CC0003AF084EC3AF09B0EFC6FDB0EFD6F000E89
:106CD00009D0DCEC3AF084EC3AF0990EFC6FDB0E54
:106CE000FD6F000EB2EC3AF0050E5FDBACEC3AF053
:106CF0008EEC3CF0020EE66E58EC72F0E552010E9E
:106D0000006E060EE15C02E2E16AE552E16E0050BF
:106D1000DFD20501F6BF03D00501160EF76F020E94
:106D2000E1EC3BF0280E0A019FAF02D0D89003D0CF
:106D30009E5D000E9F5907E39F3507E29E51310883
:106D4000000E9F5502E20DEC2EF00B0149514A1145
:106D50004B1119E0A0CAE6FFA1CAE6FF9ECAE6FFF2
:106D60009FCAE6FF010EE66E07D04BCBFBFF4ACB76
:106D7000FAFF0B014951F96EF8DF006E050EE15E76
:106D8000005000090AE124DE000907E1DE0EE66E8C
:106D90004D0EE66E010E8EEC3CF02AEC2EF00A0150
:106DA0009E6B9F6BA0CAE9FFA1CAEAFFEF6A1200BF
:106DB0008ADA0A015D512CE05E51000829E3020ED7
:106DC000F4DA910EE66EDB0EE66E000E78DA860ED1
:106DD000E66EDB0EE66E000EBAEC3CF092DB2EDACD
:106DE000D0DA7D0EE66EDB0EE66E000EBAEC3CF0FD
:106DF00088DBAA0EE76EFB0EDBCFE9FFFC0EDBCFD4
:106E0000EAFF61EC3BF0EF6A47EC3BF0BADA42DBB9
:106E10005FD281EC3CF0020EDB6A030EDB6A0A01F2
:106E20005D516EE0B4DBEE50ED106AE0220EB3EC83
:106E30003CF0CEEC97F0E552E552E55282EC3BF0A7
:106E4000F3CF00F0F4CF01F0F350F41022E0020E83
:106E5000DB2ADBCF00F0030E01E3DB2ADBCF01F0FE
:106E6000FD0E00C0DBFFFE0E01C0DBFFF1D910E01C
:106E7000EFD922080DE03AEC3CF004E103EC3CF0E1
:106E80002E0EEF6E020EDB2A030EF0E3DB2AEED7A6
:106E9000DFDB290EE66EE66AD10EE66EDC0EE66EEC
:106EA000000EDFEC3CF0D950020F96EC3CF0EE50B7
:106EB000ED100DE0C3D9790EE66EDB0EE66E000E26
:106EC00000EC3DF09AEC74F0006E070E0BD0620EF1
:106ED000E66EDB0EE66E000E00EC3DF071EC74F039
:106EE000006E050EE15E00507DEC3BF00A015E5144
:106EF000000803E2140EE1EC3BF00DEC2EF0CADAD0
:106F0000040EE15C02E2E16AE552E16EE1D1DBD917
:106F1000090199A552D009019651040A18E0070AFF
:106F200010E0020A08E0010A18E1560EE66EDB0ED8
:106F3000E66E000E11D04B0EE66EDB0EE66E000E16
:106F40000BD0420EE66EDB0EE66E000E05D0330E61
:106F5000E66EDB0EE66E000EE7DB090194510F0AC8
:106F600026E0020A1EE0090A16E0060A0EE0030AFD
:106F700006E0D90EE66EDA0EE66E000E23D02A0E7B
:106F8000E66EDB0EE66E000E1DD0140EE66EDB0E16
:106F9000E66E000E17D0060EE66EDB0EE66E000EF5
:106FA00011D0FC0EE66EDA0EE66E000E0BD0EA0E85
:106FB000E66EDA0EE66E000E05D0CC0EE66EDA0E48
:106FC000E66E000EB1DB4D0E0701CB5D12E1A3C9E9
:106FD000E6FFA4C9E6FF03EC3DF09BDB64D9A1C941
:106FE000E6FFA2C9E6FF0AEC3DF093DB5AEC3CF069
:106FF00019D0A3C900F0A4C901F0040E0BDBFEE117
:107000002AD903EC3DF0A1DB4ED9A1C900F0A2C9F9
:1070100001F0040EFFDAFEE11ED90AEC3DF095DB2B
:1070200061EC3CF081DB91EC3CF0AE0EE66EDA0EEA
:10703000E66E000EB3EC3CF06CDB35D9AC0EE66EC0
:10704000DA0EE66E000E70DB4D0E0701CB5D0EE131
:10705000CDC900F0CEC901F0CFC902F0D0C903F00C
:107060001DDA7EDB8DDA5AEC3CF039D0CDC904F064
:10707000CEC905F0CFC906F0D0C907F00FDA26C097
:1070800004F027C005F028C006F029C007F0040E60
:107090001F0B27DA07E0D890003601360236033698
:1070A000E806F9E1050E0026000E01220222032265
:1070B0000A0E2B6E2C6A2D6A2E6A00C026F001C0C3
:1070C00027F002C028F003C029F0F1ECA7F048DB5C
:1070D000BDEC74F0086E090EE15E0850F2DBB3EC13
:1070E0003CF071EC74F0050EE15EDDD80901F5515C
:1070F000F6110AE0E2D99C0EE66EDA0EE66E000E9C
:10710000B3EC3CF03DDACFD8F1DB00C0F3FF01C0B7
:10711000F4FFDED043DB55DB910EE66EDB0EE66E50
:10712000000E69D9EADAD8DAF2DEE552E552020E4B
:10713000E15C02E2E16AE552E16ECAD0E7EC3CF0C4
:107140007A0EE66EDA0EE66E000EB9D88FDB02E23A
:10715000E16AE552E16EBCD0E7EC3CF04F0EE66E22
:10716000DA0EE66E000EABD881DB02E2E16AE55290
:10717000E16EAED0E7EC3CF0D4DB1F0EE66EDA0E2B
:10718000E66E000EDFEC3CF0180EE66EDA0EE66EF0
:10719000000EE66E79D86ADB02E2E16AE552E16E42
:1071A00097D0E7EC3CF00701CAA307D0D2D8F10E84
:1071B000E66ED90EE66E000E06D0CBD8D90EE66E7E
:1071C000D90EE66E000ED6DBDEDB57D9D10EE66EA9
:1071D000D90EE66E000ECAD8CE0EE66ED90EE66E59
:1071E000000EE66E51D842DB02E2E16AE552E16E42
:1071F0006FD0B6DBFAEF3CF0B9DB8BDA82EF3BF015
:10720000E66E9ECAE6FF9FCAE6FF390EE66E4D0E99
:10721000E66E010EAFDB99DA8FDA71EC74F0036E73
:10722000050EE15E03501200D5DA9ADB8EDA7DEFAF
:107230003BF0E66EBFDA6DDA8DEF3BF0FD0EDBCF93
:10724000E6FFFE0EDBCFE6FF120094DB89EF3BF09A
:10725000DADAEF501200050E0026000E01220A0EA7
:107260002D6E2E6A00C028F001C029F066ECA8F04F
:1072700028C000F029C001F028C0E6FF29C0E6FFC1
:10728000120074DBA5EF3BF027DA85DA7DEF3BF0E7
:10729000E66EFE0EDBCFE6FF34EC2FF0E552E55252
:1072A000E552006E1200FD0EF3CFDBFFFE0EF4CFB1
:1072B000DBFF1200E66E15DA9ADB71EF3BF05ADB6A
:1072C00023EC98F077D3D9CFE6FFE1CFD9FF1200B6
:1072D000E552E7CFD9FF12005EDB64D2800E006E6C
:1072E0004E0E016E010E026E75DAE66E0EEC8CF03B
:1072F000E552E7CF02F0E552E7CF01F0E552E7CFE4
:1073000000F0F3CF03F0F4CF04F0400E2D6E2E6AA0
:10731000F3CF28F0F4CF29F0C8EC83F024C003F0B9
:1073200025C004F0056A1200E66E1ADB68DA7DEF0C
:107330003BF0F9EC75F021DBD5C9E6FFD6C9E6FFD5
:10734000D7C9E6FFD8C9E6FF0BDBF9EC75F0BDEF56
:107350003CF0010EE66EE66AEAC900F0016A026AD4
:10736000036AEAC9E6FF01C0E6FF6CD249DBC3EF5E
:107370003CF0E76EBBDAE7500026000E0122EAEF90
:107380003BF0B6D98EEC97F02CEF3CF0E552E5528D
:107390007DEF3BF0DE52B1D9DD521200010EDBCFA2
:1073A000E6FF020EDBCFE6FF12000BDA0DEF2EF048
:1073B000E7D926DBFAEF3CF0100EE66EE66AE80E3F
:1073C000E66E040EE8DA84DADE6ADD6A12001CEC8E
:1073D0009FF0E55282EF3BF044DAF3CF02F0F4CFB6
:1073E00003F0F3CFE6FFF4CFE6FF1200B9DABDEC0D
:1073F00074F0BDEF3CF0BEDACBEF3BF0DECFE9FF3F
:10740000DDCFEAFFEF501200E66E6BD9C4D982EFF0
:107410003BF00E0E1CDA90D92A0EE66EDC0EE66EFC
:10742000000EE66E120064D937DABCD161D92CDACD
:10743000B9D16FDAD89001501200FD0EDBCFE9FF11
:10744000FE0EDBCFEAFF1200100EE66EE66AD80EE3
:10745000E66E040EE66E120000500324F36E015037
:107460000420F46E02500520F86EF4CFF7FFF3CF3E
:10747000F6FF0800F550E66E1200010EE66EE66AB1
:10748000EBC900F0016A026A036AEBC9E6FF01C0BA
:10749000E6FFD8D13AEC2EF02AEF2EF00A0E2B6E32
:1074A0002C6A2D6A2E6ACDC926F0CEC927F0CFC925
:1074B00028F0D0C929F0F1EFA7F0F5C900F0F6C91E
:1074C00001F0026A036AF5C9E6FFF6C9E6FFBAD120
:1074D000060EDBCF00F0070EDBCF01F0D890015095
:1074E000120026C000F027C001F028C002F029C019
:1074F00003F01200FC0EDBCFE9FFFD0EDBCFEAFF4D
:107500001200B2EC97F056D2A3EC3EF0E552E552F1
:1075100009011200020EDBCFE9FFDB2A030EDBCFED
:10752000EAFF1200006E016AD950030FFFD9005024
:10753000EE260150ED221200F9D9EECFE6FFEECF94
:10754000E6FFEECFE6FFEFCFE6FF1200C1D9060E51
:10755000DB6A070EDB6A1200400EE66E4D0EE66E29
:10756000010E1200FE6F54EF3EF00E0EF66E000E8E
:10757000F76E000EF86E0800F550E66EE66A12002F
:10758000BDEC74F0046E090EE15E04501200D95097
:10759000FD0FE96EFF0EDA20EA6E12000DECA1F08D
:1075A000046E0A0EE15E04501200020EA0CADBFF58
:1075B000030EA1CADBFF1200A0CAE6FFA1CAE6FFC4
:1075C00012009BD891EF3CF0DBCFE6FFFFEF3BF0E2
:1075D000D1C9E6FFD2C9E6FFD3C9E6FFD4C9E6FFA9
:1075E0001200DECFE9FFDDCFEAFFE50EE926050E4A
:1075F000EA221200BF0EFC6FDC0EFD6F000E1200BF
:10760000000E005C040E015812005F0EE66E0A0EBA
:10761000E66E1200D89000360136E8041200D9CF89
:10762000E9FFDACFEAFF1200E66E02EC98F02CEFE9
:107630003CF0E2EC97F010D9000912002AEC97F028
:10764000C1D90009120065D90001800E0114120091
:10765000DAD8EF6A12001AEC90F0006E060EE15EC6
:1076600000501200EECF00F0EFCF01F0DF50001815
:107670001200DF50EA6AC30FE96E090EEA22120017
:107680009AEC74F0026E070EE15E02501200FB0EDF
:10769000DBCFE6FFFC0EDBCFE6FF1200DFCFE9FF1A
:1076A000DF2A010EDBCFEAFF1200DECF02F0DDCFD2
:1076B00003F0D89003501200760EE66E0A0EE66EC6
:1076C0001200E750E926000EEA221200A20EE66E32
:1076D000DC0EE66E000E1200DECFE6FFDDCFE6FF29
:1076E0001200020EDBCFE6FF030EDBCFE6FF120037
:1076F000000EE66E060EE66E1200F3CFDEFFF4CF4C
:10770000DDFF1200020EF3CFDBFF030EF4CFDBFF31
:107710001200A0EC74F0E2EF3CF0040EF3CFDBFFBC
:10772000050EF4CFDBFF12001ED971EC74F0006E71
:10773000050EE15E53EF39F0F3CF00F0F4CF01F026
:10774000F3CFE6FFF4CFE6FF1200A0EC74F0026E78
:10775000070EE15E02501200E66EE66AF9EF38F0BD
:10776000C0DE26C0E6FF27C0E6FF28C0E6FF29C02E
:10777000E6FFA40EE66EDA0EE66E000EB3EF3CF006
:10778000F86E0800F550E66EE66A2C0EE66EDC0E2A
:10779000E66E000E120071EC74F00CD194DD020E56
:1077A000E1261200E66E2FEC9DF0006E080EE15E01
:1077B00000501200040EDBCFE6FF050EDBCFE6FF24
:1077C0001200E66E58EC72F0E5521200E66EE66AC0
:1077D000FCEF38F000C0E6FF01C0E6FF1200E4D87D
:1077E000000EE66E060E78DDDF2A010E1200BF0ED7
:1077F000E66EDC0EE66E000EB6D881EF3AF09AEC3B
:1078000074F0E2EF3CF0020EDBCFE9FF030EDBCFBA
:10781000EAFF1200EF6AD0DE78EC89F0B7DD23EFE3
:107820003BF03AEC2EF066DEDECFEEFFDDCFEDFF73
:107830001200DBCFE6FFE66A270EE66EDC0EE66E90
:10784000000E120002C0E6FF03C0E6FF1200E66E63
:107850001CEC9FF0E5521200E552E552E552E5526C
:1078600012003CEC98F0E552E552120013DE020ED5
:10787000E15C1200EDDC2C081200AB0EFC6FDC0E9C
:10788000FD6F000EB2EF3AF0000EE66E020EE66EED
:10789000FA0EE66E040E1200000EE66E010EE66EA3
:1078A000F80EE66E040E1200010EE76EC6DD09DF6B
:1078B000EF501200F8DCBA0EE66EDA0EE66E000E3D
:1078C0001200F1DCB60EE66EDA0EE66E000E120065
:1078D000E66E86EC9CF0006E080EE15E0050120031
:1078E000D6EC90F0E552E552C6EF39F0FD0EDBCF55
:1078F00000F0FE0EDBCF01F01200E5DC030EE12606
:107900001200E1DC040EE1261200C2DC020EE15C92
:107910001200DECF00F0DDCF01F0120071DC3AEF93
:107920002EF00901A051E66EE66A1200E96EDACF88
:10793000EAFF1200D9C9E6FFDAC9E6FF5ADCDBC963
:10794000E6FFDCC9E6FF55DC0901E05105DFE3C9CC
:1079500000F0016A1200E66EE66AB8DE19EF39F04F
:10796000B5DE00EF3DF0E66E1EEF39F0AFDEE66EFD
:1079700071EF3BF0E66E78EF3BF0006E090EE15ED2
:1079800000507DEF3BF092EC75F0046E0B0EE15E63
:1079900004507DEF3BF0E66E000EE66E030EE66EE1
:1079A000FC0EE66E040E12000601006B010EE66E80
:1079B000E66A1200006E050EE15E0050120045DC22
:1079C0007DEF3BF0006E070EE15E00501200E6DE38
:1079D000D5EF39F03CEC98F0D9DC6CEF3BF0FADEF7
:1079E00050DC82EF3BF0DADCB0DECAEF39F039DF91
:1079F0009CEF3BF08EDE7DEF3BF027DC8DEF3BF024
:107A0000E66E6CEF3BF0C20EE66EDA0EE66E000E2E
:107A1000B3EF3CF0BE0EE66EDA0EE66E000EB3EF8C
:027A20003CF038
:0E7A2200D8CFE4FFE0CFE4FFE46EDACFE4FF5C
:107A3000E2CFDAFFE9CFE4FFEACFE4FFF6CFE4FFDD
:107A4000F7CFE4FFF8CFE4FFF5CFE4FFF3CFE4FF97
:107A5000F4CFE4FFFACFE4FFFBCFE4FF00EE20F029
:107A6000140EE80403E3EECFE4FFFBD700EE00F0D2
:107A7000200EE80403E3EECFE4FFFBD7E652A0ECD0
:107A8000A0F0FFECA1F0E55200EE1FF0200EE8049C
:107A900003E3E5CFEDFFFBD700EE33F0140EE8046F
:107AA00003E3E5CFEDFFFBD7E5CFFBFFE5CFFAFF23
:107AB000E5CFF4FFE5CFF3FFE5CFF5FFE5CFF8FF26
:107AC000E5CFF7FFE5CFF6FFE5CFEAFFE5CFE9FF2A
:107AD000E5CFDAFFE550E5CFE0FFE5CFD8FF1000B6
:107AE0000801009B12007DEC49F0E652D9CFE6FF79
:107AF000DACFE6FF76ECA0F0E552E552000901E1AD
:107B0000D0D0FF0E0601EB5D01E094D0C85103E038
:107B10007F0EC85D08E10A0EDF5CE8E00D0EDF5C59
:107B200002E10A0EDF6E0D0EDF5CE0E0BEEC4AF013
:107B300019EC4AF003E1015001E1EA073A0EDF5C7B
:107B40001EE1060EEA5D1BE337EC4AF018E1490E30
:107B5000015D15E1500E025D12E1440E035D0FE17F
:107B60000601EA053DEC49F0EF6A050EE66E070EE8
:107B7000E66EF7EC49F0FD0EEB6FEA6BB7D70A0E35
:107B8000DF5CB4E10601EA07EA513DEC49F0EF6A37
:107B9000040EEA5D48E337EC4AF045E1430E015D2F
:107BA00042E14D0E025D3FE1540E035D3CE1070EE4
:107BB000DF6EDF50DF2A3DEC49F0EF50220804E091
:107BC0000601EA51DF5CF5E3DF043DEC49F0EF6AC2
:107BD0000601D66B140EE66EE66A070EE66E070E19
:107BE000E66ED60EE66E060ECFEC49F00601E96BA6
:107BF000EAC6DFFFDF50DF063DEC49F0EF502C080E
:107C000003E0DF500008F6E3DF50016A000F006E6A
:107C1000070E0122020E1FEC4AF0F7EC49F0EA6B66
:107C2000FE0EEB6F63D70601B6EC49F00701006B5F
:107C3000060135D0FE0EEB5D1CE10D0EDF5C03E0AE
:107C40000A0EDF5C07E1EA51EA2B3DEC49F0200E19
:107C5000EF6E02D0BEEC4AF019EC4AF003E101509D
:107C600001E1EA07EC07EC5101E040D71FEC4BF0D3
:107C700016D00D0EDF5C08E0BEEC4AF019EC4AF0BD
:107C800003E1015001E1EA07EC070A0EDF5C03E1C2
:107C9000EA071FEC4BF0EC5101E028D7EA6BEB69E7
:107CA00025D7E55282EF49F024EC4BF038E1DF6A4A
:107CB00034EC49F00A080BE10D0EDF5C08E0080126
:107CC00000B1FDD70D0E86EC49F00FE1FBD70D0E8C
:107CD000DF5C0BE134EC49F00A0807E0080100B171
:107CE000FDD70A0E86EC49F0FCE034EC49F028E0C0
:107CF000080100B1FDD734EC49F086EC49F0FBE017
:107D00000901FCC9F6FFFC2BFDC9F7FF000EFD239E
:107D1000FEC9F8FFFE230800F550DF6EC9D734EC2A
:107D200049F00EE0080100B1FDD734EC49F086ECD3
:107D300049F0FBE00901FC2B000EFD23FE23EFD7E9
:107D4000E55282EF49F024EC4BF035E1DF6A75EC47
:107D500049F00A080BE10D0EDF5C08E0080100B1F4
:107D6000FDD70D0E86EC49F00FE1FBD70D0EDF5C61
:107D70000BE175EC49F00A0807E0080100B1FDD7F6
:107D80000A0E86EC49F0FCE075EC49F025E00801AC
:107D900000B1FDD775EC49F086EC49F0FBE0FD0E33
:107DA000DBCFE9FFDB2AFE0EDBCFEAFF01E3DB2AB4
:107DB000EFCFDFFFCCD775EC49F00EE0080100B142
:107DC000FDD775EC49F086EC49F0FBE0FD0EDB2AAF
:107DD000FE0EF1E3DB2AEFD7E55282EF49F07DECAE
:107DE00049F0080100B1FDD7FE0EDBCFE6FF4FECF6
:107DF000A0F0E5520009F8E082EF49F07DEC49F08F
:107E0000040EE126030EBCEC49F0CA0EE66ED90E54
:107E1000E66E000E9DEC49F00EE0FD0EDBCF00F0AB
:107E2000FE0EDBCF01F000C001F0006A0050060139
:107E3000F1130150F213C70EE66ED90EE66E000E76
:107E40009DEC49F00BE0FD0EDBCF28F0FE0EDBCF02
:107E500029F028500601F1132950F213040EE15CB9
:107E600002E2E16AE552E16E82EF49F07DEC49F011
:107E7000060EE126A7EC4AF0E66EFD0EDBCFE6FF2C
:107E8000FE0EDBCFE6FF0AEC49F069E0A7EC4AF012
:107E90002AEC4BF064E055EC4BF061E055EC4BF014
:107EA0005EE03FEC4AF0EF504F0859E1010EE76EFB
:107EB0003FEC4AF0E750E926000EEA22EF502D0889
:107EC0004EE1C30EE66ED90EE66E000EE66E020EB1
:107ED000E76EDBCF00F0030EDBCF01F0E7501FECC5
:107EE0004AF09FEC4AF0ADEC4AF039E0C30EE66E82
:107EF000D90EE66E000E62EC49F093EC49F0F350B7
:107F000059EC4BF0040EF3CFDBFF050EF4CFDBFF93
:107F1000D7EC49F00DE1040EDBCFE9FF050EDBCF16
:107F2000EAFFEF501CE0C20EE66ED90EE66E12D0EC
:107F300046EC4AF0040EDBCFE6FF050EDBCFE6FF92
:107F4000E2EC97F0E552E552E552E552000907E010
:107F500046EC4AF093EC49F0F3504DEC4AF0060E33
:107F6000E15C02E2E16AE552E16E82EF49F07DEC0C
:107F700049F0020EE126FE0EDBCFC8F60601C8511D
:107F8000240A01E15FD1070A01E152D1010A01E1AE
:107F900049D1030A01E115D1010A01E1FCD0600ACF
:107FA00001E1D7D0030A01E1B9D0010A01E18FD084
:107FB000030A01E178D0530A69E0030A5CE0010A90
:107FC0004FE0160A47E0030A3CE0010A33E0070AE3
:107FD00025E0010A21E0030A11E07E0A0CE07F0A95
:107FE00001E03CD136EC4BF0AFEC49F00601010E5C
:107FF000CD6F0A0E24D11CEC7DF030D10A0ED5ECE9
:108000004AF00601030ECD6F140ECE6FCF6B09013F
:10801000E86B06EC2EF022D1CD6B20D1AFEC49F00D
:1080200068EC72F00601020ECD6FDFEC49F006013C
:10803000CC6B14D1050ECD6F0A0EDFEC49F00A0EA1
:108040009ED0060ECD6F020ECE6FCF6BC96B68EC63
:1080500072F004D1E66AD4EC48F03EEC72F0FED047
:10806000090ED5EC4AF001EC4AF0460EFC6F4C0EBE
:10807000FD6F010ED4D0080ED5EC4AF001EC4AF0A9
:108080008D0EFC6F4C0EFD6F010EC9D0070ED5ECA6
:108090004AF00601030ECD6F230ECE6FCF6BC96B76
:1080A00054EC4AF0BCD0050EE66E48EC4BF00AECFE
:1080B0004AF006E2070E99EC49F00601400E05D0A1
:1080C000080E99EC49F00601020ECD6F14D0050E92
:1080D000BFEC49F0A90EFC6FD90EFD6F000EE6EC67
:1080E00049F0090E99EC49F00AEC4AF002E2430E1D
:1080F00001D0020ECD6FCAC6CEF6CBC6CFF60A0EA1
:10810000D880CE57000ECF570F0ECF03F3CFCFF648
:10811000CE03F3CFCEF6F450CF27A0D0050ED5EC8A
:108120004AF0C3EC49F00601020ECD6F3C0ECE6F53
:10813000CF6B060EC96F0901E86B0AEC2EF03EEC1E
:108140004BF05BEC4AF0E6EC49F00601400EC86FDC
:1081500085D0050ED5EC4AF0C3EC49F0BCEC49F0F3
:10816000F2EC49F0EF5014E0C7ECA7F0000910E082
:108170000601020ECD6F3C0EDFEC49F0020E70ECF2
:1081800049F00901B60EFC6FD90EFD6F000E47D005
:108190000601200EC86F020ED5EC4AF00A015E6B94
:1081A0000601CD6BC96B0901E60507E0050EE65D2A
:1081B00004E0780E0601D26F02D00601D26BD36BB9
:1081C0004DD0060ED5EC4AF03EEC4BF00601030E06
:1081D000CD6FF00ECE6FCF6B0AEC2EF00D0EBCEC17
:1081E00049F0F2EC49F0EF5007E10901F50EFC6FA0
:1081F0004C0EFD6F010E13D00901830EFC6FD90EDA
:10820000FD6F000EE6EC49F0CBEC4AF09CDDE55248
:10821000E5520901790EFC6FD90EFD6F000EE6ECF8
:1082200049F01CD00A0ECE6FCF6B400ECD6F16D02A
:10823000060ED5EC4AF00601240ECD6F1E0ECE6F51
:10824000CF6B0CD0CC51CC2B006E140E005C02E234
:10825000020E01D0030EE66E8ADEE552020EE15CEC
:1082600002E2E16AE552E16E82EF49F07DEC49F00D
:10827000110EE126FE0E0601EB5D1AE10901E6058D
:1082800007E0050EE65D04E0C3EC49F044EC4BF07A
:108290000501F6BF03D005010A0EF76F62EC4AF044
:1082A000D60EE66E060EE66E66EC4AF0BDEF45F0C1
:1082B000FF0EEB5D10E00501F6BF03D00501140EC3
:1082C000F76F9AEC4AF0E2EC33F0E552E55271ECCC
:1082D0004AF0BDEF45F00501F6BF03D005011E0EC3
:1082E000F76F0601C8517F0A02E1B6EF45F05F0A59
:1082F00001E117D2600A01E15ED1630A01E141D1D7
:10830000020A01E1F7D0330A01E1CAD0030A68E0AA
:10831000010A2CE0110A17E0010A02E0BDEF45F066
:10832000050EEA5D02E2BDEF45F080EC4AF0730E07
:10833000E66ED90EE66E000EC7EC48F002E0BDEF27
:1083400045F07F0EEAD1020EEA5D02E2BDEF45F094
:108350003BEC4AF002E0BDEF45F04B0E015D02E060
:10836000BDEF45F044EC4BF0100ED7D1040EEA5DA2
:1083700023E337EC4AF020E1430E015D1DE1530E8B
:10838000025D1AE14D0E035D17E19AEC4AF03CECF8
:1083900098F0E552E552F3CFE9FFF4CFEAFFE906A2
:1083A000000EEA5A000EE926070EEA22EF503108C5
:1083B00001E1E3D3030E5AD00601C95101E0DDD338
:1083C000020EEA5D01E2D9D33BEC4AF001E0D5D3DD
:1083D0004B0E015D01E0D1D344EC4BF0110E9DD169
:1083E000100EEA5D14E3380E0701005D10E1390E4E
:1083F000015D0DE1180EE66EE66A9AEC4AF0CD0ECC
:10840000E66E050ECFEC49F00501E46BB6D3080E1D
:108410000601EA5D16E337EC4AF013E1430E015D15
:1084200010E1500E025D0DE1420E035D0AE1460EC1
:10843000045D07E13A0E055D04E19AEC4AF016DDB1
:1084400095D1080E0601EA5D17E337EC4AF014E116
:10845000430E015D11E1500E025D0EE1490E035D18
:108460000BE1520E075D01E188D3040E99EC49F04F
:108470000601010EC96F81D30601C95101E07DD308
:10848000020EEA5D01E279D33BEC4AF001E075D3DC
:108490004B0E015D01E071D344EC4BF0120E3DD167
:1084A000060EEA5D16E337EC4AF013E1490E015D72
:1084B00010E1500E025D0DE1520E035D0AE1390E2E
:1084C000065D07E009012C0EFC6F4D0EFD6F010EDD
:1084D0006DD1020E0601EA5D01E24FD33BEC4AF09A
:1084E00001E04BD34B0E015D01E047D344EC4BF070
:1084F000210E13D1020EEA5D0BE33BEC4AF008E1DA
:108500004B0E015D05E171EC4AF0CC6B220E05D1FA
:10851000050E0601EA5D07E3450E0701005D03E174
:10852000520E015D05E0F8EC4AF0C7EC48F002E1BC
:10853000230EF3D084EC4AF0610EE66ED90EE66E9F
:10854000000EC7EC48F001E018D3A7EC4AF0E66E45
:108550009AEC4AF00AEC49F001E10FD3A7EC4AF09B
:108560002AEC4BF001E109D3080EE66EE66ACBEC8B
:108570004AF0EC0EE66E090ECFEC49F00901F46BFF
:10858000FCD2D8EC4AF001E0F8D22C0E0701085DCD
:1085900003E1070E091502D0070E07150901E66F62
:1085A000E80404E0050EE65D01E0E7D271EC4AF074
:1085B000CC6B400EB2D0020EEA5D16E3450E070109
:1085C000005D12E1520E015D0FE1020E0601C95D70
:1085D00003E0030EC95D02E1410E9FD0050EC95DA7
:1085E00001E0CBD2030E99D0020E0601EA5D06E34C
:1085F0003BEC4AF003E14B0E015D0BE0530E07012B
:10860000005D03E1480E015D04E0050E0601C95D51
:108610006DE10601EA6B1E0ECE6FCF6B0901E76BB1
:108620003EEC4BF00601C92BC951080A5DE00F0A68
:1086300048E0010A43E0030A3AE0010A31E0070A90
:1086400026E0010A0DE0030A01E097D20901470E76
:10865000FC6FD90EFD6F000EE6EC49F0050E0FD051
:1086600009013A0EFC6FD90EFD6F000EE6EC49F0E1
:10867000050EE0EC4AF0060EE0EC4AF0070EFBECCB
:1086800048F0440EFC6FD90EFD6F000E8FD0040E23
:10869000BFEC49F02C0EFC6FD90EFD6F000E86D09A
:1086A00009011E0EFC6FD90EFD6F000E7FD009016F
:1086B000140EFC6FD90EFD6F000E78D05BEC4AF003
:1086C00075D0030EBFEC49F0000EFC6FD90EFD6FA4
:1086D000000EE6EC49F0040EFBEC48F0F60EFC6FE1
:1086E000D80EFD6F000E62D0200E17D0070EEA5D87
:1086F0000DE3080EE66EE66AED0EE66ED80EE66E47
:10870000000EC7EC48F002E1020E07D001EC4BF07E
:10871000C7EC48F001E031D2020EE66EB7EC3FF054
:1087200026D0D8EC4AF025E12C0E0701085D03E1C4
:10873000070E091502D0070E07150901E66FE804B8
:1087400003E0050EE65D05E10601D26BD36BE66A38
:108750000AD00601D251D31101E00FD2780ED26FA8
:10876000D36B010EE66EE66ACCECA1F0E552E55261
:1087700004D280EC4AF0DB0EE66ED80EE66E000EF8
:10878000C7EC48F016E10901E60507E0050EE65DD5
:1087900004E0C3EC49F044EC4BF0010E70EC49F0FE
:1087A00009010D0EFC6F4D0EFD6F010EE6EC49F058
:1087B000E4D1020EE66EE66AD80EE66ED80EE66EDC
:1087C000000EC7EC48F001E0BCD076EC4AF001E3C3
:1087D000B8D0C4EC4AF0020EE66E070EACEC49F0DD
:1087E000CEEC48F00EE013EC4AF0020E26C0DBFFA0
:1087F000030E27C0DBFF040E28C0DBFF050E29C0D7
:10880000DBFFCEEC48F005E0F2EC49F00A0EEFCFCA
:10881000DBFFCEEC48F00EE013EC4AF0060E26C06B
:10882000DBFF070E27C0DBFF080E28C0DBFF090EA9
:1088300029C0DBFFCEEC48F005E0F2EC49F00B0E6E
:10884000EFCFDBFFCEEC48F005E0F2EC49F00C0E88
:10885000EFCFDBFFCEEC48F0CEEC48F0CEEC48F0AA
:1088600008E093EC49F00D0EF3CFDBFF0E0EF4CFD2
:10887000DBFFADEC4AF001E180D10C0EDB50010BC7
:108880000901E06FE8505AE00A0EDB50530818E186
:10889000020EDBCF00F0030EDBCF01F0040EDBCFC6
:1088A00002F0050E6AEC4AF0020E00C0DBFF030E78
:1088B00001C0DBFF040E02C0DBFF050E03C0DBFFBF
:1088C0000B0EDB50570818E1060EDBCF00F0070E49
:1088D000DBCF01F0080EDBCF02F0090E6AEC4AF0A4
:1088E000060E00C0DBFF070E01C0DBFF080E02C052
:1088F000DBFF090E03C0DBFF020EDBCFD1F9030E55
:10890000DBCFD2F9040EDBCFD3F9050EDBCFD4F9E0
:10891000060EDBCFD5F9070EDBCFD6F9080EDBCF7D
:10892000D7F9090EDBCFD8F90D0EDBCFDBF90E0E30
:10893000DBCFDCF90901780EE36F1FD10901E36B8E
:108940001CD1030EE66EE66AD20EE66ED80EE66E17
:10895000000EC7EC48F022E176EC4AF01FE2C4ECCE
:108960004AF0030EE66E070EACEC49F008E093EC1B
:1089700049F00F0EF3CFDBFF100EF4CFDBFFADECB1
:108980004AF001E1FAD00901E05101E1F6D00F0E01
:10899000DBCFD9F9100EDBCFDAF9EFD00A0EE66E95
:1089A000E66AC70EE66ED80EE66E000EC7EC48F01B
:1089B00004E10901E75123E117D0070EE66EE66AEC
:1089C000BF0EE66ED80EE66E000EE1DB3FE1110E43
:1089D000E66EE66AAD0EE66ED80EE66E000ED7DBEA
:1089E00012E10901E7510BE1010EE66EE66E90EC33
:1089F0004AF00DEC2EF0AEEC2EF02AEC2EF0090130
:108A0000010EE76FBAD0150EE66EE66A970EE66EB7
:108A1000D80EE66E000EBBDB01E1AFD0110EE66EA4
:108A2000E66A850EE66ED80EE66E000EB0DB54E008
:108A30000901E76B020EE66E48EC4BF00901E60512
:108A400068E0050EE65D01E098D063D080EC4AF066
:108A50007F0EE66ED80EE66E000E99DB12E12C0E4C
:108A60000701085D09E1070E0715006E070E0615E0
:108A70000A0DF350002402D0070E06150901E96F14
:108A80007CD0070EE66EE66A770EE66ED80EE66ECE
:108A9000000E7DDB56E00B0EE66EE66A6B0EE66EB0
:108AA000D80EE66E000E73DB03E10A015E6B65D043
:108AB00084EC4AF0640EE66ED80EE66E000E67DBBC
:108AC0000BE00C0EE66EE66A570EE66ED80EE66E0A
:108AD000000E8CEC49F004E10AEC2EF0420E34D08A
:108AE000090EE66EE66A4D0EE66ED80EE66E000ED4
:108AF0004EDB0FE0F8EC4AF08CEC49F00AE001ECB8
:108B00004BF04CEC4BF0026E070EE15E0250000998
:108B100004E10AEC2EF0410E17D0040EE66EE66A70
:108B2000490EE66ED80EE66E000E31DB0AE084ECEC
:108B30004AF0420EE66ED80EE66E000E8CEC49F05E
:108B400007E10AEC2EF0010EE66EB7EC3FF014D010
:108B500084EC4AF03B0EE66ED80EE66E000E17DB94
:108B60000CE19AEC4AF009EC37F005D062EC4AF0DF
:108B7000EEEC7FF0E552E552E552110EE15C02E2C7
:108B8000E16AE552E16EBED3B8DB080EE1260601CC
:108B9000C8517F0A01E15AD15F0A42E0220A3EE051
:108BA000230A31E0330A29E0030A1DE0010A11E03B
:108BB000110A01E04DD1050ECE5D000ECF5902E243
:108BC000020EB7DB0901090EFC6F4D0EFD6F010EA1
:108BD0003BD13EDB01E03CD10901460EFC6F4C0E5F
:108BE000FD6F010E31D134DB01E032D109018D0E70
:108BF000FC6F4C0EFD6F010E27D12ADB01E028D15E
:108C000054EC4AF021D1140ECE5D000ECF5901E391
:108C10001FD184EC4AF0CCECA1F0E1D0E66A23D07D
:108C2000FF0EEB5D09E0ED0503E1ED6BEB6910D0A4
:108C3000ED51010801E2ED07000ED880D255000E7B
:108C4000D35508E2D207000ED35BD251D31102E113
:108C5000210E08D088EC4AF009E25E2B5E513C08F8
:108C600005E2400EE66EB7EC3FF0BAD00901E6052A
:108C700004E0050EE65D01E0EBD00A019E519F1174
:108C800006E00A015D0503E10A015E5127E0FF0EDF
:108C9000060195EC4AF063E20A015D0560E10A0114
:108CA0005E515DE141EC4BF0200E060195EC4AF07F
:108CB00004E2F19B9EEC38F0CBD0040E95EC4AF028
:108CC00010E2F195F35101E0C3D0060E0A019E6F48
:108CD0009F6BA0CAE9FFA1CAEAFFEF6A89EC36F0F0
:108CE000B7D0080E95EC4AF006E2F197EEA3B0D0AB
:108CF000D1EC38F0ADD0100E95EC4AF004E2F199C9
:108D0000ACEC38F0A5D0020E95EC4AF00AE2F193F3
:108D100041EC4BF0020EE66E74EC2FF0E5520208C7
:108D20001BD0010E95EC4AF01AE2F1910901E851CD
:108D3000000815E2020EDF6E41EC4BF0DFCFE6FFDC
:108D400076EC31F0D0EC4AF074EC2FF0E552DF6EA7
:108D5000020EDF5C01E17CD02AEC2EF079D0000E0F
:108D60000601F115006EFF0EB4EC4AF047E241EC4B
:108D70004BF035DB000E0601F115006E200EF4DB22
:108D800005E2F29B58DA21EC59F029D0C5DB040E3C
:108D9000EBDB12E2F295F3515BE1360EE66ED80E94
:108DA000E66E000E54DB23EC98F013EC4BF0040E4F
:108DB0004EDB41DA8BDB4CD0AFDB080ED5DB07E2B4
:108DC000F297EEA345D037DA6AEC59F008D0A4DB6D
:108DD000100ECADB07E2F2992EDA36EC59F0E552B2
:108DE000E55236D099DB020EBFDB02E2F29306D0E9
:108DF00093DB010EB9DB02E2F2912AD009019F5107
:108E0000000816E20501ED51000812E20A015E5168
:108E10000FE10901E85100080BE23EEC4BF0020EB5
:108E2000E66E69EC30F0E552020802E02AEC2EF022
:108E300062DB02E39DDB0CE159DB0AE20901680E0B
:108E4000FC6F4C0EFD6F010EC1DA02D03CEC7DF0E0
:108E5000080EE15C02E2E16AE552E16E53D20601DE
:108E6000C851200A01E0120053DB02E2E9EF49F0A9
:108E70007FDB14E03EEC4BF00901120EFC6F4D0E4F
:108E8000FD6F010EFE6F54EC3EF0080141510008E9
:108E900003E2010E25DAF9D7020E22DA12002DDAEA
:108EA000030EE1260901EA5104E1EDD90901EB6B5A
:108EB00001D0E9D909019DB907D00F0E0901EB5D79
:108EC00009E2090199AF03D00901EB6B0ED009014A
:108ED000EB2B0BD00F0EEB5D08E109019951800BD4
:108EE00004E1EAC9EBF90701CA930901EB510F0844
:108EF00025E209019951800B21E1020E0701CA15F3
:108F00000AE10F0E0901EB5D0901D880EA5503E380
:108F10000701CA830CD0020E0701CA150FE00D0E1F
:108F20000901EB5D0901EA5D09E30701CA93080E37
:108F3000E66EE66AFEEC3EF0E552E5520601C851E7
:108F4000200A1BE1E5DA02E244DA17D00901E7055D
:108F500010E10901E85100080CE293DB5BDB01E062
:108F60005EDB0C0E24D901E086DB2BD902E02AEC73
:108F70002EF0010E0601C919C96F030EE15C02E271
:108F8000E16AE552E16EBED112006ADB0AE0020E30
:108F9000945D07E00F0E945D04E0ADDA02E3000E8D
:108FA00001D0010E5CDA49E1050E0901A05D29E25C
:108FB000800E0901991525E10601F0510FE1090123
:108FC000E7050DE10A015E510AE10601EEA502D0B6
:108FD000BAEC38F00601480EF06F01D0F007060138
:108FE000EF510DE1FCD90601EEA505D024D94BECDB
:108FF00059F0E552E5520601480EEF6F06D0EF0733
:1090000004D00601060EEF6FF06F0901E70515E1C8
:109010000901E85112E1030EDB500FE079DA02E2B8
:10902000D8D90BD0F7DA01E0FADA0C0EC0D801E09B
:1090300022DBC7D802E02AEC2EF0040EE15C02E24B
:10904000E16AE552E16E5ED10BDB0AE0020E945D4F
:1090500007E00F0E945D04E04EDA02E3000E01D04B
:10906000010EFDD918E10901E70515E10901E851F3
:1090700012E1030EDB500FE14BDA02E2AAD90BD06A
:10908000C9DA01E0CCDA0C0E92D801E0F4DA99D812
:1090900002E02AEC2EF0040EE15C02E2E16AE55205
:1090A000E16E30D10601F351000801E2F307D02B45
:1090B000000ED123CD51000810E2CEC600F0CFC67D
:1090C00001F0CE07000ECF5B0050011006E1CDC6C7
:1090D000E6FFB7EC3FF0E55201D056DD5BD91E0E3E
:1090E0002D6E2E6A83D801E1BADE42DA01E1D7DEC5
:1090F00051D92C0E2D6E010E2E6E78D801E144DF71
:1091000049D9580E2D6E020E2E6E70D801E13DDF4A
:1091100041D9100E2D6E0E0E2E6E68D806E194DF2A
:10912000100E0601D05F0E0ED15B0601D407000EB3
:10913000D55BD451D5111EE1E66A36D8060196DA20
:109140000501EF2BEF51E66EE66AE66AE66AE66A2B
:10915000000EE66E060EE66EA0EC74F0006E070ED2
:10916000E15E0050000EE66E060EE66E1A0E95D910
:109170003EEC72F012001200800E946E33ECA0F000
:109180000901E66BE66AB7EC3FF0E552120084DABB
:10919000006E070EE15E005000091200F5D9000EC6
:1091A000E66EE66ACCD944D273DA44EF4BF0E66E51
:1091B0000FDA010EDBCFE9FF020EDBCFEAFFEF5043
:1091C0001200DFCFE6FF74EC2FF0EAD969EC30F043
:1091D000E7D988EC30F0E4D976EC31F0E1D920EC35
:1091E00032F0E552DF6E020EDF5C1200D0C628F0CE
:1091F000D1C629F0F4D15DDAF3CF00F0F4CF01F05D
:10920000F3CFE6FFF4CFE6FFA3EC3EF0E552E552E4
:1092100009011200E3ECA3F006DA42DAADEF4AF0FE
:10922000E66EDFCFE6FF5AEC32F0E552E552E5524A
:10923000E552DF6E1200010EDBCFE6FF020EDBCF40
:10924000E6FF1200000ED8800054000E01541200F8
:10925000CEC600F0CFC601F0030E2D6E2E6ACEC62C
:1092600028F0CFC629F0BBD1FCC9F6FFFDC9F7FF36
:10927000FEC9F8FF0800F5501200EA6A000FE96E17
:10928000070EEA221200CCECA7F026C000F027C09F
:1092900001F028C002F029C003F02C6A2D6A200ECC
:1092A0002E6E410E2F6E26C027F001C028F002C09E
:1092B00029F003C02AF041EC83F0B6EC84F029C019
:1092C000EAF91200E66E000EE66EE66AE3ECA3F041
:1092D000AAD9020EF3CFDBFF030EF4CFDBFF12009F
:1092E000E66E58EC72F0E5521200FD0EDBCFE9FF9E
:1092F000FE0EDBCFEAFFEF501200D9CFE6FFE1CF41
:10930000D9FF1200E552E7CFD9FF1200E66E4FEC0D
:10931000A0F0E55200091200BFD9016E070EE15E10
:1093200001500009120037D978EC89F0E552E55276
:109330001200E66EE66A90EF4AF0E66E2CD9C8ECB1
:1093400098F0026E050EE15E0250F3CF00F0F4CF0C
:1093500001F0F350F4101200E66EF1D869D1E6681E
:1093600097D9E668E66ADCD8F3EFA1F07FD936EC4E
:1093700041F00601EA6B12009CD950EF4BF0E66E0B
:1093800087D9090112000601D26BD36B0901050EC2
:10939000E66F1200D0C600F0D1C601F01200E66EF2
:1093A0009AEC98F0006E060EE15E00501200D95063
:1093B000020FE96EDACFEAFFEE50ED101200CE6F29
:1093C000CF6BC96B0901E86B0AEF2EF0FE6F54EF0B
:1093D0003EF0050E0601D05F000ED15B1200E66A7A
:1093E000E8EF4AF0DECFE9FFDDCFEAFF120078ECCC
:1093F00089F0E552E552F3CFECF606013C0EED6F35
:1094000012000601030ECD6F5F0ECE6FCF6BC96BDE
:10941000090112000601CA07000ECB5BD880CA55AD
:10942000000ECB551200B7D86CEC73F0E552E55244
:109430001200EA51006E016AC80E001812000026E0
:10944000000E012200C0E6FF01C0E6FF1200E66E3A
:10945000D950030FE66E000EDA20E66E1200E76EBA
:10946000030EE7CFDBFF0601C851200A12002B0EC6
:109470000701005D12004F0E0701005D1200020E91
:10948000DBCFE9FF030EDBCFEAFF1200020EDBCFDA
:10949000E6FF030EDBCFE6FF1200E66E63EC9FF003
:1094A000E552E552E55212000901A80EFC6F4C0E80
:1094B000FD6F010E12000901910EFC6FD90EFD6FB8
:1094C000000E1200EAC6E6FF9AEF4AF0DBEC60F00D
:1094D00013EF4BF0DBCF03F0001E011E021E031E34
:1094E00012000A0E0601CA6FCB6B1200010E0601B4
:1094F000EE1500081200800E0901991500081200EF
:10950000050EE66EE66A1200060EE66EE66A1200C8
:109510000A015E5100081200000EF115006E1200E3
:10952000CCECA1F0E552E5521200F115006E016A93
:1095300022EF49F0000EE66E070EE66E1200E3EC35
:10954000A3F0026E050EE15E025050EF4BF0C50E27
:10955000E66ED90EE66E000E1200D9CFE9FFDACF23
:10956000EAFFEE50ED101200F215016E22EF49F005
:1095700011DF3C0E2D6E2E6AF6EF48F0EA51EA2B11
:109580007CDEDFCFEFFF1200D60EE66ED80EE66E61
:10959000000EE66E1200DECFE6FFDDCFE6FF120022
:1095A000E552DF6EDFCFE6FF1200E66ED4EF48F043
:1095B000A7DF5B0EE66ED90EE66E000EC7EF48F031
:1095C0001ADE360EFC6FD90EFD6F000EE6EF49F085
:1095D0001CEC9FF0E552DE5263D8DD52120066ECBF
:1095E000A8F024C000F025C001F02450251012007E
:1095F0000A0EE66EE66A680EE66ED90EE66E000E9C
:1096000012000B0EE66EE66AE10EE66ED80EE66E0E
:10961000000E1200020EDF6E0B0ED7EF48F00BDECD
:10962000010E10EF49F0006E050EE15E00501200D1
:10963000DECF00F0DDCF01F0005001101200EA5142
:109640001CDEEF6AB6EF49F058DEE6527F0E0601E7
:10965000C85D1200E66E000EE66EE66A0AEF49F09B
:109660004CDE040EE126090194051200080ED46FA9
:10967000070ED56F1200DFDD10EF49F0020E70EF1C
:1096800049F00A0E70EF49F0E66AE66A90EF4AF098
:10969000010EE66E90EF4AF0E66E4CDF2AEF97F08F
:1096A000F3CFDEFFF4CFDDFF120051DF0BDED7EF8B
:0C96B00049F0E66E1CEC9FF0E552120041
:0496BC0018EC58F05E
:1096C0005EEC58F0EE6AEE6AEE6AEE6A91EC57F0E4
:1096D000EE6AEE6AEE6AEE6ACDEC54F0010EEE6EC2
:1096E000230EEE6E450EEE6E670EEE6ECDEC54F070
:1096F000040E0FEC56F0890EEE6EAB0EEE6ECD0E34
:10970000EE6EEF0EEE6ECDEC54F0080E0FEC56F050
:10971000FE0EEE6EDC0EEE6EBA0EEE6E980EEE6E75
:10972000CDEC54F00C0E0FEC56F0760EEE6E540E9F
:10973000EE6E320EEE6E100EEE6EE552E7CFD9FFF2
:10974000120018EC58F0080EE126030E046E91EC9E
:1097500057F043EC56F003E063EC56F0FDE13F0EAA
:1097600000169DEC56F0D2EC57F0F90EDBCF04F06A
:10977000FA0EDBCF05F0066A076A05AE02D006686E
:109780000768030E1F0B07E0D8900436053606362F
:109790000736E806F9E191EC57F00450EF26EECFDA
:1097A00000F00550EF22EECF01F00650EF22EECF91
:1097B00002F00750EF22EECF03F0F90EDBCF08F0F6
:1097C000FA0EDBCF09F00A6A0B6A09AE02D00A680A
:1097D0000B68030E1F0B03E074EC56F0FDE108501C
:1097E000005C095001580A5002580B50035806E219
:1097F0005EEC58F0EE2AEE22EE22EE227BEC56F0E2
:10980000026A036A01AE02D0026803681D0E63ECAF
:1098100056F0FDE15EEC58F00BEC58F0400E046E93
:10982000056A066A076AD9CFE9FF49EC56F0EE509F
:109830000758060E00C0DBFF070E01C0DBFF7BEC04
:1098400056F035EC58F001500318E8AE02D003345E
:1098500004D00250005C035001586AE3060EDBCFCF
:10986000E6FF070EDBCFE6FF37EC56F014EC58F0BE
:10987000E9CF02F0EACF03F0DB50E924006E010EDD
:10988000DB50EA2093EC56F049EC97F0046E060E9C
:10989000E15E045014EC58F02EEC56F0CDEC54F090
:1098A000E9CF02F0EACF03F052EC56F0060EDBCF20
:1098B00028F0070EDBCF29F0040E28C0DBFF050ED1
:1098C00029C0DBFF3F0EE76EFBEC57F0E7500026A8
:1098D000000E0122F4EC57F001500318E8AE02D05C
:1098E000033404D00250005C035001581EE2040E01
:1098F000DBCF02F0050EDBCF03F0FB0EDB500224C2
:10990000006EFC0EDB50032093EC56F0CDEC54F0CF
:10991000E9CF04F0EACF05F052EC56F051EC58F0E4
:10992000400EEE26000EED22CDD73CEC58F004D0D0
:10993000040EDB6A050EDB6AF4EC57F0040EDB5014
:10994000025C006E050EDB50035893EC56F06AEC97
:1099500056F0046EFC0EDB500720056E04C0E6FFD7
:10996000E66E14EC58F0E9CF0AF0EACF0BF0DB50CA
:10997000E924086E010EDB50EA20096E08C0E6FFFC
:10998000E66E49EC97F00C6E060EE15E0C50080E88
:10999000E15C02E2E16AE5523EEF56F088EC56F0F7
:1099A000080E5DEC56F0100E0FEC56F02EEC56F053
:1099B000D9CFE6FFDACFE6FF82EC56F0030E046E55
:1099C00043EC58F0100E0FEC56F043EC56F003E069
:1099D00063EC56F0FDE13F0E00169DEC56F081EC75
:1099E00057F0380EEE5C000EEE58000EEE58000EEA
:1099F000EE580DE2380E046E056A066A076A5AECE4
:109A000058F049EC56F0026EEE50075813D0780E1D
:109A1000086E096A0A6A0B6A5AEC58F0A2EC58F010
:109A2000085C006EEE500958016EEE500A58026E46
:109A3000EE500B58036E9EEC57F00C0EDBCFE6FF9A
:109A40000D0EDBCFE6FF000EE66E0B0EE66E37EC7A
:109A500056F08CEC56F0080EE66EE66AD9CFE6FFBB
:109A6000DACFE6FF37EC56F08CEC56F0100E5DECDA
:109A700056F02EEC56F0FD0EDBCFE6FFFE0EDBCFF0
:109A8000E6FF82EC56F0100EE15C02E2E16AE5527C
:109A90003EEF56F088EC56F0CDEC54F0EECFDFFF01
:109AA000010EEECFDBFF020EEECFDBFF030EEECF9B
:109AB000DBFF040E73EC57F0040EEECFDBFF050E58
:109AC000EECFDBFF060EEECFDBFF070EEECFDBFFA8
:109AD000080E73EC57F0080EEECFDBFF090EEECF49
:109AE000DBFF0A0EEECFDBFF0B0EEECFDBFF0C0E23
:109AF00073EC57F00C0EEECFDBFF0D0EEECFDBFF5D
:109B00000E0EEECFDBFF0F0EEECFDBFF400EE66E4C
:109B1000E66AE66AE66A37EC56F0A20EE66E0A0ED0
:109B2000E66E43EC53F0006E080EE15E0050E7EC89
:109B300056F02EEC55F0780E0026A40E01226A0E87
:109B40000222D70E1DEC58F003E073EC54F0FDE157
:109B500045EC54F0190E62EC54F0FDE1A1EC56F026
:109B60003BEC55F0560E0026B70E0122C70E02221E
:109B7000E80E8FEC58F003E073EC54F0FDE155EC87
:109B800054F0140E62EC54F0FDE1BCEC56F048ECDD
:109B900055F0DB0E0026700E0122200E0222240E4C
:109BA00062EC58F003E073EC54F0FDE138EC54F053
:109BB0000F0E62EC54F0FDE1D4EC56F055EC55F08C
:109BC000EE0E0026CE0E0122BD0E0222C10E93EC37
:109BD00058F003E073EC54F0FDE148EC54F00A0E49
:109BE00062EC54F0FDE197EC58F062EC55F0AF0EEA
:109BF00000260F0E01227C0E0222F50E1DEC58F0FD
:109C000003E073EC54F0FDE145EC54F0190E62EC06
:109C100054F0FDE1A1EC56F06FEC55F02A0E002651
:109C2000C60E0122870E0222470E8FEC58F003E089
:109C300073EC54F0FDE155EC54F0140E62EC54F06A
:109C4000FDE1BCEC56F07CEC55F0130E0026460E00
:109C50000122300E0222A80E62EC58F003E073ECF1
:109C600054F0FDE138EC54F00F0E62EC54F0FDE1DD
:109C7000D4EC56F089EC55F0002A950E0122460EE0
:109C80002FEC58F0160E1F0B03E073EC54F0FDE1BF
:109C900048EC54F00A0E62EC54F0FDE197EC58F0F9
:109CA00096EC55F0D80E0026980E0122800E022266
:109CB000690E1DEC58F003E073EC54F0FDE145EC47
:109CC00054F0190E62EC54F0FDE1A1EC56F0A3EC57
:109CD00055F0AF0E0026F70E0122440E02228B0E25
:109CE0008FEC58F003E073EC54F0FDE155EC54F0C8
:109CF000140E62EC54F0FDE1BCEC56F0B0EC55F003
:109D0000B10E00265B0E0122FF0E022262EC58F01B
:109D100003E073EC54F0FDE138EC54F00F0E62EC0C
:109D200054F0FDE1D4EC56F0BDEC55F0BE0E00262B
:109D3000D70E01225C0E0222890E93EC58F003E04C
:109D400073EC54F0FDE148EC54F00A0E62EC54F070
:109D5000FDE197EC58F0CAEC55F0220E0026110EEA
:109D60000122900E02226B0E1DEC58F003E073EC02
:109D700054F0FDE145EC54F0190E62EC54F0FDE1B5
:109D8000A1EC56F0D7EC55F0930E0026710E01228F
:109D9000980E98EC56F00C0F12EC54F094EC54F032
:109DA0000C0E1F0B03E073EC54F0FDE155EC54F086
:109DB000140E62EC54F0FDE1BCEC56F0E4EC55F00E
:109DC0008E0E0026430E0122790E0222A60E62ECB0
:109DD00058F003E073EC54F0FDE138EC54F00F0E52
:109DE00062EC54F0FDE1D4EC56F0F1EC55F0210EAC
:109DF0000026080E0122B40E0222490E93EC58F000
:109E000003E073EC54F0FDE148EC54F00A0E62EC10
:109E100054F0FDE108EC57F03BEC55F0620E0026E3
:109E2000250E01221E0E0222F60E21EC58F003E050
:109E300073EC54F0FDE145EC54F01B0E62EC54F071
:109E4000FDE124EC57F07CEC55F0400E0026B30EFB
:109E50000122400E0222C00E66EC58F003E073ECC3
:109E600054F0FDE155EC54F0170E62EC54F0FDE1B6
:109E7000FBEC56F0BDEC55F0510E00265A0E0122B7
:109E80005E0E0222260E6AEC58F003E073EC54F0EA
:109E9000FDE138EC54F0120E62EC54F0FDE110ECF0
:109EA00057F02EEC55F0AA0E0026C70E0122B60E72
:109EB0000222E90E6EEC58F003E073EC54F0FDE181
:109EC00048EC54F00C0E62EC54F0FDE108EC57F055
:109ED0006FEC55F05D0E0026100E01222F0E0222AF
:109EE000D60E21EC58F003E073EC54F0FDE145ECA4
:109EF00054F01B0E62EC54F0FDE124EC57F0B0EC92
:109F000055F0530E0026140E0122440E0222020EBA
:109F100066EC58F003E073EC54F0FDE155EC54F0BE
:109F2000170E62EC54F0FDE1FBEC56F0F1EC55F04D
:109F3000810E0026E60E0122A10E0222D80E6AEC46
:109F400058F003E073EC54F0FDE138EC54F0120EDD
:109F500062EC54F0FDE110EC57F062EC55F0C80EE5
:109F60000026FB0E0122D30E0222E70E6EEC58F003
:109F700003E073EC54F0FDE148EC54F00C0E62EC9D
:109F800054F0FDE108EC57F0A3EC55F0E60E002686
:109F9000CD0E0122E10E0222210E21EC58F003E049
:109FA00073EC54F0FDE145EC54F01B0E62EC54F000
:109FB000FDE124EC57F0E4EC55F0D60E0026070E38
:109FC0000122370E0222C30E66EC58F003E073EC58
:109FD00054F0FDE155EC54F0170E62EC54F0FDE145
:109FE000FBEC56F055EC55F0870E00260D0E0122C5
:109FF000D50E0222F40E6AEC58F003E073EC54F034
:10A00000FDE138EC54F0120E62EC54F0FDE110EC7E
:10A0100057F096EC55F0ED0E0026140E01225A0E64
:10A020000222450E6EEC58F003E073EC54F0FDE1B3
:10A0300048EC54F00C0E62EC54F0FDE108EC57F0E3
:10A04000D7EC55F0050E0026E90E0122E30E0222A0
:10A05000A90E21EC58F003E073EC54F0FDE145EC5F
:10A0600054F01B0E62EC54F0FDE124EC57F048EC88
:10A0700055F0F80E0026A30E0122EF0E0222FC0E70
:10A0800066EC58F003E073EC54F0FDE155EC54F04D
:10A09000170E62EC54F0FDE1FBEC56F089EC55F044
:10A0A000D90E0026020E01226F0E0222670E6AEC04
:10A0B00058F003E073EC54F0FDE1DADB120E62ECD1
:10A0C00054F0FDE110EC57F0CAEC55F08A0E002672
:10A0D0004C0E01222A0E02228D0E6EEC58F003E087
:10A0E00073EC54F0FDE1D4DB0C0EECDBFEE13FEC55
:10A0F00057F06FEC55F0420E0026390E0122FA0E91
:10A100000222FF0E25EC58F002E0EDDBFEE1BDDBA4
:10A110001C0ED8DBFEE157EC57F096EC55F0810EA3
:10A120000026F60E0122710E0222870E72EC58F004
:10A1300002E0D9DBFEE1B9DB150EC4DBFEE146EC43
:10A1400057F0BDEC55F0220E0026610E01229D0E47
:10A1500002226D0E76EC58F002E0C5DBFEE188DBF2
:10A16000100EB0DBFEE15FEC57F0E4EC55F00C0EA6
:10A170000026380E0122E50E2FEC58F0170E1F0BAB
:10A1800002E0B1DBFEE184DB090E9CDBFEE13FEC8B
:10A1900057F03BEC55F0440E0026EA0E0122BE0EAD
:10A1A0000222A40E25EC58F002E09DDBFEE16DDBFF
:10A1B0001C0E88DBFEE157EC57F062EC55F0A90E5F
:10A1C0000026CF0E0122DE0E02224B0E72EC58F05A
:10A1D00002E089DBFEE169DB150E74DBFEE146EC93
:10A1E00057F089EC55F0600E00264B0E0122BB0E95
:10A1F0000222F60E76EC58F002E075DBFEE138DB69
:10A20000100E60DBFEE15FEC57F0B0EC55F0700E25
:10A210000026BC0E0122BF0E0222BE0E9BEC58F09F
:10A2200002E061DBFEE134DB090E4CDBFEE13FECDA
:10A2300057F0D7EC55F0C60E00267E0E01229B0E7D
:10A240000222280E25EC58F002E04DDBFEE11DDB7A
:10A250001C0E38DBFEE157EC57F02EEC55F0FA0EF1
:10A260000026270E0122A10E0222EA0E72EC58F0FF
:10A2700002E039DBFEE119DB150E24DBFEE146ECE2
:10A2800057F055EC55F0850E0026300E0122EF0EEA
:10A290000222D40E76EC58F002E025DBFEE1E8DA8B
:10A2A000100E10DBFEE15FEC57F07CEC55F0050E74
:10A2B00000261D0E0122880E0222040E9BEC58F08F
:10A2C00002E011DBFEE1E4DA090EFCDAFEE13FEC2C
:10A2D00057F0A3EC55F0390E0026D00E0122D40E13
:10A2E0000222D90E25EC58F002E0FDDAFEE1CDDACB
:10A2F0001C0EE8DAFEE157EC57F0CAEC55F0E50E1B
:10A300000026990E0122DB0E0222E60E72EC58F0B6
:10A3100002E0E9DAFEE1C9DA150ED4DAFEE146EC34
:10A3200057F0F1EC55F0F80E00267C0E0122A20E3B
:10A3300002221F0E76EC58F002E0D5DAFEE198DA40
:10A34000100EC0DAFEE15FEC57F0A2DB650E0026CE
:10A35000560E0122AC0E0222C40E9BEC58F002E015
:10A36000C2DAFEE195DA090EADDAFEE12DEC57F026
:10A3700075DB440E0026220E0122290E0222F40E65
:10A380002AEC58F002E0AFDAFEE17FDA1A0E9ADA30
:10A39000FEE118EC57F0BDDB970E0026FF0E012200
:10A3A0002A0E0222430E7AEC58F002E09CDAFEE11B
:10A3B0007CDA160E87DAFEE14DEC57F0E4EC55F04E
:10A3C000A70E0026230E0122940E0222AB0E7EEC75
:10A3D00058F002E088DAFEE14BDA110E73DAFEE1A2
:10A3E00036EC57F07CDB390E0026A00E0122930ECE
:10A3F0000222FC0E82EC58F002E075DAFEE148DA47
:10A400000B0E60DAFEE12DEC57F0C4DBC30E002624
:10A41000590E01225B0E0222650E2AEC58F002E072
:10A4200062DAFEE132DA1A0E4DDAFEE118EC57F08C
:10A430003CDB920E0026CC0E01220C0E02228F0E67
:10A440007AEC58F002E04FDAFEE12FDA160E3ADA33
:10A45000FEE14DEC57F084DB7D0E0026F40E012268
:10A46000EF0E0222FF0E7EEC58F002E03CDAFEE135
:10A47000FFD9110E27DAFEE136EC57F0FCDAD10EE7
:10A4800000265D0E0122840E0222850E82EC58F019
:10A4900002E029DAFEE1FCD90B0E14DAFEE12DEC24
:10A4A00057F044DB4F0E00267E0E0122A80E02223A
:10A4B0006F0E2AEC58F002E016DAFEE1E6D91A0E29
:10A4C00001DAFEE118EC57F08CDBE00E0026E60E18
:10A4D00001222C0E0222FE0E7AEC58F002E003DA82
:10A4E000FEE1E3D9160EEED9FEE14DEC57F004DBA8
:10A4F000140E0026430E0122010E0222A30E7EEC52
:10A5000058F002E0F0D9FEE1B3D9110EDBD9FEE13B
:10A5100036EC57F04CDBA10E0026110E0122080E7E
:10A5200002224E0E82EC58F002E0DDD9FEE1B0D9F5
:10A530000B0EC8D9FEE12DEC57F0C4DA820E0026CE
:10A540007E0E0122530E0222F70E2AEC58F002E092
:10A55000CAD9FEE19AD91A0EB5D9FEE118EC57F026
:10A560000CDB350E0026F20E01223A0E0222BD0E41
:10A570007AEC58F002E0B7D9FEE197D9160EA2D9CD
:10A58000FEE14DEC57F084DABB0E0026D20E01221C
:10A59000D70E02222A0E7EEC58F002E0A4D9FEE18A
:10A5A00067D9110E8FD9FEE136EC57F0CCDA910E57
:10A5B0000026D30E0122860E0222EB0E82EC58F00A
:10A5C00002E091D9FEE164D90B0E7CD9FEE10BD9F2
:10A5D000E4D9DEEC57F0040E73EC57F0C5EC57F0FD
:10A5E000080E73EC57F0B8EC57F00C0E73EC57F004
:10A5F000ABEC57F0100EE15C02E2E16AE5523ED3AB
:10A6000012DBFCDA3AE2DFCF06F0010EDBCF07F017
:10A61000D89006360736D89006360736FB0EDB5044
:10A62000062431EC58F00720EA6EEECF02F002501B
:10A63000E66EFBEC57F0B8D9080E44D9FEE10450A1
:10A64000E66E010E67EC57F0AFD9100E3BD9FEE174
:10A650000450E66E020E67EC57F0A6D9180E32D9F8
:10A66000FEE10450E66E030E67EC57F095EC57F0F0
:10A67000E552E750EF6EE4DAC4D7080EE15C02E27F
:10A68000E16AE552FBD2CFDAB9DA01E3A2D022DBEC
:10A6900031EC58F00720EA6EEFCF02F0036A046A4B
:10A6A000056A010E0C6E0D6A0E6A0F6A51EC58F0C5
:10A6B000EE500C26EE500D22EE500E22EE500F22E0
:10A6C000FB0EDB500C2431EC58F00D20EA6EEFCF7E
:10A6D00008F0096A0A6A0B6A080E1F0B02E004DB25
:10A6E000FEE108500212095003120A5004120B50E6
:10A6F0000512020E146E156A166A176A51EC58F0AC
:10A70000EE501426EE501522EE501622EE5017226F
:10A71000FB0EDB50142431EC58F01520EA6EEFCF1D
:10A7200010F0116A126A136A100E1F0B07E0D8901E
:10A730001036113612361336E806F9E110500212BF
:10A74000115003121250041213500512030E1C6E06
:10A750001D6A1E6A1F6A51EC58F0EE501C26EE501E
:10A760001D22EE501E22EE501F22FB0EDB501C2439
:10A7700031EC58F01D20EA6EEFCF18F0196A1A6A12
:10A780001B6A180E1F0B07E0D890183619361A36B8
:10A790001B36E806F9E118500212195003121A503C
:10A7A00004121B500512DFCF00F0010EDBCF01F0C9
:10A7B000D89000360136D89000360136B6DB02C09C
:10A7C000EEFF03C0EEFF04C0EEFF05C0EEFF38DA77
:10A7D0005BD7080EE15C02E2E16AE5524FD288DB0A
:10A7E00090DBABEF57F084DB040E00C0DBFF050EFF
:10A7F00001C0DBFF060E02C0DBFF070E03C0DBFF5C
:10A8000051EC58F0B8EF57F073DB98DB86EC58F05A
:10A81000DACFEAFFDEEF57F06BDBC4DB55EC58F024
:10A82000C5EF57F0E96EDACFEAFF0BEF58F0DACF59
:10A83000EAFF0C50EE14086E0D50EE14096E0E5027
:10A84000EE140A6E0F50EE140B6EC4D303220050A8
:10A85000DE260150DE220250DE220350DD22DD52D0
:10A86000DD5255EC58F04AEC58F0EFCF03F01200EF
:10A87000080EDBCF04F0090EDBCF05F00A0EDBCFAC
:10A8800006F00B0EDBCF07F0120055EC58F0BAD3F0
:10A89000040EDBCF04F0050EDBCF05F0060EDBCF98
:10A8A00006F0070EDBCF07F012000C0EDBCF04F032
:10A8B0000D0EDBCF05F00E0EDBCF06F00F0EDBCF5B
:10A8C00007F01200D8900732063205320432E8064B
:10A8D0001200A2EC58F00816EE500916EE500A16B7
:10A8E000EE500B1677D3D890003601360236033679
:10A8F000E8061200A2EC58F00416EE500516EE50D1
:10A900000616EE5007161200DACFEAFF0850EE18CE
:10A91000046E0950EE18056E0A50EE18066E0B50C4
:10A92000EE18076E045012000C0EDBCF00F00D0E77
:10A93000DBCF01F00E0EDBCF02F00F0EDBCF03F00A
:10A940001200080EDBCF00F0090EDBCF01F00A0E7B
:10A95000DBCF02F00B0EDBCF03F012004CDB35EF48
:10A9600058F0F0DB041AEE50051AEE50061AEE50BD
:10A97000071A04501200E6DB081AEE50091AEE50CE
:10A980000A1AEE500B1A1200DDDB0412EE5005120B
:10A99000EE500612EE5007121200FD0EDBCFE9FF5B
:10A9A000FE0EDBCFEAFF1200C0DAE552E750EF6E91
:10A9B000DFCF08F0010EDBCF09F0D890083609365A
:10A9C000D89008360936FB0EDB5008244ADB0920F4
:10A9D000EA6E18D30C0EDBCF08F00D0EDBCF09F0BA
:10A9E0000E0EDBCF0AF00F0EDBCF0BF01200080EBD
:10A9F000DBCF08F0090EDBCF09F00A0EDBCF0AF03F
:10AA00000B0EDBCF0BF01200040EDBCF08F0050EAF
:10AA1000DBCF09F0060EDBCF0AF0070EDBCF0BF021
:10AA2000120043DBEECF08F0EECF09F0EECF0AF0D4
:10AA3000EFCF0BF01200DBCF0FF00C1E0D1E0E1E21
:10AA40000F1E1200081E091E0A1E0B1ED9501200EE
:10AA5000041E051E061E071ED95012000A01A2255B
:10AA6000006E0550A321016E0650A421026E07500E
:10AA7000A521036E12000A01A625006E0550A7212C
:10AA8000016E0650A821026E0750A921036E120024
:10AA90000A01AA25006E0550AB21016E0650AC21BB
:10AAA000026E0750AD21036E12000A01AE25006E42
:10AAB0000550AF21016E0650B021026E0750B12142
:10AAC000036E12000A01B225006E0550B321016E1B
:10AAD0000650B421026E0750B521036E12000A0120
:10AAE000B625006E0550B721016E0650B821026EE2
:10AAF0000750B921036E12000A01BA25006E0550F5
:10AB0000BB21016E0650BC21026E0750BD21036EB1
:10AB100012000A01BE25006E0550BF21016E0650CD
:10AB2000C021026E0750C121036E12000A01C22526
:10AB3000006E0550C321016E0650C421026E0750FD
:10AB4000C521036E12000A01C625006E0550C721FB
:10AB5000016E0650C821026E0750C921036E120013
:10AB60000A01CA25006E0550CB21016E0650CC218A
:10AB7000026E0750CD21036E12000A01CE25006E31
:10AB80000550CF21016E0650D021026E0750D12111
:10AB9000036E12000A01D225006E0550D321016E0A
:10ABA0000650D421026E0750D521036E12000A010F
:10ABB000D625006E0550D721016E0650D821026EB1
:10ABC0000750D921036E12000A01DA25006E0550E4
:10ABD000DB21016E0650DC21026E0750DD21036E81
:10ABE00012000A01DE25006E0550DF21016E0650BD
:10ABF000E021026E0750E121036E1200F70EDBCF59
:10AC000000F0F80EDBCF01F0EFD94BDA0050EE5C2C
:10AC10000150EE580250EE580350EE581200E9264B
:10AC2000000EEA22120004DA080EE12625DA040EEC
:10AC3000DB6A050EDB6A060EDB6A070EDB6A1200B2
:10AC400034DAEE2A000EEE22EE22EE222ADA040E8A
:10AC5000EE26000EEE22EE22EE221200E9CF00F0E8
:10AC6000EACF01F0E9CFE6FFEACFE6FF1200FB0EE4
:10AC7000DBCFE6FFFC0EDBCFE6FF1200E16EE55214
:10AC8000E7CFD9FF120004501F0B04DAEECF03F018
:10AC9000120058DA045C006EEE500558016EEE505A
:10ACA00006581200E9CFE6FFEACFE6FF4AEC4DF086
:10ACB000E552E552E552E5521200E66EE66AE66AB2
:10ACC000E66A43EF58F0D890033202320132003284
:10ACD000E8061200040EDBCF06F0050EDBCF07F00E
:10ACE000FB0EDB5006241200D890083609360A36CF
:10ACF0000B36E8061200F90EDBCF00F0FA0EDBCFC0
:10AD000001F012007DDC026E080EE15E02501200BE
:10AD10008FD9100EE1261200A1EC4BF0006E060E4A
:10AD2000E15E00501200016E00C0E6FFE66E120008
:10AD30000222FD0E0322D9501200016A026A036A40
:10AD400012006ADDA5DDD9CFE9FFD4DDAED9EECFA3
:10AD50000CF0EECF0DF0EECF0EF0EFCF0FF00C1E9B
:10AD60000D1E0E1E0F1EA6D917EF54F00322D95048
:10AD7000080F58DDA1EF54F047DD87DDC7D9BADDF4
:10AD80000C0EDBCF0CF00D0EDBCF0DF00E0EDBCF7B
:10AD90000EF00F0E50DEDAD917EF54F00322D9501F
:10ADA0000C0F40DD94EF54F01ADD7FDD83D9A2DD76
:10ADB000080EDBCF0CF0090EDBCF0DF00A0EDBCF57
:10ADC0000EF00B0E38DED9CFE9FF17EF54F050DD4F
:10ADD000BDD990DD040EDBCF0CF0050EDBCF0DF0FE
:10ADE000060EDBCF0EF0070E26DE90D917EF54F0DB
:10ADF0000322D9508FD108DD4BDD88D97BDD04DEFD
:10AE0000081E091E0A1E0B1ED9CFE9FF69EF54F078
:10AE1000EADC4BDD9BD96EDDDDDD14DE080F8FD162
:10AE2000DEDC33DD47D966DDFCDD0CDE0C0F87D1BF
:10AE3000F3DC1EDD041E051E061E071ED9CFE9FF2A
:10AE4000A3DD84D9B1EF54F0E7DC12DDD9CFE9FFFF
:10AE500051DDCDDDF7DD040F72D1C5DC26DDF8DD77
:10AE6000040FE96E91DD26D9B1EF54F0B8DC0DDDA9
:10AE7000EFDD080FE96E88DD49D9B1EF54F0B3DC9E
:10AE8000B6DD64D978DD42D984EF54F0BDDCC9DD8C
:10AE90003DD971DD5BD984EF54F0B6DCF9DCD8DD47
:10AEA0000C0FE96E71DDD9CFE9FFB1EF54F0B4DCDE
:10AEB000ABDDD9CFE9FF5FDDFDD884EF54F08FDC47
:10AEC00089DDF8D858DDD9CFE9FF84EF54F0006E62
:10AED00034DFE7D8EE500026EE500122EE50022279
:10AEE000EE5003221200E76E58DDE7500FEF56F0E8
:10AEF00004500012055001120650021207500312AE
:10AF00001200080E00C0DBFF090E01C0DBFF0A0EB5
:10AF100002C0DBFF0B0E03C0DBFFCCD8DACFEAFFA9
:10AF200012003BDD100E0FEF56F0FD0EDB5000243B
:10AF3000E96EFE0EDB500120EA6E12000C0E00C01E
:10AF4000DBFF0D0E01C0DBFF0E0E02C0DBFF0F0E9C
:10AF500003C0DBFF12000C0EDB50EE260D0EDB50A3
:10AF6000EE220E0EDB50EE220F0EDB50EE22120010
:10AF7000080EDB50EE26090EDB50EE220A0EDB50E7
:10AF8000EE220B0EDB50EE221200040EDB50EE26FA
:10AF9000050EDB50EE22060EDB50EE22070EDB50D4
:10AFA000EE22120000C0DFFF010E01C0DBFF020E27
:10AFB00002C0DBFF030E03C0DBFF1200DF50EE26F2
:10AFC000010EDB50EE22020EDB50EE22030EDB50B0
:10AFD000EE22120008500412095005120A500612FF
:10AFE0000B50071204501200F90EDBCF02F0FA0EDC
:10AFF000DBCF03F01200040EDBCF00F0050EDBCF39
:10B0000001F01200EECF04F0EECF05F0EECF06F027
:10B01000EFCF07F012000050EE260150EE22025052
:10B02000EE220350EE221200B8DC180E0FEF56F09D
:10B03000D9CFE6FFE1CFD9FF120008DC070E1F0BC6
:10B04000120004DC050E1F0B120026EC54F0040E57
:10B050001F0B120026EC54F0060E1F0B120068DEC8
:10B0600059D0E96EFC0EDB501200060EDBCF02F069
:10B07000070EDBCF03F01200DE6ADE6ADE6ADD6AED
:10B08000DD52DD521200FB0EDBCFE9FFFC0EDBCF01
:10B09000EAFF1200EECF00F0EECF01F0EECF02F0AB
:10B0A000120054D8DACFEAFF1200D9CFE9FFDACF85
:10B0B000EAFF1200D950080FE96E120032DF040EC9
:10B0C0000FEF56F053DE110E1F0B120067DE090E54
:10B0D0001F0B12004BDE0E0E1F0B120089DE140E2A
:10B0E0001F0B12005BDE0B0E1F0B12003FDE100E5B
:10B0F0001F0B120053DE0A0E1F0B120037DE0F0E5D
:10B100001F0B120075DE150E1F0B1200D9500C0F0D
:10B11000E96E1200040F12EC54F0AEEF54F03EDE74
:10B120000C0E1F0B120064DE160E1F0B1200F3EC48
:10B1300053F0E7EF56F05CDE170E1F0B1200E96EBE
:10B1400069EF54F0DACFEAFFEE501200D950040F45
:04B15000E96E120092
:0CB15400ADEC62F06CEC64F009E1090164
:10B16000700EFC6FDF0EFD6F000E0AEC63F017D05F
:10B170000901660EFC6FDF0EFD6F000E0AEC63F036
:10B18000D4EC63F052EC64F00901620EFC6FDF0E48
:10B19000FD6F000E0AEC63F0020E23EC63F0B2EFD9
:10B1A00062F06CEC64F003E1B8EC63F006D00901E6
:10B1B0005D0EFC6FDF0EFD6F000E0AEF63F0ADEC6D
:10B1C00062F00501F3B50BD097EC62F0FBCAFCF915
:10B1D000FCCAFDF9FDCAFEF954EC3EF0E2DFB2EF25
:10B1E00062F0ADEC62F00501F3B509D097EC62F0C6
:10B1F000FECAE6FFFFCAE6FF52EC64F0D2DFB2EF10
:10B2000062F0FCEC63F0F3A502D0000E11D0C0ECAC
:10B2100064F09EEC64F087EC37F0E552E5529EEC6A
:10B2200064F05FEC74F0E552E552B6EC62F0010EAA
:10B230004EEC63F002E2E16AE552E16E0050B2EFDB
:10B2400062F0FCEC63F0F3B509D0E2EC64F0CD0EF3
:10B25000FC6F330EFD6F010E8FEC64F0020EE15CAB
:10B2600002E2E16AE552E16EB2EF62F0FCEC63F0FB
:10B27000F3B509D0E2EC64F0E80EFC6F330EFD6F1D
:10B28000010E8FEC64F0020EE15C02E2E16AE5522D
:10B29000E16EB2EF62F002EC64F00A0EC0EC64F012
:10B2A0000901A051E66EE66A340EE66EDF0EE66E28
:10B2B000000E0CEC64F0DDEC62F02D0EE66EDF0E9D
:10B2C000E66E000E0FEC64F002E2E16AE552E16E18
:10B2D000B2EF62F002EC64F00A0EC0EC64F0070119
:10B2E000CAA308D0ECEC62F0060EE66EDF0EE66E46
:10B2F000000E07D0ECEC62F0EE0EE66EDE0EE66EAF
:10B30000000EE8EC64F0B8EC64F039EC63F0E60EA3
:10B31000E66EDE0EE66E000EF7EC62F0E30EE66E11
:10B32000DE0EE66E000E0FEC64F002E2E16AE5521A
:10B33000E16EB2EF62F002EC64F0E66A1AEC63F0E0
:10B3400044EC63F0FD0EDBCFE6FFFE0E66EC63F02F
:10B3500002E1010E06D00501F3B302D028EC63F040
:10B36000000E4EEC63F002E2E16AE552E16E00503D
:10B37000B2EF62F0CFEC64F0D950FB0FA3EC64F0B5
:10B380000BE044EC63F0FB0EDBCFE6FFFC0E66EC5B
:10B3900063F002E1010E06D00501F3B302D028EC00
:10B3A00063F0000E4EEC63F002E2E16AE552E16EFA
:10B3B0000050B2EF62F0ADEC62F08CEC63F021E093
:10B3C00073EC64F092EC64F0D4EC63F03CEC98F035
:10B3D000CBEC64F0E7CF01F0E552E7CF00F000508E
:10B3E000F3240A01F96F0150F420FA6FF9CA00F052
:10B3F000016EFD0EDB50001807E1FE0EDB50011858
:10B4000003E1F36AF46A16D0FD0EC4EC63F070EC4D
:10B4100064F008E0E0EC62F005E0DF2A010EF7E3FB
:10B42000DB2AF5D770EC64F003E13DEC64F0EF6AE1
:10B4300092EC63F0020EE15C02E2E16AE552E16E39
:10B44000B2EF62F0ADEC62F08CEC63F016E0FD0E52
:10B45000C4EC63F0E0EC62F005E0DF2A010EFAE3F1
:10B46000DB2AF8D7DECF00F0DDCF01F00A01F95179
:10B47000001806E1FA51011803E1F36AF46A21D0D9
:10B48000DF2A010E01E3DB2AD9CFE9FFDACFEAFF99
:10B49000FD0EEECFDBFFFE0EEDCFDBFF70EC64F0B8
:10B4A00008E0E0EC62F005E0DF2A010EF7E3DB2ABA
:10B4B000F5D770EC64F003E13DEC64F0EF6A92ECD8
:10B4C00063F0020EE15C02E2E16AE552E16EB2EF86
:10B4D00062F002EC64F0E66A1AEC63F00501F3A591
:10B4E00002D0000E0BD097EC62F0DBEC63F0CF0ED5
:10B4F000E66EDE0EE66E000EE0EC63F04EEC63F0FE
:10B5000002E2E16AE552E16E0050B2EF62F0ADECAA
:10B5100062F0D4EC63F0E66ABFEC63F0F3A502D00E
:10B52000000E0AD0FFEC63F0900EFC6F320EFD6F40
:10B53000010E0AEC63F0010EB2EF62F0CFEC64F0A2
:10B540000501F3A502D0000E0BD097EC62F0DBEC06
:10B5500063F0BD0EE66EDE0EE66E000EE0EC63F00C
:10B560004EEC63F002E2E16AE552E16E0050B2EFA8
:10B5700062F0ADEC62F0C9EC63F0010EE66EBFEC78
:10B5800063F0F3A502D0000E0AD0FFEC63F0BD0E0D
:10B59000FC6F320EFD6F010E0AEC63F0010EB2EF8C
:10B5A00062F0FCEC63F0F3A502D0000E27D0C0ECF3
:10B5B00064F0D1C9E6FFD2C9E6FFD3C9E6FFD4C91A
:10B5C000E6FF0C0EE66E340EE66E010EE8EC64F05B
:10B5D00098EC63F0D5C9E6FFD6C9E6FFD7C9E6FF08
:10B5E000D8C9E6FFBB0EE66EDE0EE66E000EE5EC99
:10B5F00064F098EC63F0B6EC62F0010E4EEC63F090
:10B6000002E2E16AE552E16E0050B2EF62F0ADECA9
:10B6100062F0D4EC63F0F5DDE552E552B2EF62F092
:10B62000ADEC62F0070EE1260501F3A502D0000E95
:10B6300070D0FFEC63F057EC64F0070EF36E020E6F
:10B64000F3CFDBFFDF6A200EDF5C62E2DFCFE6FFD5
:10B650001CEC9FF0E552030EF3CFDBFF040EF4CF9A
:10B66000DBFF030EDBCFE9FF040EDBCFEAFFEF5079
:10B670004DE0DFCFE6FFE66AB10EE66EDE0EE66E67
:10B68000000E0CEC64F0A0EC63F0030EDBCFE6FFE1
:10B69000040EDBCFE6FFAF0EE66EDE0EE66E000EAA
:10B6A000E66E050EDBCFE6FF060EDBCFE6FF9AEC7B
:10B6B00074F0A0EC63F0050EDBCF00F0060EDBCFDC
:10B6C00001F0000E005E060E015A010E00C0DBFF05
:10B6D000DBCFE6FF020EDB50E552E724006E016A85
:10B6E000013412E20050A008000E01540DE259DDB1
:10B6F000140EE2EC64F057EC64F0010EDB50070F1F
:10B70000E76E020EE7CFDBFFB6EC62F0DF2A9BD7D5
:10B71000010E006E070EE15C02E2E16AE552E16EA5
:10B720000050B2EF62F0ADEC62F0E652020EDF6E56
:10B73000200EDF5C11E2D0EC63F00EE01FEC63F052
:10B7400006E1E3EC62F003E1C4EC62F002D0C9EC84
:10B7500063F00DEC63F0ECD7FFEC63F0DF0EFC6FF1
:10B76000320EFD6F010E8FEC64F0A0EC92F06CECE9
:10B7700064F002E060EC63F0000EE552B2EF62F0BC
:10B7800097EC64F0DF6A010EE66E1CEC9FF0E55268
:10B79000B4EC64F0200EDF5C11E2D0EC63F00EE05C
:10B7A0001FEC63F006E1E3EC62F003E1C4EC62F04D
:10B7B00002D0C9EC63F00DEC63F0ECD76CEC64F0F4
:10B7C00004E0E66AB7EC3FF0E552000E006E030EAF
:10B7D000E15C02E2E16AE552E16E0050B2EF62F034
:10B7E000FCEC63F0F3A502D0000E34D097EC62F0CD
:10B7F000A70EE66EDE0EE66E000ED2EC62F0080ECC
:10B80000A9EC62F0990EE66EDE0EE66E000EA5EC77
:10B8100062F00E0EA9EC62F0890EE66EDE0EE66EA8
:10B82000000EA5EC62F0020EA9EC62F07F0EE66E4F
:10B83000DE0EE66E000EA5EC62F0030EA9EC62F0DF
:10B840006D0EE66EDE0EE66E000EA5EC62F0B6EC56
:10B8500062F0010E4EEC63F002E2E16AE552E16E45
:10B860000050B2EF62F09BEC64F0080E9DEC62F0C9
:10B8700011E0C9EC63F0020E9DEC62F00BE0C9EC44
:10B8800063F0030E9DEC62F005E0C9EC63F00E0E70
:10B89000F2EC63F0C0EC62F0A3DF006E060EE15E36
:10B8A0000050DF6EA0EC92F06CEC64F002E060EC13
:10B8B00063F0DF50E552B2EF62F0FCEC63F0F3A509
:10B8C00002D0000E56D097EC62F0670EE66EDE0EE8
:10B8D000E66E000ED2EC62F0050EA9EC62F05F0E8F
:10B8E000E66EDE0EE66E000EA5EC62F0060EA9EC2A
:10B8F00062F0560EE66EDE0EE66E000EA5EC62F00D
:10B90000070E42EC64F0EC0EE66E090EE66E410E98
:10B91000E66EDE0EE66E000EE5EC64F09AEC74F076
:10B92000DDEC62F00A015D5106E01E0EE66EDE0EF1
:10B93000E66E000E19D0200E0601C85D06E1FB0E72
:10B94000E66EDD0EE66E000E0FD0C851E66EE66ABA
:10B95000DC0EE66EDD0EE66E000EC6EC64F0DA0E6E
:10B96000E66EDD0EE66E000EA1EC62F0B6EC62F063
:10B97000010E4EEC63F002E2E16AE552E16E005026
:10B98000B2EF62F09BEC64F0050E9DEC62F01DE0FE
:10B990001FEC63F006E1E3EC62F003E1C4EC62F05B
:10B9A00002D0C9EC63F0060E9DEC62F00EE01FECD5
:10B9B00063F006E1E3EC62F003E1C4EC62F002D074
:10B9C000C9EC63F0070EF2EC63F0C0EC62F075DFD7
:10B9D00052EC63F002E060EC63F0DF50E552B2EF4E
:10B9E00062F0FCEC63F0F3A502D0000E2AD0FFEC6D
:10B9F00063F0D00EFC6FDD0EFD6F000E0AEC63F0FD
:10BA00000D0EE66E1AEC63F0E0EC62F007E109015E
:10BA1000C70EFC6FDD0EFD6F000E06D0DBEC63F091
:10BA200052EC64F0B8EC63F00AEC63F0EC0EE66EF6
:10BA3000090EE66EBD0EE66EDD0EE66E000EE0EC63
:10BA400063F04EEC63F002E2E16AE552E16E005011
:10BA5000B2EF62F002EC64F0D0EC63F009E1010EA9
:10BA6000DB6AD950010FE66E000EDA20E66E02D0D6
:10BA7000C9EC63F00D0EF2EC63F0C0EC62F0B1DFE4
:10BA800052EC63F002E060EC63F0DF504EEC63F0E8
:10BA900002E2E16AE552E16E0050B2EF62F0FCECC6
:10BAA00063F0F3A502D0000E23D097EC62F0B50E40
:10BAB000E66EDD0EE66E000ED2EC62F0040EA9EC2E
:10BAC00062F0AE0EE66EDD0EE66E000EA5EC62F0E4
:10BAD000090E42EC64F00A0EA9EC62F0A10EE66ECB
:10BAE000DD0EE66E000EA5EC62F0B6EC62F0010E23
:10BAF0004EEC63F002E2E16AE552E16E0050B2EF13
:10BB000062F09BEC64F0040E9DEC62F00BE0C9EC7B
:10BB100063F0090E9DEC62F005E0C9EC63F00A0EDB
:10BB2000F2EC63F0C0EC62F0BADF52EC63F002E0DA
:10BB300060EC63F0DF50E552B2EF62F0FCEC63F0D2
:10BB4000F3A502D0000E9ED097EC62F09B0EE66E3D
:10BB5000DD0EE66E000ED2EC62F00901F751E66EE2
:10BB6000E66A900EE66EDD0EE66E000EAAEC64F05C
:10BB70000901F851E66EE66A850EE66EDD0EE66EA8
:10BB8000000EAAEC64F00601C851E66EE66A760E75
:10BB9000E66EDD0EE66E000EC6EC64F00901EA51B9
:10BBA000000812E2ECEC62F06A0EE66EDD0EE66E64
:10BBB000000EF7EC62F039EC63F0640EE66EDD0E19
:10BBC000E66E000EF7EC62F00501F551E66EE66AEE
:10BBD000590EE66EDD0EE66E000EAAEC64F005016D
:10BBE000F6514DE04F0EE66EDD0EE66E000EA1EC56
:10BBF00062F00501F6A107D04A0EE66EDD0EE66E94
:10BC0000000EA1EC62F00501F6A307D0450EE66E2A
:10BC1000DD0EE66E000EA1EC62F00501F6A507D080
:10BC2000410EE66EDD0EE66E000EA1EC62F005013F
:10BC3000F6A707D03D0EE66EDD0EE66E000EA1EC17
:10BC400062F00501F6A907D0390EE66EDD0EE66E4C
:10BC5000000EA1EC62F00501F6AB07D0310EE66EE6
:10BC6000DD0EE66E000EA1EC62F00501F6AD07D028
:10BC7000290EE66EDD0EE66E000EA1EC62F0B6EC6B
:10BC800062F0010E4EEC63F002E2E16AE552E16E11
:10BC90000050B2EF62F097EC64F00501F3A502D01A
:10BCA000000E2CD0FFEC63F01F0EFC6FDD0EFD6F5D
:10BCB000000E0AEC63F0DF6A100EDF5C1EE2A3ECFC
:10BCC00063F0EF5018E0DFCFE6FFE66A1B0EE66E8A
:10BCD000DD0EE66E000E35EC63F0A3EC63F0EF5082
:10BCE000E66EE66AAF0EE66EDE0EE66E000EB9ECAC
:10BCF00062F0B6EC62F0DF2ADFD7010E006E030EB1
:10BD0000E15C02E2E16AE552E16E0050B2EF62F0FE
:10BD1000ADEC62F0E652D0EC63F002E1000E31D0FF
:10BD200074EC63F0DF6EC3EC64F0000EDF5C28E3BC
:10BD3000100EDF5C25E2D0EC63F022E074EC63F0DF
:10BD4000E66EA3EC63F0E552E750EF6E080EDF5CA1
:10BD500007E3C9EC63F0080EDF5C180FF2EC63F048
:10BD60000F0EDF5C02E1A0EC92F0FFEC63F0F90E45
:10BD7000FC6F320EFD6F010E0AEC63F0010E01D074
:10BD8000000EE552EFD306EC64F017E0F90EDBCFBE
:10BD9000E6FFFA0EDBCFE6FF180EE66EE66AE66A0D
:10BDA00007D04BCBFBFF4ACBFAFF0B014951F96E91
:10BDB000F8DF006E050EE15E0050FFEC63F00F0E41
:10BDC000FC6F330EFD6F010E09EF64F006EC64F0BA
:10BDD00017E0F90EDBCFE6FFFA0EDBCFE6FF140E1D
:10BDE000E66EE66AE66A07D04BCBFBFF4ACBFAFF6A
:10BDF0000B014951F96EF8DF006E050EE15E00504F
:10BE0000FFEC63F0220EFC6F330EFD6F010E09EFA5
:10BE100064F006EC64F017E0F90EDBCFE6FFFA0EF3
:10BE2000DBCFE6FF160EE66EE66AE66A07D04BCB7E
:10BE3000FBFF4ACBFAFF0B014951F96EF8DF006EA8
:10BE4000050EE15E0050FFEC63F0390EFC6F330E1F
:10BE5000FD6F010E09EF64F006EC64F017E0F90ED7
:10BE6000DBCFE6FFFA0EDBCFE6FF150EE66EE66AE5
:10BE7000E66A07D04BCBFBFF4ACBFAFF0B014951D7
:10BE8000F96EF8DF006E050EE15E0050FFEC63F026
:10BE9000520EFC6F330EFD6F010E09EF64F006ECDD
:10BEA00064F017E0F90EDBCFE6FFFA0EDBCFE6FF1A
:10BEB000170EE66EE66AE66A07D04BCBFBFF4ACB6D
:10BEC000FAFF0B014951F96EF8DF006E050EE15ED5
:10BED0000050FFEC63F0670EFC6F330EFD6F010E38
:10BEE00009EF64F03ADBE150F90FA3EC64F001E1F3
:10BEF0008BD0C9EC63F02AEC99F0E552E552C9DB2E
:10BF000001E190D0030EE66EE66A170EE66EDD0ED6
:10BF1000E66E000E4BDB12E1150EE66EDD0EE66EF0
:10BF20000A0EE66EE66AE66A07D04BCBFBFF4ACB09
:10BF3000FAFF0B014951F96EF8DF53D0030EE66E9C
:10BF4000E66A110EE66EDD0EE66E000E2FDB12E1E4
:10BF50000F0EE66EDD0EE66E0A0EE66EE66AE66A25
:10BF600007D04BCBFBFF4ACBFAFF0B014951F96ECF
:10BF7000F8DF37D0030EE66EE66A0B0EE66EDD0ED6
:10BF8000E66E000E13DB12E1090EE66EDD0EE66EC4
:10BF90000A0EE66EE66AE66A07D04BCBFBFF4ACB99
:10BFA000FAFF0B014951F96EF8DF1BD0030EE66E64
:10BFB000E66A050EE66EDD0EE66E000EF7DA24E1A7
:10BFC000030EE66EDD0EE66E0A0EE66EE66AE66AC1
:10BFD00007D04BCBFBFF4ACBFAFF0B014951F96E5F
:10BFE000F8DF006E050EE15E0050C3EC64F0D8DBB4
:10BFF00019E0F90EDBCFE6FFFA0EDBCFE6FF0F0EFE
:10C00000E66EE66AE66A09D0000E14D04BCBFBFF61
:10C010004ACBFAFF0B014951F96EF8DF006E050EAD
:10C02000E15E0050ECDB830EFC6F330EFD6F010E02
:10C03000F1DA010E97D2EADB14E0000EE66EE66A52
:10C040000B0EE66EE66AE66A07D04BCBFBFF4ACBE7
:10C05000FAFF0B014951F96EF8DF006E050EE15E43
:10C0600000500601F36BCBDBA00EFC6F330EFD6FAF
:10C07000010ECFD3CBDB14E0000EE66EE66A0C0EA9
:10C08000E66EE66AE66A07D04BCBFBFF4ACBFAFFC7
:10C090000B014951F96EF8DF006E050EE15E0050AC
:10C0A00006011E0EF36FABDBB70EFC6F330EFD6F98
:10C0B000010EAFD397EC64F0010EDF6E020EDF6E5F
:10C0C0000E0EF66E000EF76E000E44DBEB0EE66E03
:10C0D000DC0EE66E000EC9DA0F0EF66E000EF76E7D
:10C0E000000ED8DB100EF66E000EF76E000ED2DBDF
:10C0F0000E0E2FDAE70EE66EDC0EE66E000EE66E32
:10C10000A7DB7AEC64F0B4EC64F00701CC51CD11FC
:10C11000CE110AE0CCC7E6FFCDC7E6FFCEC7E6FFEB
:10C1200097DB9DDBB4EC64F0DFCFE6FFE66AE40E5C
:10C13000E66EDC0EE66E000E1CDAF9D917DA010E97
:10C14000006E030EE15C02E2E16AE552E16E00502E
:10C1500009D258DB030EE66EB7EC3FF0E552000E55
:10C160009DDA02E2E16AE552E16E0050FBD1F5D9B9
:10C17000FE0EDB50330A0AE0010A05E0030A19E16A
:10C1800051DA08E009D0B7DA14E104D0B4DA11E1E9
:10C1900049DA02E1000E0ED04BDB22EC5AF0E552F8
:10C1A000E552F4CF01F0D4EC64F0F3CFEEFF01C020
:10C1B000EDFF010ED7D1D1D9070EE126FB0EE4DA4F
:10C1C000FFD917E08DDB15E0FBD960080DE255DBE8
:10C1D000EFCF00F07B0E005C07E2F2D9E00FE66ED5
:10C1E0004CDBE552E750EF6EDF2A010EE9E3DB2A74
:10C1F000E7D776DB04E1DF2A010E01E3DB2A020E3A
:10C20000DB6A030EDB6A55DAABDA04BE0568040E9E
:10C2100079DAFEE1EFD901E119D13B0E066E340E59
:10C22000076E010E086E020EDBCF09F0030EDBCFA6
:10C230000AF00B6A0ABE0B68040ED89009360A365B
:10C240000B36E806FAE106500924036E07500A206F
:10C25000046E08500B20056E03C0E6FF04C0E6FF25
:10C26000E66E4AEC98F097DB27C000F028C001F09A
:10C2700029C002F00006000E015A025A53DB3B0EA1
:10C280000F6E340E106E010E116E020EDBCF12F027
:10C29000030EDBCF13F0146A13BE1468040ED8909B
:10C2A000123613361436E806FAE10F5012240C6EDB
:10C2B000105013200D6E115014200E6E0C2A000E1B
:10C2C0000D220E220CC0E6FF0DC0E6FF0EC0E6FFF9
:10C2D000CDDA2AEC97F0156E070EE15E15500009D5
:10C2E00001E0ADD0040EDB6A66DADBEC59F0E55212
:10C2F000E55207DBD950050FE66E000EDA20E66E38
:10C3000053DAD7D92DDA04BE0568040EFBD9FEE155
:10C3100071D9E66E2CDF066E050EE15E065000094F
:10C3200001E1BED00B014C514D114E1124E0050E20
:10C33000DBCFE6FF060EDBCFE6FFFB0EDBCFE6FF33
:10C34000FC0EDBCFE6FFFD0EDBCFE6FFFE0EDBCF04
:10C35000E6FF010EE66E07D04ECBFBFF4DCBFAFF9A
:10C360000B014C51F96EF8DF006E070EE15E0050D4
:10C37000000901E095D0020EDBCFE9FF030EDBCF11
:10C38000EAFFEA02F3CFEAFFE902F3CFE9FFF45054
:10C39000EA26000EE9260A0EEA22EECF00F0EECFE2
:10C3A00001F0EFCF02F0050EDBCFE6FF060EDBCF8C
:10C3B000E6FFFB0EDBCFE6FFFC0EDBCFE6FFFD0E5C
:10C3C000DBCFE6FFFE0EDBCFE6FF06D002C0FBFFB1
:10C3D00001C0FAFF0050F96EF9DF036E060EE15E50
:10C3E0000350E76E040EE7CFDBFFDB5059E00B0193
:10C3F0004C514D114E1120E0050EDBCFE6FF060E2D
:10C40000DBCFE6FFFB0EDBCFE6FFFC0EDBCFE6FF6C
:10C41000FD0EDBCFE6FFFE0EDBCFE6FFE66A07D0C0
:10C420004ECBFBFF4DCBFAFF0B014C51F96EF8DF01
:10C43000006E070EE15E0050D1EC58F031D0020ED4
:10C44000DB2A030E01E2DFD6DB2ADDD60B014F51DA
:10C45000501151111FE0DECFE6FFDDCFE6FFFB0EEE
:10C46000DBCFE6FFFC0EDBCFE6FFFD0EDBCFE6FF0A
:10C47000FE0EDBCFE6FF07D051CBFBFF50CBFAFF20
:10C480000B014F51F96EF8DF006E060EE15E0050B1
:10C49000000906E1EBD988D9D8EC36F07CDAE55210
:10C4A000070EE15C02E2E16AE552E16E5BD0A4D9DD
:10C4B000F3A502D0000E34D0A2D9DA0EFC6FDC0E48
:10C4C000FD6F000EA7D8DE6ADD6AF8D904BE0568E4
:10C4D000040E18D9FEE18ED822E00901D80EFC6FB7
:10C4E000DC0EFD6F000E96D8E9D904BE0568040E77
:10C4F00009D9FEE1005003240901FC6F015004201A
:10C50000FD6F02500520FE6FFC2B000EFD23FE2365
:10C5100054EC3EF0DF2A010ED8E3DB2AD6D7010E19
:10C52000BDD802E2E16AE552E16E00501BD03CD971
:10C53000AAEC58F0E552E552120054D924DAD0EFB3
:10C5400063F043DA8CD9F7EF63F03FDAD3D9F7EF32
:10C5500063F0E66E1CEC9FF071D1D9CFE6FFE1CF1E
:10C56000D9FF1200E552E7CFD9FF1200E7D952EF09
:10C5700064F0E66E6DD9A0EC74F0F1D9B4EF64F01C
:10C5800008D974D9D4EF63F0010EE76EF90EDBCF52
:10C5900000F0FA0EDBCF01F0E7500026000E01227A
:10C5A00092EF64F015DA5BD9F7EF63F0E66EF1D83D
:10C5B0002AEC97F0D4D900091200D1D9F7EF63F033
:10C5C0005CD9EF501200010EE76EA2D9E750E926C0
:10C5D000000EEA22EF501200010EE66EE66AEAC98A
:10C5E00000F0016A026A036AEAC9E6FF6ED1EDD97A
:10C5F000B8EF64F000500324F36E01500420F46E91
:10C6000002500520F86EF4CFF7FFF3CFF6FF0800D5
:10C61000F5501200FE6F54EF3EF0DF50DF2AE2D8F3
:10C62000C3EF64F005D9C7D9BAEC59F0B4D9E552D3
:10C63000000912001CEC9FF0E552F7EF63F068D997
:10C64000EF502D081200E66E58EC72F0E552120021
:10C650000A017E0EFB6F320EFC6F010EFD6FA4D837
:10C66000DFEC58F0E552E5521200D6D878D9B4EF95
:10C6700064F0010EE66EE66AEBC900F0016A026A38
:10C68000036AEBC9E6FF21D196D83CEC98F0E5525D
:10C69000D5D00B0149514A114B111200006E020E08
:10C6A000E15C1200006E060EE15E0050DF6E6CEF82
:10C6B00064F03B0E006E340E016E010E026E12002D
:10C6C000400EE66EB7EC3FF0E5521200DBCFE6FF1E
:10C6D00072D86FEC98F0026E060EE15E025000090F
:10C6E0001200E652C9EF63F054D878EC89F0E552B5
:10C6F000E552F35012005FD99BEC59F0E552E55238
:10C7000000091200D890033604360536E8061200F8
:10C71000020EE12605011200020EE126D950FD0F9E
:10C72000A3EF64F0E0D800C0F3FF01C0F4FF1200F3
:10C73000F9EC75F0006E090EE15E0050F7EF63F062
:10C740000ED981EF64F0DF50EA6AE50FE96E050E5D
:10C75000EA221200F86E0800F550E66EE66A120052
:10C76000020EDBCF03F0030EDBCF04F0056A1200EC
:10C7700009015F0EFC6FDF0EFD6F000E120063EC0F
:10C780009FF009D905011200DBCFDEFFDBCFDDFF13
:10C790001200F90EDBCFE6FFFA0EDBCFE6FF120048
:10C7A000D950F90FA3EF64F0FD0EDBCFE6FFFE0ECC
:10C7B000DBCFE6FF1200DECFE6FFDDCFE6FF1200A3
:10C7C00007D99AEC74F0CBD8D1DE010E120022EC1E
:10C7D0005AF0E552E552F90EF3CFDBFFFA0EF4CF33
:10C7E000DBFF1200E66E63EC9FF0CBEF64F0F3CF5B
:10C7F000DEFFF4CFDDFF1200B0DE88EF63F097DEDE
:10C8000009011200AADE020EE1261200A6DE49EF9F
:10C8100063F000DF010EA6D6DBD8A0EF74F091DE46
:10C82000A5DED1EC58F0050E0EDF020EE15C120021
:10C83000BBD8EECFE6FFEFCFE6FF1200E552F3CF15
:10C8400000F0F4CF01F0F3CFE6FFF4CFE6FF1200E3
:10C85000010EDBCFE6FF020EDBCFE6FF120071EC2C
:10C8600074F0006E050EE15E00501200FB0EDBCF8F
:10C87000E6FFFC0EDBCFE6FF1200DECFE9FFDDCFE7
:10C88000EAFF120066DE490EE66EDE0EE66E000E70
:10C89000A5EF62F05FDFE90EE66EDC0EE66E000EDD
:10C8A000B9EF62F0A3EC3EF0E552E5521200B30E90
:10C8B000FC6FDE0EFD6F000E0AEF63F0FADEDECFD6
:10C8C00003F0DDCF04F0056A120001C0E6FF02C0EC
:10C8D000E6FF03C0E6FF12007F0E0601C85D1200EE
:10C8E0006FDE20081200FD0EDBCF00F0FE0EDBCF66
:10C8F00001F012009AEC74F0026E070EE15E025035
:10C900001200050EF3CFDBFF060EF4CFDBFF1200A3
:10C91000F90EDBCFE9FFFA0EDBCFEAFF12007ADE79
:10C92000D1EF58F000C0E6FF01C0E6FF120015DEAF
:10C93000030EE126120011DE71EF63F0000EE66EC9
:10C94000060EE66E1200E96EFF0EDA20EA6EEE5079
:10C95000ED1012003AD8A0EC74F0DDEF62F0006E3A
:10C96000070EE15E00501200DE5241DFDD52120080
:10C9700092EC75F0046E0B0EE15E0450F7EF63F07D
:10C9800062DE97EF62F005DFE7EF63F01ED800ECA0
:10C9900075F0DDEF62F0E552E552E552120032DF4C
:10C9A000010EE66E1AEF63F0FA0EDBCFE9FFFB0E25
:10C9B000DBCFEAFF1200FC0EDBCFE6FFFD0EDBCF84
:10C9C000E6FF120040DEFFEF63F0E66EDBEF63F0A0
:06C9D000E66E9EEF64F02C
:0AC9D60098EC6BF0020EE126E00E73
:10C9E0006214DF6E0F0E65140B01406F66CF41FBC2
:10C9F00067CF42FB68CF43FB69CF44FB6ACF45FB5F
:10CA00006BCF46FB6CCF47FB6DCF48FB609EDF5082
:10CA100001E067D20B014151A60A01E15BD2030A92
:10CA200001E12FD2010A01E122D2070A01E115D268
:10CA30003D0A01E1F7D1080A01E178D1030A01E1D9
:10CA400036D11C0A01E1FAD0010A01E1E8D00D0A51
:10CA500001E1B4D0010A01E191D0070A6FE0010AB7
:10CA600067E0030A45E0010A18E0860A01E046D2C1
:10CA70001B0E425D03E145CBDDF90BD01A0E425D82
:10CA800001E03CD24551000EF35046250901DE6F0E
:10CA9000DF6B0901010EE56F31D242CBA0F944CB27
:10CAA00001F0006A435109010024A16F000E01202A
:10CAB000A26F48CB01F0006A0B0147510901002425
:10CAC000A36F000E0120A46F0901700ED880A1553C
:10CAD000170EA25502E2A16BA26B0901700ED8805D
:10CAE000A355170EA45501E309D2A36BA46B06D27C
:10CAF00077EC6BF003E0A3EC6BF0FDE13FEC6BF047
:10CB000003E0AAEC6BF0FDE148EC6BF003E0C8EC4D
:10CB10006BF0FDE100500C240901A56F01500D20C0
:10CB2000A66F02500E20A76F03500F20A86FE6D10A
:10CB300042CBADF90901780EE16FE0D177EC6BF0F3
:10CB400003E0A3EC6BF0FDE13FEC6BF003E0AAEC3B
:10CB50006BF0FDE148EC6BF003E0C8EC6BF0FDE13D
:10CB600000500C240901D16F01500D20D26F0250EA
:10CB70000E20D36F03500F20D46FC0D177EC6BF031
:10CB800003E0A3EC6BF0FDE13FEC6BF003E0AAECFB
:10CB90006BF0FDE148EC6BF003E0C8EC6BF0FDE1FD
:10CBA00000500C240901D56F01500D20D66F0250A2
:10CBB0000E20D76F03500F20D86FA0D142CBE0F9E1
:10CBC0000901E05129E044CB01F0006A0B01435117
:10CBD00009010024D96F000E0120DA6F680ED919FF
:10CBE00005E1010EDA1902E1D96BDA6BF00E0B01E7
:10CBF000461504E00901DB6BDC6B0AD046CB01F083
:10CC0000006A455109010024DB6F000E0120DC6F32
:10CC10000901780EE36F72D10901E36B6FD142CB4A
:10CC200090F947CB91F944CB01F0006A43510901D7
:10CC30000024926F000E0120936F60D14D0E07010A
:10CC4000CB5D03E142CB9FF926D042CB26F0276A89
:10CC5000286A296A490E2B6E060E2C6E2D6A2E6AE2
:10CC600089ECA7F022C026F023C027F024C028F0CA
:10CC700025C029F0F40E2626010E2722000E2822B8
:10CC80002922E80E2B6E030E2C6E2D6A2E6AF1EC13
:10CC9000A7F026C09FF944CB01F0006A0B01435175
:10CCA000090100248E6F000E01208F6F27D109012A
:10CCB00094510B01425D0EE009019451020803E218
:10CCC0000F0E945D07E1040E0B01425D03E0040EBC
:10CCD00058EC6BF0090194510B01425D05E109012B
:10CCE00095510B01435D0CE0020E58EC6BF00B010B
:10CCF000420506E1D7EC6BF003E20901010E096F72
:10CD000042CB94F943CB95F90501F3A104D00F0E62
:10CD10000B01451504D00B0146390F0B0F0B090110
:10CD2000966F44CB97F948CB98F9E8D00F0E0901DC
:10CD3000945D02E10B0142890B0142510901995DA9
:10CD40000FE10B01435109019A5D0AE10B014451C6
:10CD500009019B5D05E10B01455109019C5D03E063
:10CD6000010E58EC6BF0800E09019A150AE1800E55
:10CD70000B01431506E0100E431503E0100E58ECAE
:10CD80006BF0020E09019C1507E1020E0B0145151F
:10CD900003E0200E58EC6BF042CB99F943CB9AF9A3
:10CDA00044CB9BF945CB9CF9EDEC6BF021E10901FB
:10CDB000A951AA11AB11AC111BE10901A551A61192
:10CDC000A711A81115E0D7EC6BF003E20901010EE1
:10CDD000096FA5C9A9F9A6C9AAF9A7C9ABF9A8C934
:10CDE000ACF90901A907000EAA5BAB5BAC5B16D0DE
:10CDF000EDEC6BF001E182D00901A951AA11AB1150
:10CE0000AC1101E17BD0D7EC6BF003E20901010E1C
:10CE1000096F0901A96BAA6BAB6BAC6B010E58ECE7
:10CE20006BF06CD04351640D11EC6CF0800E002659
:10CE3000000E0122080E0F0B05E0D89001320032DF
:10CE4000E806FBE10B014451640DF3500024090195
:10CE5000F56FF4500120F66F51D042CBC0F943CBAF
:10CE6000C1F947CBC2F90901780EE26F47D0010E34
:10CE7000DB6ACFEC6BF042E2B1EC6BF0BDEC6BF037
:10CE8000F8D7010EDB6ACFEC6BF006E2B1EC6BF089
:10CE9000070FBDEC6BF0F7D7410E0B01445D03E0CB
:10CEA000420E445D03E10501320E02D00501310E50
:10CEB000CA6F380E0B01445D02E10501F381330EA8
:10CEC0000B01425D03E10501530E02D005014E0E38
:10CED000CB6F14D042CBBCF943CBBDF944CBBEF9E8
:10CEE0000DD00B0141510E0A09E1425109019E5D2D
:10CEF00003E0010E58EC6BF042CB9EF9010E006E80
:10CF0000020EE15C02E2E16AE552E16E005091EF4F
:10CF10006BF098EC6BF0E6520F0E0F0155150B01FC
:10CF2000406F56CF41FB57CF42FB58CF43FB59CF01
:10CF300044FB5ACF45FB5BCF46FB5CCF47FB5DCF45
:10CF400048FB50CFDFFF0F01509F070EDF1404088E
:10CF500032E1020E0B01415D01E089D00501E5518E
:10CF6000000801E384D0EDEC6BF001E180D00B010F
:10CF7000435109019F5D01E17AD0D7EC6BF001E3E9
:10CF800076D041CB00F942CB01F99FC902F9F00EEE
:10CF90000B0144150901036F45CB04F946CB05F994
:10CFA00047CB06F948CB07F90F0140B7FDD787DB20
:10CFB000E5C508F95CD0070EDF14020821E10B017A
:10CFC0004451000804E243CBC7F944CBC3F94851AC
:10CFD000000804E247CBC8F948CBC4F94251000825
:10CFE00004E241CBC9F942CBC5F94651000804E23D
:10CFF00045CBCAF946CBC6F90901780EE46F37D0A4
:10D000000B014151FA0A33E144CB00F0016A026A94
:10D01000036A45CB04F0056A066A076A080E1F0B0F
:10D0200002E091DBFEE1F1EC6BF046CB08F0096A1F
:10D030000A6A0B6A100E1F0B02E08CDBFEE1005047
:10D0400008240901CD6F01500920CE6F02500A203B
:10D05000CF6F03500B20D06F48CB01F0006A0B015B
:10D06000475109010024CB6F000E0120CC6F010E47
:10D07000E55257D30901085102E1E5C508F9000C52
:10D080000901095114E0096B0F0140B7FDD7F1DA2E
:10D09000060E466FD00E476F070E486F496B4A6BFE
:10D0A0004B6B4C6B400E4D6F080E456F406F090186
:10D0B000085101E1000C020E005D11E10501E5518E
:10D0C00000080DE28ADB0BE072DB09E2010EE66E7E
:10D0D0007CECA8F0E5520F0140B7FDD7F0DA09016A
:10D0E0000807000C0F0140B7FDD7C3DA0A0E466FE0
:10D0F000010E456F080E406F40B7FED712000F01BA
:10D1000040B7FDD7B6DA060E466F2C0E476F010EFC
:10D11000486F496B4A6B090E4B6F100E4C6F86DBE4
:10D1200040B7FED7120004DB0F0140B7FDD775DB17
:10D13000190E95DA40B7FED7D5DFF3D2F9DA0F0131
:10D1400040B7FDD76ADB020E8ADA40B7FED7CADFE6
:10D15000E8D2EEDA0F0140B7FDD75FDB030E7FDACE
:10D1600040B7FED7BFDFDDD2E3DA040EE12647DBAE
:10D17000EDEC89F0E552E55226C0DEFF27C0DEFF68
:10D1800028C0DEFF29C0DDFFDD52DD52FE0EDB5080
:10D19000020802E122DB4EE10F0140B7FDD769DA58
:10D1A0000B0E466FFE0EDBCF47FF486B496BACDAC8
:10D1B00000504A6FA9DA080EFEDAFEE100500F01B6
:10D1C0004B6FA2DA100EF7DAFEE100500F014C6F40
:10D1D00016DB3CEC98F0F6DA040ED89000360136F7
:10D1E000E804FBE1026A036A180E086ED9CFE9FF72
:10D1F000DACFEAFFE8501F0BEECF04F0EECF05F0D8
:10D20000EECF06F0EECF07F007E0D89007320632F7
:10D2100005320432E806F9E10F0E0416056A066AC3
:10D22000076ADFDA00C04DFF0F01080E456F406F3F
:10D2300040B7FED7040EE15C02E2E16AE552E16E1E
:10D2400070D276DA0F0140B7FDD7E7DA1B0E07DAA6
:10D2500040B7FED7FE0EDB041AE1DFDA1A0E476F85
:10D26000486B496BFD0EDBCF01F001C000F00150AF
:10D270004A6FFF0EE76EFC0EDBCF00F0E7500016A2
:10D28000016A00C04BFF4C6BD1DA40B7FED72ADFF2
:10D2900048D24EDA0F0140B7FDD7EBD9090E466FE1
:10D2A000476BFE0EDBCF48FF030E456F080E406F45
:10D2B00040B7FED717DF35D23BDA030EE126020E68
:10D2C000DB6AFC0EDBCF28F0FD0EDBCF29F0180E59
:10D2D000281801E1295001E110D1170E281801E1A9
:10D2E000295001E1EED0160E281801E1295001E184
:10D2F000E2D0150E281801E1295001E1D6D0140E14
:10D30000281801E1295001E1CAD0130E281801E1C3
:10D31000295001E1BFD0120E281801E1295001E186
:10D32000B4D0110E281801E1295001E180D0100E6F
:10D33000281801E1295058E00F0E281801E1295062
:10D340004DE00C0E281801E1295034E00B0E28188E
:10D3500001E1295016E00A0E281801E1295002E0E7
:10D36000000EECD00501F45101E1CAD0FA0EDBCF7A
:10D37000E6FFFB0EDBCFE6FF49DAD5DEE552B2DE93
:10D38000C8D00501F45101E1BBD0040E0901991583
:10D390000BE0070E0901955D07E0010EE66ED9DE90
:10D3A000E5520601F36BB5D0890EE66E4D0EE66EC2
:10D3B000010EB4D00501F45101E1A2D0090199A9EF
:10D3C00007D0E66AC6DEE55206011E0EF36FA1D055
:10D3D000AF0EE66E4D0EE66E010EA0D00501F451C3
:10D3E00001E18ED007DA20D00501F45101E188D0A7
:10D3F000A0CADEFFA1CADDFFA0D908E09ED92C0893
:10D4000005E0DF2A010EF8E3DB2AF6D796D92C08CF
:10D4100036E1DCD901E3DB2AEF6A87D984DEE55205
:10D42000DECFE6FFDDCFE6FFF1D988DE71D0050162
:10D43000F45166E0A0CADEFFA1CADDFF7ED908E094
:10D440007CD92C0805E0DF2A010EF8E3DB2AF6D7A9
:10D4500074D92C0814E1BAD901E3DB2AEF6ADECFD4
:10D46000E6FFDDCFE6FF78EC89F0ACD9F3CFE6FF3D
:10D47000F4CFE6FF5AD9E5DEE552E55249D0430E36
:10D48000E66E4D0EE66E010E49D00501F45138E00E
:10D4900029DE03D00501F45133E031DE3AD0050135
:10D4A000F45112E0A7D9020E17D00501F4510CE097
:10D4B000A1D9E66A12D00501F45106E09BD9030E0A
:10D4C0000BD00501F45106E1550EE66E4D0EE66EE9
:10D4D000010E0CD08FD9010EE66E46DEE552E55204
:10D4E000E552400EE66E4D0EE66E010E9AD8010E24
:10D4F000F36E020EF3CFDBFF12D00501F45106E10B
:10D50000550EE66E4D0EE66E010E08D00ED9C1DE48
:10D51000E552400EE66E4D0EE66E010E82D8FE0E0E
:10D52000DB500BE03AEC2EF0020EE66E58EC72F097
:10D53000E552E66A76EC31F0E552010E006E030E1C
:10D54000E15C02E2E16AE552E16E0050EAD0D9CF37
:10D55000E6FF020EE1260501540EC86F520EC96F98
:10D56000CA6BCB6BCC6B900E6F6E6EAEFED7606AE3
:10D570000F01A00E196F1869016B200E006F506B20
:10D58000E00E1D6F1C69800E096F680E086F400E5B
:10D590000D6F800E0C6F116B106F706AD20E716E72
:10D5A000020E726E200E736E02D902E26F6A02D012
:10D5B000600E6F6E0901006B086B096B0601EE854A
:10D5C0000701A60ECF6F510ED06F010ED16F07016C
:10D5D000D60ED56FC90ED66F000ED76F0701120E8B
:10D5E000D86FCF0ED96F000EDA6F0701740EED6F92
:10D5F000D00EEE6F000EEF6F0701800EF06FD00EB1
:10D60000F16F000EF26F0B01B80E496FD20E4A6F28
:10D61000000E4B6F020EE15C02E2E16AE552E16E40
:10D6200080D0E66EECD8390EE66E4D0EE66E010E39
:10D63000E66E000EE66E060EE66EA0EC74F0026E6C
:10D64000070EE15E0250EDD8F3CFE6FFF4CFE6FF20
:10D6500071EC74F0036E050EE15E03501200476F2B
:10D66000486B496BFE0EDBCF4AFF4B6B4C6B16EFE2
:10D670006CF0406B400E426F200E416F1200B1D82B
:10D6800047CB08F0096A0A6A0B6A100E1F0B1200DA
:10D6900008500026095001220A5002220B50032292
:10D6A00048CB0CF00D6A0E6A0F6A180E1F0B1200A1
:10D6B000E66EE66AFEEC3EF0E552E5521200406B83
:10D6C000426B800E416F00C946FF01C947FF02C986
:10D6D00048FF03C949FF04C94AFF05C94BFF06C9F2
:10D6E0004CFF07C94DFF080E456F406F120045CB38
:10D6F00000F0016A026A036A46CB04F0056A066A12
:10D70000076A080E1F0B1200D9CFE9FFDACFEAFF34
:10D71000EECF00F0EECF01F0EECF02F0EFCF03F04E
:10D720001200E552E7CFD9FF120064D806EF6CF083
:10D73000D9CFE6FFE1CFD9FF1200DECFE9FFDDCF81
:10D74000EAFFEF501200D890043605360636073649
:10D75000E8061200D890083609360A360B36E80675
:10D760001200010EDB28EA6A410FE96E0B0EEA2275
:10D77000EF50E66E010EDB501200EA6AAE0FE96E62
:10D78000090EEA22E552E750EF6E010EDB2A120085
:10D79000D8900C360D360E360F36E8061200070EFE
:10D7A000F36E010EDBCFF4FFF350F45C12000501C1
:10D7B000F45100081200D8900332023201320032D4
:10D7C000E8061200E552E55211EF6CF0DFCFE9FFF9
:10D7D000DF2A010EDBCFEAFF1200800E0901991546
:10D7E0001200045000260550012206500222075064
:10D7F00003221200A0CAE6FFA1CAE6FF1200FC0E37
:10D80000DBCFE6FFFD0EDBCFE6FF120078EC89F000
:10D81000E552E552F350E66E12002BDF050E466F1F
:10D820001200F3CF00F0F4CF01F012004D6B080EA0
:06D83000456F406F12007D
:0AD8360053544154002B4355534452
:10D840003A002B4346554E3A005244590053454E38
:10D8500044204641494C00434F4E4E4543542046D8
:10D8600041494C00434C4F534544004441544120EE
:10D870004143434550540053454E44204F4B002BE9
:10D880004353513A0053544154453A205443502095
:10D89000434C4F5345440053544154453A2054435C
:10D8A0005020434F4E4E454354494E470053544138
:10D8B00054453A20434F4E4E454354204F4B00535E
:10D8C000544154453A2000434F4E4E454354204F57
:10D8D0004B0036342C002C00322C002B434C49508A
:10D8E000002B5044503A204445414354002B4352AE
:10D8F00045473A203000222C2236383637220D0098
:10D9000041542B43495053544152543D22544350A7
:10D91000222C220041542B43494653520D004154BE
:10D920002B434950484541443D310D0041542B4360
:10D93000494943520D00222C220041542B43535499
:10D94000543D2200220D0041542B434744434F4E87
:10D95000543D312C224950222C22002B4352454762
:10D96000002B434F50533A002B434D452045525214
:10D970004F5200534554555000223B2B434F5053B8
:10D980003F0D0041542B434F50533D312C312C223D
:10D990000041542B434C504F52543D22544350228B
:10D9A0002C2236383637220D0041542B4349504340
:10D9B0004C4F53450D0041542B4349505348555447
:10D9C0000D00002D002200495000534D53005629F0
:10D9D00000562C207265663D004D502D3020504180
:10D9E0003132562042415454455259204F4B202841
:10D9F000004D502D30205041414C455254212121A1
:10DA00002031325620424154544552592043524904
:10DA1000544943414C2028002520534F4329004DB1
:10DA2000502D30205041414C45525421212120435A
:10DA30005249544943414C20534F43204C4556458D
:10DA40004C20415050524F41434845442028004DFE
:10DA5000502D302050415472756E6B2068617320D8
:10DA60006265656E206F70656E6564202876616CF6
:10DA70006574206D6F6465292E004D502D30205047
:10DA80004156656869636C6520616C61726D2069DF
:10DA90007320736F756E64696E6721000D204341BA
:10DAA000433A20000D204F444F3A200025000D201E
:10DAB000534F433A2000206B6D00206D6900202DEC
:10DAC00020000D2052616E67653A20004E6F742071
:10DAD0006368617267696E67004368617267696E47
:10DAE000672053746F707065640043686172676982
:10DAF0006E672C2048656174696E670050726570AE
:10DB00006172696E67004368617267696E6720447D
:10DB10006F6E65004368617267696E672C20546F91
:10DB20007070696E67206F6666004368617267692E
:10DB30006E6700506572666F726D616E6365202D51
:10DB4000200052616E6765202D200053746F726152
:10DB50006765202D20005374616E64617264202D0E
:10DB600020002C312C496E76616C6964205553532A
:10DB70004420726573756C74002C302C00202D20AD
:10DB80004D53473A2000534D532046524F4D3A20B3
:10DB9000004D502D30205041000D00222C31350D0C
:10DBA0000041542B435553443D312C22004D502D00
:10DBB000302063332C302C004D502D302063312C1D
:10DBC000302C004D502D302061004D502D30200064
:10DBD0004D502D53203020004D502D3020482A2DFF
:10DBE0004F564D2D446562756743726173682C30E2
:10DBF0002C323539323030302C004D502D3020450C
:10DC000054004D502D3020670043312D362C4334C5
:10DC1000302D34312C433439004D502D30205600F6
:10DC20004D502D302044002F56002F002E004D5017
:10DC30002D30204600302C302C004D502D302057F8
:10DC4000004D502D30204C002C706572666F726D47
:10DC5000616E6365002C72616E6765002C73746F72
:10DC600072616765002C7374616E64617264002C6C
:10DC700073746F70706564002C68656174696E6799
:10DC8000002C70726570617265002C646F6E6500A7
:10DC90002C746F706F6666002C6368617267696EC2
:10DCA00067002C004D502D3020530020004D502D8A
:10DCB00043203020004D502D3020454D001A000DDE
:10DCC0000A0041542B43495053454E440D00232034
:10DCD000004D502D302063002000436F6D6D616E4C
:10DCE00064733A002F56002F002E004F564D5320DC
:10DCF0004669726D776172652076657273696F6EC1
:10DD00003A2000340050455200330052414E003159
:10DD10000053544F003000535441000D0A20004678
:10DD2000656174757265733A002053544B554E46C5
:10DD3000002053544B46554C002052490020544F6C
:10DD4000002050440020504F520020424F52000A01
:10DD5000202E2E6C6173743A000A2043726173683E
:10DD600065733A00207265663D000A203132562004
:10DD70004C696E653A000A204E4554205374617414
:10DD8000653A3078000A2047524E204C65643A00CC
:10DD90000A20524544204C65643A00444941473AC0
:10DDA000000D0A20506172616E6F69643A000D0ABD
:10DDB0002049503A005365727665723A0043757295
:10DDC00072656E743A2000286E6F6E65290D0A0028
:10DDD00047534D4C4F434B3A200029000D0A204732
:10DDE000534D2F475052533A204E6F7420636F6E3D
:10DDF0006E656374656420283078000D0A204753EF
:10DE00004D3A204F4B0D0A205365727665723A20C9
:10DE10004E6F7420636F6E6E6563746564000D0AE7
:10DE200020475052533A204F4B0D0A2053657276CB
:10DE300065723A20436F6E6E6563746564204F4B64
:10DE4000000D0A2047534D3A000D0A2050617373AC
:10DE5000776F72643A000D0A20557365723A000DAF
:10DE60000A2041504E3A00475052533A000D0A20C2
:10DE70004E6F74696669636174696F6E733A000D01
:10DE80000A20556E6974733A000D0A205665686958
:10DE9000636C65547970653A000D0A2056656869AF
:10DEA000636C6549443A004D6F64756C653A003A9D
:10DEB000000A00506172616D733A002C004D6F646E
:10DEC000756C652070617373776F72643A200052CD
:10DED000656769737465726564206E756D626572DD
:10DEE0003A2000562900562C207265663D004D50A0
:10DEF0002D30205041313256204241545445525920
:10DF0000204F4B2028004D502D30205041414C4592
:10DF1000525421212120313256204241545445523D
:10DF20005920435249544943414C2028002520534D
:10DF30004F432900414C455254212121204352494D
:10DF4000544943414C20534F43204C4556454C20A7
:10DF5000415050524F41434845442028001A000D7B
:10DF60000A00220D0A0041542B434D47533D220025
:10DF7000232000303132333435363738394142438B
:10DF800044454600232053746F70706564204341FC
:10DF90004E2073696D0D0A002320537461727469F9
:10DFA0006E672043414E2073696D0D0A0041542B6A
:10DFB0004353510D0041542B4350494E3F0D0041F6
:10DFC000542B434F50533F0D000A00232020536928
:10DFD0006D2054783A200020657374206D696C655B
:10DFE00073290D0A0020696465616C2C20002520CE
:10DFF0002800232020534F433A20202020202000B7
:10E00000290D0A0020280023202056494E3A2020BE
:10E0100020202020000D0A0A002320205369676E6B
:10E02000616C3A2020200020560D0A002320203168
:10E030003256204C696E653A200023202053574900
:10E040005443483A202020002F56002F002E002352
:10E05000204669726D776172653A20000D0A2320AF
:10E06000444941470D0A0A0023204C656176696ED8
:10E070006720446961676E6F7374696373204D6FC5
:10E0800064650D0A002320274D2720434F4D4D4145
:10E090004E44533A0D0A20200023202753272043C3
:10E0A0004F4D4D414E44533A0D0A2020002320434A
:10E0B0004F4D4D414E44533A2048454C50203F204F
:10E0C00044494147205245534554206F7220532004
:10E0D0002E2E2E0D0A000D0A004F564D5344494175
:10E0E00047000D0A23204E4F5449465920414C41C8
:10E0F000524D20414C4552540D0A000D0A23204E2A
:10E100004F54494659205452554E4B20414C45528C
:10E11000540D0A000D0A23204E4F544946592043FE
:10E12000484152474520414C4552540D0A001B5B63
:10E13000324A1B5B30313B3031480D23204F564D66
:10E140005320444941474E4F5354494353204D4F68
:10E1500044450D0A0A002000200D0A5477697A7997
:10E1600020436F6D6D616E64733A00562000432941
:10E170002000432E2E0043202800503A00426174B4
:10E1800074657279206D6F6E69746F722072657339
:10E1900065742E0052542D5057522D4261747443B1
:10E1A000656C6C2C0052542D5057522D4261747482
:10E1B0005061636B2C004D502D302048004D0043C2
:10E1C000200054656D70733A20003A003A2B0043EA
:10E1D000002E2E2E004F4B20006D56200053443A47
:10E1E000003F002100566F6C74733A20000A2046ED
:10E1F000756C6C206368617267653A20000A205470
:10E20000696D653A2000206F7220004F464600433A
:10E21000686172676520416C6572743A2000554EE2
:10E22000534554004D617820696465616C207261CA
:10E230006E67653A20000D204F444F3A2000252993
:10E2400000252E2E00252028000D20534F433A2074
:10E2500000206B6D00206D6900202D20000D2052E4
:10E26000616E67653A20000D2046756C6C2063680E
:10E27000617267653A20004E6F742063686172674F
:10E28000696E6700206D696E2E000D2046756C6CFE
:10E290003A20000D204348473A20004368617267E6
:10E2A000696E672053746F707065640043686172B3
:10E2B00067696E6720446F6E6500436861726769C5
:10E2C0006E672C20546F7070696E67206F666600F1
:10E2D0004368617267696E67002073733D00206C4C
:10E2E00074613D002074613D002074773D00206C16
:10E2F00076613D002076613D000A232076773D005F
:10E30000204449523D0020414C543D00204C4F4E8A
:10E310003D00204C41543D000A23204649583D0011
:10E320002053513D002064723D002064693D00206F
:10E330004F444F3D00205354533D002C302C00637C
:10E34000004D502D3020004D502D30205041002CDC
:10E3500030004D502D302063004D502D302048525C
:10E36000542D5057522D5573616765537461747302
:10E370002C302C3836343030000D20446F776E202E
:10E38000006D20000D20557020000D204465636550
:10E390006C20000D20416363656C20002520000D7A
:10E3A00020436F6E7374200025002057682F6B6D1B
:10E3B00020523D00456666696369656E6379200099
:10E3C0002057680D20446F776E20006D202D0020AF
:10E3D00057680D20557020002057680D2044656354
:10E3E000656C20002057680D20416363656C200038
:10E3F00025202D00206B6D0D20436F6E737420005F
:10E40000205768200020576800202B00506F776548
:10E4100072202D00495000534D53000A00232073F1
:10E42000696D2064617461206C696E6520002C0048
:10E430002C38363430302C004D502D30204852547A
:10E440002D4750532D4C6F672C002C002C302C0086
:10E4500063004D502D302000545A004E4C00544360
:10E46000004F32005254005641005452002C002CF0
:0BE47000302C0063004D502D302000C8
:04E47C00FF0012008B
:10E48000D3EC77F0060EDF5C05E29EA2FED79E92EB
:10E49000DF2AF8D7FCEF76F0D3EC77F07A0EDF5C6A
:10E4A00005E29EA2FED79E92DF2AF8D7FCEF76F017
:10E4B0008EEC77F0FE0EDB50000804E2EDDFFE0E7E
:10E4C000DB06F8D7ACEF77F070EF77F070EF77F00E
:10E4D00081B005D08180050EE66EEADFE5528190BD
:10E4E000140EE66EE5DFE552818012008EEC77F0C7
:10E4F0000E0E5DEC77F0EDEC89F000EC77F02E0E6F
:10E50000E66E87EC77F0CEEC97F083EC77F00C0EAC
:10E51000F3CFDBFF0D0EF4CFDBFFF3CF00F0F4CF32
:10E5200001F0F350F41001E1C6D0040EDB6A050ED1
:10E53000DB6A060EDB6A070EDB6A010EF36E080E5D
:10E54000F3CFDBFF090EDB6A0A0EDB6A0B0EDB6A18
:10E550000C0EDB2ADBCFE9FF0D0E01E3DB2ADBCF5C
:10E56000EAFFEF5057E0040EDBCF00F0050EDBCFE3
:10E5700001F0060EDBCF02F0070EDBCF03F052EC0A
:10E5800077F000C026F001C027F002C028F003C0D9
:10E5900029F089ECA7F02EEC77F00C0EDBCFE9FF29
:10E5A0000D0EDBCFEAFFEF50D00F046E056A066A4E
:10E5B000076AE85000260550012206500222075043
:10E5C0000322040E00C0DBFF050E01C0DBFF060EB8
:10E5D00002C0DBFF070E03C0DBFF080EDBCF26F017
:10E5E000090EDBCF27F00A0EDBCF28F00B0EDBCFB6
:10E5F00029F052EC77F089ECA7F0080E22C0DBFF7F
:10E60000090E23C0DBFF0A0E24C0DBFF0B0E25C062
:10E61000DBFF9ED7C2EC77F0EECF08F0EECF09F02B
:10E62000EECF0AF0EFCF0BF09CDB040EDBCF14F043
:10E63000050EDBCF15F0060EDBCF16F0070EDBCF95
:10E6400017F014C026F015C027F016C028F017C028
:10E6500029F03EEC82F027C010F028C011F029C04C
:10E6600012F02AC013F0080EDBCF1CF0090EDBCF2E
:10E670001DF00A0EDBCF1EF00B0EDBCF1FF01CC00F
:10E6800026F01DC027F01EC028F01FC029F03EEC68
:10E6900082F027C018F028C019F029C01AF02AC04B
:10E6A0001BF04DDBE4DBEEEC82F0EADB48DB9BDBCE
:10E6B00058EC82F002D039DBB6DB4ADB27C026F00B
:10E6C00028C027F029C028F02AC029F00E0EE15CEE
:10E6D00002E2E16AE55260D38EEC77F0080EEDDBE2
:10E6E00005DF8EDBC2EC77F0EECF00F0EECF01F06D
:10E6F000EECF02F0EFCF03F02C6A2D6AC80E2E6E1B
:10E70000420E2F6EC6DBEEEC82F00CEC85F0040EB0
:10E7100026C0DBFF050E27C0DBFF060E28C0DBFF8F
:10E72000070E29C0DBFF040EDBCF04F0050EDBCFA4
:10E7300005F0060EDBCF06F0070EDBCF07F073DB2C
:10E7400007DBC2EC77F0EECF10F0EECF11F0EECF9A
:10E7500012F0EFCF13F0040EDBCF18F0050EDBCF75
:10E7600019F0060EDBCF1AF0070EDBCF1BF0640E9C
:10E770002B6E2C6A2D6A2E6A18C026F019C027F05D
:10E780001AC028F01BC029F089ECA7F022C018F0AD
:10E7900023C019F024C01AF025C01BF022C026F0B7
:10E7A00023C027F024C028F025C029F03EEC82F0D9
:10E7B00027C014F028C015F029C016F02AC017F0A1
:10E7C000BEDA55DB57EC82F05BDB2C6A2D6A700EEB
:10E7D0002E6E420E2F6EEEEC82F027C008F028C09D
:10E7E00009F029C00AF02AC00BF0A9DA52DB58EC74
:10E7F00082F01CDB9ADA77DBF6DA41EC83F0A8DAF8
:10E800002C6A2D6A2E6A450E2F6E41EC83F00CECBB
:10E8100085F0080EE15C02E2E16AE552BDD27EDBE2
:10E82000040EE126DE68DD68FB0EDBCF00F0FC0E97
:10E83000DBCF01F0013435E200500008000E015436
:10E8400030E2A2DA01E3DB2AEF50DF1AFB0EDB062F
:10E85000FC0E01E2DB06020EDB6A030EDB6A020E2F
:10E86000DBCF00F0030EDBCF01F0D890015004E6BF
:10E87000080E005C000E0158D7E2DF50010B06E0E5
:10E880001FDB010E001AA00E011A01D019DB00C017
:10E89000DEFF01C0DDFF020EDB2A030EE0E3DB2A10
:10E8A000DED7DECF00F0DDCF01F000C0F3FF01C006
:10E8B000F4FF040EE15C02E2E16AE5526DD22EDB68
:10E8C00019DBEE50ED100CE06BDB0AE069DB0D08A4
:10E8D00003E10BDA0A0EEF6EBDDAF2E3DB2AF0D7C2
:10E8E0003BD31CDBD950FA0F72DBEFCFF6FFEE2AD9
:10E8F000EFCFF7FF000EEE22EFCFF8FFEE22080079
:10E90000F55058DB04E0A6DAEDE3DB2AEBD7E6D1DD
:10E9100005DBFB0EDBCFE9FFDB2AFC0EDBCFEAFFDA
:10E9200001E3DB2AEF5046DB04E094DAF2E3DB2A72
:10E93000F0D7D4D1D5D901E0C9D942DB58DB5CD2BC
:10E94000CFD901E0C3D969DA98EC8AF0DCDAE55274
:10E9500027DB04E07FDAFCE3DB2AFAD7BFD1C0D99A
:10E9600001E0B4D9BFD932EC8BF0A2DA19DB04E0B4
:10E9700071DAFCE3DB2AFAD7B1D1B2D901E0A6D92A
:10E98000B1D925EC8CF094DA0BDB04E063DAFCE31C
:10E99000DB2AFAD7A3D144DA54DA040EEE26000EAD
:10E9A000ED22FB0EDBCFE9FFFC0EDBCFEAFFEF6AC7
:10E9B000040EDF6EDF5023E08BDAE76EFD0EDBCF57
:10E9C00003F0FE0EE7500316046A056AE7D9FB0E52
:10E9D000DB06DBCFE9FFFC0E01E2DB06DBCFEAFF63
:10E9E000E552E750EF6E86DA040E0F0B06E0EC52AC
:10E9F000D890ED32EF32E806FAE1DF06DBD7FCD142
:10EA00006FD901E063D909DAC6DF7DDAE552C8DAE9
:10EA100004E020DAFCE3DB2AFAD760D101DAD9502E
:10EA2000F90FD5DA080EEE26000EED22F90EDBCF37
:10EA3000E9FFFA0EDBCFEAFFEF6A080EDF6EDF5068
:10EA40002AE046DA036E046A056A066AFAD9EE50CD
:10EA50000316EE500416EE500516EE5006169ED91B
:10EA6000F90EDB06DBCFE9FFFA0E01E2DB06DBCFB6
:10EA7000EAFFE552E750EF6EE4D9040EE76ED89056
:10EA8000030EEB32020EEB32010EEB32EF32E706F1
:10EA9000F6E1DF06D4D7B0D123D901E017D922D9C6
:10EAA000BDDF06DA7DDA04E0D5D9FCE3DB2AFAD74C
:10EAB00015D134DA0C0EA2D901E008D91FDA33DA05
:10EAC00025EC8CF0F5D91ADA3CEC98F0E552E552D9
:10EAD0000B0EF3CFDBFFDB50006E016AF40EDBCFD1
:10EAE00002F0F50EDBCF03F001500318E8AE02D0C0
:10EAF000033404D00250005C0350015809E244D9A9
:10EB000001E3DB2AF30EDBCFEFFF0B0EDB2AE3D7AB
:10EB1000F5D96DDAE55253D90C0EE15C02E2E16AF7
:10EB2000E5523AD1FBD9050EE126010EDE6EDE6A12
:10EB3000DE6ADD6ADD52DD52F40EDB50E76E040E54
:10EB4000E7CFDBFFDB50000817E21CDAABD9EECFD2
:10EB500026F0EECF27F0EECF28F0EFCF29F089ECAA
:10EB6000A7F025C0EDFF24C0EDFF23C0EDFF22C0BC
:10EB7000EFFF040EDB06E6D7BFD8EEEC83F022D918
:10EB80002BDAEDDE086E090EE15E0850F4D9FCD8F0
:10EB900001E3DB2A2E0EEF6E300EE66EF40EDBCFB5
:10EBA000E6FFF50EDBCFE6FFA7D82EC0F5FFEEECB3
:10EBB00083F0F5AE08D0000E226C231E2322241E03
:10EBC0002422251E25224AD922C0E6FF23C0E6FFC3
:10EBD00024C0E6FF25C0E6FF38D96BDF086E0C0EB7
:10EBE000E15E0850ECD8050EE15C02E2E16AE55214
:10EBF000D3D094D9040E02D901E068D8D950F60FC9
:10EC0000E6D9D890030EEB50000A08E6000EEE5C41
:10EC1000000EEE58000EEE58000EEE5821E2B4D869
:10EC200001E3DB2A2D0EEF6EF60EDBCF00F0F70EC0
:10EC3000DBCF01F0F80EDBCF02F0F90EDBCF03F0F3
:10EC4000001E011E021E031EF60E00C0DBFFF70EA3
:10EC500001C0DBFFF80E02C0DBFFF90E03C0DBFFD3
:10EC6000F60EDBCF08F0F70EDBCF09F0F80EDBCFA6
:10EC70000AF0F90EDBCF0BF074D82C6A2D6A2E6ADD
:10EC8000450E2F6EEEEC82F063D82DD9EEEC82F0BB
:10EC9000CDD8060EE66EE66A48D82C6A240E2D6E94
:10ECA000740E2E6E490E2F6E9ED841EC83F00CEC44
:10ECB00085F088D8CAD836DF086E0B0EE15E0850A2
:10ECC000040EE15C02E2E16AE55266D085D909DE14
:10ECD000006E050EE15E0050BBEF77F041D93CD1EC
:10ECE0001DD92DD114D993EF77F0FD0EDBCFE9FFBD
:10ECF000FE0EDBCFEAFF1200F60EDBCF04F0F70EBC
:10ED0000DBCF05F0F80EDBCF06F0F90EDBCF07F016
:10ED10003ED9DFCF2BF0010EDBCF2CF0020EDBCF84
:10ED20002DF0030EDBCF2EF012002CD9EECF04F025
:10ED3000EECF05F0EECF06F0EFCF07F0120027C0C0
:10ED40002CF028C02DF029C02EF02AC02FF0120080
:10ED500027C000F028C001F029C002F02AC003F04B
:10ED6000120008C026F009C027F00AC028F00BC026
:10ED700029F03EEC82F027C004F028C005F029C03D
:10ED800006F02AC007F01200FD0EDBCFE9FFDB2AF8
:10ED9000FE0EDBCFEAFF1200E16EDED0005003244E
:10EDA000F36E01500420F46E02500520F86EF4CF8B
:10EDB000F7FFF3CFF6FF0800F550E66E1200DBD840
:10EDC000B0EF77F026C000F027C001F028C002F0B5
:10EDD00029C003F026C0E6FF27C0E6FF28C0E6FFF3
:10EDE00029C0E6FF120004C027F005C028F006C0C5
:10EDF00029F007C02AF01200E552AED0E1269FD0DC
:10EE0000E552E55226C0DEFF27C0DEFF28C0DEFF48
:10EE100029C0DDFFDD52DD52120079D8E0EF77F036
:10EE20007DD8E6521200B3D83EEF82F027C0DEFF55
:10EE300028C0DEFF29C0DEFF2AC0DDFFDD52DD5223
:10EE40001200D950FB0FE7EF77F0E66AE66AE66A50
:10EE500087EF77F0FD0EDB2AFE0E120022C000F0D5
:10EE600023C001F024C002F025C003F0120010C03E
:10EE700027F011C028F012C029F013C02AF01200A8
:10EE800027C00CF028C00DF029C00EF02AC00FF0EA
:10EE9000120000C027F001C028F002C029F003C012
:10EEA0002AF012000A0E2B6E2C6A2D6A2E6A1200AE
:10EEB000006E060EE15E00501200E12687EF77F04B
:10EEC000DECF00F0DDCF01F0D89001320032120029
:10EED000730E006EDF0E016E000E026E0F0E12003A
:10EEE000D9CFE6FF39D02C6A2D6A610E2E6E450E01
:10EEF0002F6E1200D950FD0FE7EF77F0D9CFE6FF64
:10EF0000DACFE6FF1200E552E552E5521200FD0E9F
:10EF1000DBCFE6FFFE0EDBCFE6FF1200D9CFE6FF28
:10EF2000E1CFD9FF1200D950F60F51D8EECFE6FF4E
:10EF3000EECFE6FFEECFE6FFEFCFE6FF1200FA0ED0
:10EF4000DBCF00F0FB0EDBCF01F0FC0EDBCF02F0DD
:10EF50000050011002101200E552E7CFD9FF120055
:10EF6000FD0EDBCF00F0FE0EDBCF01F000C0F3FFA3
:10EF700001C0F4FF1200FD0EF3CFDBFFFE0EF4CF55
:10EF8000DBFF1200D9CFE9FFDACFEAFF120004C09D
:10EF900026F005C027F006C028F007C029F01200AF
:10EFA000A4DEEF5012003CDFDF6A7C0ECA6ECC6A32
:10EFB000CB681200E66E99DEE552E750EF6E120064
:10EFC000F80EDBCFE6FFF90EDBCFE6FF1200E96EAD
:10EFD000FF0EDA20EA6E1200FA0EDBCFE6FFFB0E20
:10EFE000DBCFE6FFFC0EDBCFE6FF87EF77F08FDFAE
:06EFF0008FDC83EF77F0D7
:0AEFF600DEEC7CF0030EE126020EB3
:10F00000DB6A000E0901E76EE119E8AE02D0E135D6
:10F0100003D0E750D880E15501E2E107000E090175
:10F02000E76EE219E8AE02D0E23503D0E750D880AF
:10F03000E25501E2E20709010A51000807E20A0766
:10F0400003E109019B9102D009019B810901A52BD4
:10F05000000EA623A723A8230901905157E0090118
:10F060008E518F1153E0090199B715D00C0E9913E9
:10F070000901966B0901976B0901010E946F090153
:10F08000030E956F0901100E916F0901926B936B3E
:10F090000901986B5FD00901052B3C0E055D63E308
:10F0A000056B0901922B000E932309019051026E0A
:10F0B000036A90C928F003C029F08EC92DF08FC9CA
:10F0C0002EF04FEC84F026C000F027C001F00001C4
:10F0D0002650090106270001275009010723000EC9
:10F0E00008230923600E065DEA0E0759000E085931
:10F0F000000E095938E30901982B600E0901065FDB
:10F10000EA0E075B000E085B095B2DD009019051E8
:10F110002AE109018E518F1126E1090199A723D017
:10F12000F30E99170901966B0901976B5F0E0901A0
:10F13000A05D0AE20901150E946F09010E0E956F8C
:10F14000040ECDEC7CF006D00901040E946F090189
:10F15000030E956F0901056B066B076B086B096B56
:10F16000020ECDEC7CF009010F5119E0010EE66EA4
:10F1700058EC72F0E5520DEC2EF0100EE66E090E12
:10F18000E66E000EE66E060EE66E02EC98F0E552B4
:10F19000E552E552E5523AEC2EF009010F6B0451AD
:10F1A00008E10901905105E109018E518F1101E13A
:10F1B00092D00501F45101E18ED0DE6ADD6A9ADB5E
:10F1C00006BE076819EC7DF00050011001E181D006
:10F1D0009E0E046E500E056E010E066EDECF07F019
:10F1E000DDCF08F0096A08BE0968050E2C6E2D6A8D
:10F1F0002E6A07C027F008C028F009C029F06DEC7E
:10F2000084F024C007F025C008F026C009F004509F
:10F210002424F36E05502520F46E06500BEC7DF08F
:10F22000020EE0DB0800F550026E036AC8C728F042
:10F23000C9C729F02D6E03C02EF066ECA8F024C0DB
:10F2400000F025C001F0245025103DE1020EDB50F6
:10F2500002E04CEC72F00F0140B7FDD7406B4ADB87
:10F2600006BE0768E6DB070E0016000E0116050E47
:10F27000D89000360136E804FBE100C042FF3ADBDB
:10F2800006BE0768D6DB030ED89001320032E804D0
:10F29000FBE100C041FF0F01030E466F220E476FD6
:10F2A00029DB06BE0768B2DB01C000F0016A00C0BE
:10F2B00048FF20DB06BE0768A9DB005052DBF36E77
:10F2C000020EF3CFDBFFDF2A010E01E278D7DB2A43
:10F2D00076D70901046B000E006E030EE15C02E2BA
:10F2E000E16AE55238D36ADB080EE1266250026E0D
:10F2F000036A050ED89003320232E804FBE1615044
:10F30000046E056A030ED89004360536E804FBE166
:10F3100002500424006E03500520016E060E00C04A
:10F32000DBFF070E01C0DBFF0F0E65140B01406F02
:10F3300066CF41FB67CF42FB68CF43FB69CF44FBFD
:10F340006ACF45FB6BCF46FB6CCF47FB6DCF48FBCD
:10F35000609E09013C0E0A6F43CB03F0026A0B0169
:10F3600044510224006E000E032000C0DEFFDD6E5B
:10F37000020E45CBDBFFDECF00F0DDCF01F009014F
:10F380000D51001854E10E51011851E1060EDBCF6A
:10F3900002F0070EDBCF03F00B51021848E10C51CD
:10F3A000031845E10F5143E1520EE66EE40EE66E9E
:10F3B000000EE66E100EE66E090EE66E71EC74F04D
:10F3C000006E050E1ADB2E0EE66EE66A500EE66E35
:10F3D000E40EE66E000E81DA060EDBCFE6FF070EC6
:10F3E000DBCFE6FF4C0EE66EE40EE66E000E75DA3D
:10F3F000DECFE6FFDDCFE6FFFADA6FDA030EDB6A77
:10F40000080EF36E030EDBCFF4FFF350F45C08E25A
:10F41000030E98DAE66AEBDA60DA030EDB2AF0D73D
:10F420000901010E0F6F0B6B0C6B0D6B0E6B620EF7
:10F430000B01425D02E0010EDED0D950060FE96EED
:10F44000DACFEAFFEC0EEE1801E091D0070EED18CE
:10F4500001E08DD0000EDFCF28F0010EDBCF29F0C8
:10F46000340E281802E1830E291859E0430E28189B
:10F4700002E11C0E29184FE04F0E281802E1430E3E
:10F48000291845E01E0E281802E1800E29183BE0DD
:10F490001F0E281802E1800E291827E0680E281890
:10F4A00002E1430E291818E0690E281801E0A2D0E5
:10F4B000430E291801E09ED0020EDB50006E016A57
:10F4C000050E2D6E2E6A00C028F001C029F066ECF2
:10F4D000A8F028C090F98ED0020EDB5009018E6F83
:10F4E0008F6BD8908E378F3785D009013C0EE16F36
:10F4F000020EDB50E8307F0B006E280E005E000E1F
:10F5000000C0ADF977D009013C0EE26F73D04CDA40
:10F5100000C0C2F96FD048DA00C0C0F96BD0090151
:10F520003C0EE26F020EDB50270DF3CF00F0F4CF5C
:10F5300001F0630E50DAC8EC83F028C000F029C057
:10F5400001F028C0A0F909012850250DF3CFA1F939
:10F55000F4CFA2F9640E3FDA66ECA8F028C0A1F956
:10F5600029C0A2F928C0A3F929C0A4F943D0D950D1
:10F57000060FE96EDACFEAFFE80EEE183BE1070E60
:10F58000ED1838E1D9CFE9FFDACFEAFF0D0EEE181A
:10F5900031E1EE502FE14B0E0701CB5D04E1020E8D
:10F5A000DBCF9FF927D0020EDBCF26F0276A286A2F
:10F5B000296AE80E2B6E030E2C6E2D6A2E6A89ECDA
:10F5C000A7F022C026F023C027F024C028F025C0D1
:10F5D00029F0F40E2626010E2722000E28222922C9
:10F5E000490E2B6E060E2C6E2D6A2E6AF1ECA7F0DA
:10F5F00026C09FF9010E006E080EE15C02E2E16A8E
:10F60000E552A9D1DBD9020EE1260F0E0F015515E7
:10F610000B01406F56CF41FB57CF42FB58CF43FB06
:10F6200059CF44FB5ACF45FB5BCF46FB5CCF47FB32
:10F630005DCF48FB50CFDFFF0F01509F0901010E46
:10F64000046F3C0E0A6F070EDF14020850E0070E2D
:10F65000DF1403080EE1010EDB6AB5D907E2010EE3
:10F6600071D9010EDB50090F87D9F7D70901BF6B9C
:10F670003ED0070EDF1404080DE10901310EAE6F14
:10F68000010EDB6AA0D933E2010E5CD9010EDB2842
:10F6900073D9F8D7070EDF14050829E10B01415192
:10F6A00017E10901998D999F0901A951AA11AB117F
:10F6B000AC111DE1A5C9A9F9A6C9AAF9A7C9ABF959
:10F6C000A8C9ACF9A907000EAA5BAB5BAC5B0DD077
:10F6D0000901999D998F0901A951AA11AB11AC118A
:10F6E00006E0A96BAA6BAB6BAC6B010E56D9010E91
:10F6F000006E020EE15C02E2E16AE5522CD15ED9B5
:10F70000FC0EDBCF28F0FD0EDBCF29F02E0E2818E3
:10F710004CE129504AE16BD9E66E84D9F7D80CE068
:10F7200036D9F3CF0BF9F4CF0CF961D9E66E000EA0
:10F73000E66EE66AEBD802E1000E38D028D9F3CFA6
:10F740000DF9F4CF0EF909010F6B4CEC72F00F01BB
:10F7500040B7FDD7406B070E09010B15006E016A1B
:10F76000050ED89000360136E804FBE100C042FFE8
:10F770000BC900F00CC901F0030ED8900132003221
:10F78000E804FBE100C041FF080E09010B27000E51
:10F790000C230F01030E466F220E476F016A0EC93C
:10F7A00048FF09010D51DDD801D0000EE552E7CF29
:10F7B000D9FF1200D9CFE6FF020EE1260501560E51
:10F7C000C86F410EC96FCA6BCB6BCC6B0901DC0EE5
:10F7D000006FDA0E016FD40E026F340E036F046BEC
:10F7E000056B066B076B086B096B0A6B0B6B0C6B7D
:10F7F0000D6B0E6B0F6B0901E5690901A56BA66B1B
:10F80000A76BA86B900E6F6E6EAEFED7606A0F018D
:10F81000196B1869016BFD0E006F506BE00E1D6FC8
:10F820001C69C00E096F400E086F200E0D6F9C0EF4
:10F830000C6F800E116FA20E106FA00E156F260EAA
:10F84000146F010E706ED20E716E020E726E200E6B
:10F85000736E0501F451000802E26F6A02D0600E77
:10F860006F6E0701E60ED56FF20ED66F000ED76FE2
:10F870000701040ED86FF60ED96F000EDA6F07017C
:10F88000F60EDB6FEF0EDC6F000EDD6F0B01FE0E70
:10F89000496FF60E4A6F000E4B6F0601EE81EE8344
:10F8A000010E006E020EE15C02E2E16AE55253D005
:10F8B000050E2C6E2D6A2E6A05C027F006C028F0B2
:10F8C00007C029F06DEC84F002502424F36E03503D
:10F8D0002520F46E04500BEF7DF0E66E040EDBCFB6
:10F8E000E6FF050EDBCFE6FFA0EC74F0006E070E1E
:10F8F000FDEF7CF09E0E026E500E036E010E046E44
:10F90000DECF05F0DDCF06F0076A1200E3ECA3F0CE
:10F91000006E050EE15E0050FA0EF3CFDBFFFB0E2A
:10F92000F4CFDBFFD950FA0FE96EFF0EDA20EA6E52
:10F93000EE50ED1012000900F5CF00F00800F5CFF1
:10F9400001F01200DB50EA6A410FE96E0B0EEA2269
:10F95000EF50E66E1200E16E0050E552E7CFD9FF9E
:10F9600012000F01496F4A6B4B6B4C6B4D6B080ECD
:10F97000456F406F010E1200EA6AAE0FE96E090E84
:10F98000EA22E552E750EF6E010EDB2A12004AD858
:10F9900078EC89F0E552E5521200E66EE66AFEEC7C
:10F9A0003EF0E552E552120009013C0EE26F020EF4
:10F9B000DB50006E280E005E000E1200D9CFE6FF6D
:10F9C000E1CFD9FF1200080EF36E010EDBCFF4FF7A
:10F9D000F350F45C12002D6E2E6AF3CF28F0F4CFB2
:10F9E00029F01200F626000EF722F82212004A0E25
:10F9F000E66EE40EE66E000E1200E15E0050040EAC
:10FA0000F3CFDBFF050EF4CFDBFF120051DF030E57
:10FA1000E9DF9BEF7CF02620F86EF4CFF7FFF3CF01
:10FA2000F6FF1200FA0EDBCFE6FFFB0EDBCFE6FFA0
:08FA300012003EDF9BEF7CF0A9
:08FA38000A0EE66E010EE66EF7
:10FA40008DEC81F00A0EE66EE66A8DEC81F0F3EC47
:10FA5000A1F00601CE6BCF6B0601CD6B09012E0E16
:10FA6000FC6FE10EFD6F000ED2EC81F0F4C5E7F8FB
:10FA70000801E869E969120065EC81F0030EE126EE
:10FA80000801800EE91501E0A5D0140E006E450EA8
:10FA9000016E010E026E1C0E066E450E076E010E03
:10FAA000086EE8C809F0E9C80AF0090E0A02F3CFA7
:10FAB0000AF00902F3CF09F0F4500A260B6A0ABED5
:10FAC0000B6806500924F36E07500A20F46E0850A4
:10FAD0000B20DDEC81F00800F5CF03F0046A056A25
:10FAE000D890033604360536BFDB0900F5CFDEFFBC
:10FAF0000A00F5CFDDFF0F01406B9DEC81F0070E92
:10FB00000016000E0116050ED89000360136E804E6
:10FB1000FBE100C042FF9DEC81F0030ED890013262
:10FB20000032E804FBE100C041FF010EF36E020E5B
:10FB3000F3CFDBFF6DDB04BE0568DAEC81F0F5CFB7
:10FB400046FF66DB04BE0568DAEC81F0F5CF47FFBF
:10FB50005FDB04BE0568DAEC81F0F5CF48FF58DBC7
:10FB600004BE0568DAEC81F0F5CF49FF51DB04BE35
:10FB70000568DAEC81F0F5CF4AFF4ADB04BE056880
:10FB8000DAEC81F0F5CF4BFF43DB04BE0568DAEC1D
:10FB900081F0F5CF4CFF3CDB04BE0568DAEC81F068
:10FBA000F5CF4DFF0F01080E456F4087010E08018C
:10FBB000E825E86F000EE921E96F110E2D6E2E6A1F
:10FBC000E8C828F0E9C829F0C8EC83F024C0E8F8B8
:10FBD00025C0E9F8040E0601F115006E040EB2DB33
:10FBE00009E00901140EFC6FE10EFD6F000EAFDBA2
:10FBF000F195F295100EF115006E100EA3DB09E0E1
:10FC00000901FB0EFC6FE00EFD6F000EA0DBF19909
:10FC1000F299200EF115006E200E94DB09E0090127
:10FC2000E20EFC6FE00EFD6F000E91DBF19BF29B8C
:10FC3000030EE15C02E2E16AE552E16E4BD345DB83
:10FC4000020EE126E66A1CEC9FF0E552F3CFDEFFE0
:10FC5000F4CFDDFF43DB0FE0140EE66EE66ADECF85
:10FC6000E6FFDDCFE6FF76DB9AEC98F0006E060E3D
:10FC7000E15E005008D0D90EE66EE00EE66E6ADB5B
:10FC800002EC98F06CDBFADA31DB3CEC98F0E552F0
:10FC9000E552F350E66E2ADB5DDBDBEC60F098DBCF
:10FCA000020EE15C02E2E16AE552E16E13D30DDB84
:10FCB000E5DA1CDBB6EC34F0E552E5520A019E5160
:10FCC0009F1105E00A015E5102E189EC36F002D392
:10FCD000FCDAD4DA27DBAD0EFC6FE00EFD6F000E10
:10FCE00061DB0901990EFC6FE00EFD6F000E5ADB1F
:10FCF00052DB51DBA4DF33DB0901850EFC6FE00E24
:10FD0000FD6F000E4FDBE66A20EC32F0E552E2D2E6
:10FD1000DCDAE66A010EE66E00DBE66AE66AFDDA28
:10FD2000F3ECA1F0ABDAFEDA680EFC6FE00EFD6FCB
:10FD3000000E38DB0A0E39DB3EEC72F0CBD2C5DAAE
:10FD4000050EE126010EF36E020EF3CFDBFFF36E1C
:10FD5000DB6E09015C0EFC6FE00EFD6F000E22DB16
:10FD60000E0EF66E000EF76E000ED1DA4F0EE66E36
:10FD7000E00EE66E000E3EDB0F0EF66E000EF76E26
:10FD8000000E30DB100EF66E000EF76E000E2ADB52
:10FD90000E0EE66E1CEC9FF0E552F3CF00F0F4CFB0
:10FDA00001F0F3CFE6FFF4CFE6FFA7DA9AEC74F0A8
:10FDB000026E070EE15E0250DFDA0701CC51CD1171
:10FDC000CE1108E0CCC7E6FFCDC7E6FFCEC7E6FF01
:10FDD0001FDB19DB020EDBCFE6FFE66A480EE66E9C
:10FDE000E00EE66E000EC5DACEDAC7ECA7F0E66EDE
:10FDF000E66A3A0EE66EE00EE66E000E60DAC3DAF0
:10FE0000CCECA7F026C000F027C001F028C002F01B
:10FE100029C003F02C6A2D6A200E2E6E410E2F6E23
:10FE200026C027F001C028F002C029F003C02AF044
:10FE300041EC83F0DDEC84F028C0DEFF29C0DDFF5B
:10FE4000010EE66EE66A79DA026A036A00C0E6FF2E
:10FE500001C0E6FF02C0E6FF03C0E6FF2C0EE66E1F
:10FE6000E00EE66E000E2BDA92EC75F0046E0B0ECF
:10FE7000E15E045081DA270EE66EE00EE66E000EBB
:10FE8000E5D90901E951E66EE66A190EE66EE00E63
:10FE9000E66E000EAFDA150EE66EE00EE66E000EB0
:10FEA000D5D9AE0EE66E090EE66E070EE66EE00ED2
:10FEB000E66E000E04DA28DAC80EE66E050EE66E6F
:10FEC000040EE66EE00EE66E000E53DA1DDA000E4A
:10FED000E66EE00EE66E000EB9D90901A051E66E9D
:10FEE000E66AF20EE66EDF0EE66E000E83DAA1C958
:10FEF000E6FFA2C9E6FFEE0EE66EDF0EE66E000E2E
:10FF000092DAA3C9E6FFA4C9E6FFE50EE66EDF0EAE
:10FF1000E66E000E88DAD70EE66EDF0EE66E000E95
:10FF200095D90801800EE9150FE1E8C8E6FFE9C898
:10FF3000E6FFCB0EE66EDF0EE66E000E5BDA110E0C
:10FF4000E66EE66ADAD91FDA0901C90EFC6FDF0E28
:10FF5000FD6F000EC6D9BF0EFC6FDF0EFD6F000EE9
:10FF6000C0D9B50EFC6FDF0EFD6F000EBAD9AD0E15
:10FF7000FC6FDF0EFD6F000E15DA050EE15C02E28C
:10FF8000E16AE552E16EA6D1A0D9B0D978EC89F04A
:10FF9000E552E552F3CFE9F99DD197D9F4C5E7F8D9
:10FFA0000501010EF46FA0EC92F00801E86BE96B1B
:10FFB0000901980EFC6FDF0EFD6F000E30D285D95F
:10FFC000E7C8F4F5A0EC92F00801E869E9690901D5
:10FFD000840EFC6FDF0EFD6F000E21D276D9040E69
:10FFE000E12666D9EF5001E10CD162D9EF50230828
:10FFF00001E107D1FD0EDBCFDEFFDBCFDDFF6ED9E8
:020000040001F9
:1000000018E06CD9200815E069D960080DE2E5D93F
:10001000EFCF00F07B0E005C07E260D9E00FE66EE8
:10002000DCD9E552E750EF6EDF2A010EE8E3DB2A68
:10003000E6D754D9200804E1DF2A010E01E3DB2AC8
:10004000020EDB6A030EDB6AB50E006E450E016E12
:10005000010E026E020EDBCF03F0030EDBCF04F0C5
:10006000056A04BE056880D903C027F004C028F0E3
:1000700005C029F06DEC84F024C003F025C004F025
:1000800026C005F000502424F36E01502520F46EA4
:100090000250262092D90800F55001E1A0D0B50EFB
:1000A000056E450E066E010E076E020EDBCF08F0E0
:1000B000030EDBCF09F00A6A09BE0A6855D908C0E9
:1000C00027F009C028F00AC029F06DEC84F024C0A4
:1000D00008F025C009F026C00AF005502424026E5D
:1000E00006502520036E07502620046E02C0E6FF4E
:1000F00003C0E6FFE66E4AEC98F0E552E552E552A1
:1001000027C000F028C001F027C0E6FF28C0E6FFA6
:10011000B50E0E6E450E0F6E010E106E020EDBCF89
:1001200011F0030EDBCF12F0136A12BE13681CD954
:1001300011C027F012C028F013C029F06DEC84F034
:1001400024C011F025C012F026C013F00E50242454
:100150000B6E0F5025200C6E105026200D6E0BC01C
:10016000E6FF0CC0E6FFE66E16D92AEC97F0146E97
:10017000070EE15E145000092BE1020EDBCFE9FF10
:10018000030EDBCFEAFFEA02F3CFEAFFE902F3CF87
:10019000E9FFF450EA26EA0EE926080EEA22EECF3D
:1001A00000F0EECF01F0EFCF02F0DECFE6FFDDCFC3
:1001B000E6FFFD0EDBCFE6FFFE0EDBCFE6FF06D04F
:1001C00002C0FBFF01C0FAFF0050F96EF9DF18D042
:1001D000020EDB2A030E01E237D7DB2A35D768D8B7
:1001E000EF50530805E1EFD803E150D828DD08D0DF
:1001F0005FD8EF504D0805E1E6D803E147D857DD59
:10020000AED8040EE15C02E2E16AE552E16E62D032
:100210001C0E006E450E016E010E026E020EDBCF4B
:10022000F3FFDB2AF350066E076A090E286E296A6F
:10023000E8C82DF0E9C82EF022EC84F02650062400
:10024000036E27500720046E056A120092D8DBD88F
:10025000000EE66E060EE66EA3EC3EF0E552E552A9
:100260001200A0EC74F0C9D000500324F36E0150CA
:100270000420F46E02500520DDEF81F00901D60E56
:10028000FC6FE00EFD6F000ED2EF81F0020EE76E04
:10029000FD0EDBCF00F0FE0EDBCF01F0E7500026B5
:1002A000000E012200C0E6FF01C0E6FFCBEF81F0A7
:1002B000FD0EDBCFE9FFFE0EDBCFEAFF1200E66E9C
:1002C000000EE66E060EE66E1200D9CFE6FFE1CF15
:1002D000D9FF1200E552E7CFD9FF12007ED8EF50C8
:1002E000120060D8050E61D809011200FB0EDBCFA9
:1002F000E6FFFC0EDBCFE6FF12004B0EE66EE00ED3
:10030000E66E000EB9EF81F09AEC74F076D0F86EDC
:100310000800F550E66EE66A1200CCECA1F0E5525A
:10032000E5521200010E41D809011200E750E926FA
:10033000000EEA22EF5020081200DECF00F0DDCFE1
:1003400001F01200F215016E0050011012002AD8BF
:1003500006011200D60EE66E060EE66E1200E5529B
:10036000E552E552E55212001B0E2C6E2D6A2E6AE4
:100370001200E66E08EF82F0030EF3CFDBFF040EEF
:10038000F4CFDBFF12006DDFD60EE66EE00EE66EF8
:10039000000E26EF81F0FD0EDBCFE6FFFE0EDBCF79
:1003A000E6FF1200FE6F54EF3EF0E66E58EC72F07E
:1003B000E552120059DF08001200F86EF4CFF7FF83
:1003C000F3CFF6FF1200010EE76E72DF96EF81F0B9
:1003D000006E050EE15E00501200DECFE9FFDDCFBA
:1003E000EAFF120094DF4D0EE66EE00EE66E000EA0
:1003F00013EF82F064DF31EF81F0006E070EE15EF3
:100400000050BCEF81F071EC74F0E2DFBCEF81F0E2
:10041000030EDBCFE6FF040EDBCFE6FF1200C2DFE8
:0C042000020EC3DF57D7A5DF31EF81F0DB
:04042C00219E05D038
:10043000219E29AE02D0296C218E29C023F0226A88
:10044000336A326A860E246E256ABDEF85F0219EDE
:1004500008D0219E29AE05D0286C291EE86A2922E1
:10046000218E29C023F028C022F0336A326A8E0E12
:10047000246E256ABDEF85F0219E0CD0219E29AE09
:1004800009D0266C271E281E291EE86A272228224A
:100490002922218E29C023F028C022F027C033F062
:1004A00026C032F09E0E246E256ABDEF85F02F7EA9
:1004B000216AF9EC85F011EC86F021B6A1EF85F008
:1004C00021A20AD021AA03D021BEA1EF85F021A448
:1004D000ADEF85F0AAEF85F021AA05D021ACADEFF4
:1004E00085F0AAEF85F021A00AD021A808D021BE6E
:1004F00004D021A402D0B6EF85F0BAEF85F0326ABD
:10050000256A2F502A5C316E10E327C033F028C0D3
:1005100022F029C023F02AC030F02CC027F02DC0D3
:1005200028F02EC029F0213A09D02CC033F02DC07C
:1005300022F02EC023F02FC030F0316C219E21BC60
:10054000218E30C024F021B0E9EF85F01A0E316021
:10055000E9EF85F0246A2A6A21A408D0276C281EB6
:10056000291E2A1EE86A282229222A2221AC08D024
:10057000336C221E231E241EE86A222223222422F8
:10058000266A315207E02A342932283227322632AD
:10059000312EF9D7275033262850222229502322E2
:1005A0002A50242226C032F0219E24AE0BD0326C79
:1005B000331E221E231E241EE86A332222222322F7
:1005C0002422218E24A006D0D88023322232333236
:1005D0003232302A30C024F0BDEF85F0216AF9ECC8
:1005E00085F011EC86F021B6A1EF85F021A205D0AF
:1005F00021BAA1EF85F0A8EF85F021BAB4EF85F01C
:1006000021A005D021B8A1EF85F0B4EF85F021B885
:10061000A8EF85F0256A7F0E2A24246EE86A252239
:100620002F50245EE86A255A1A0E306E2A6A326A02
:10063000336A226A236A2C50275E2D50285A2E5086
:10064000295A000E2A5A09E72C5027262D50282215
:100650002E502922000E2A2201D0328AD890273625
:10066000283629362A36D890323633362236233683
:10067000302EE1D7295028102710D8A4328ABDEF98
:1006800085F0216AF9EC85F011EC86F021B6A1EF36
:1006900085F021A205D021B8A1EF85F0A8EF85F063
:1006A00021AA05D021B0A1EF85F0A8EF85F021B0F7
:1006B00002D021A802D0B4EF85F0256A2F502A2459
:1006C000246EE86A25227E0E245EE86A255A326A84
:1006D000336A226A236A2E502902F4CF23F0F3CF23
:1006E00022F02D502902F3503326F4502222000E1E
:1006F00023222E502802F3503326F4502222000EDB
:1007000023222C502902F3503226F4503322000EBB
:10071000222223222D502802F3503226F450332275
:10072000000E222223222E502702F3503226F450AC
:100730003322000E222223222C502802F45032268B
:10074000000E3322222223222D502702F45032267B
:10075000000E332222222322BDEF85F0206A2EAE26
:10076000B4EF83F02E6C201E29AEB9EF83F0296C14
:10077000201EB9ECA8F029BEC3EF83F020AE000C18
:10078000296C256C000C20BEC0EF83F02188FF0C83
:10079000206A2EAED1EF83F02D6C2E1EE86A2E2239
:1007A000201E29AED9EF83F0286C291EE86A292281
:1007B000201E66ECA8F029BEE9EF83F020AE000C05
:1007C000286C291EE86A2922246C251EE86A252245
:1007D000000C20BEE0EF83F02188FF0C206AE86A5D
:1007E0002EAEFBEF83F02B6C2C1E2D1E2E1E2C220A
:1007F0002D222E22201E29AE06EF84F0266C271E05
:10080000281E291E272228222922201EF1ECA7F0CB
:1008100029BE1DEF84F020AE000C266C271E281E7A
:10082000291EE86A272228222922226C231E241E40
:10083000251E232224222522000C20BE0DEF84F049
:100840002188FF0C29C033F028C032F028502D0237
:10085000F4CF27F0F3CF26F029502E02F4CF29F061
:10086000F3CF28F02D02F3502726F4502822E86A0F
:10087000292232502E02F3502726F4502822E86A0B
:1008800029222EAE48EF84F03250285E3350295A88
:1008900033AE000C2D50285E2E50295A000C28C073
:1008A00032F028502D02F4CF27F0F3CF26F0295054
:1008B0002E02F4CF29F0F3CF28F02D02F350272693
:1008C000F4502822E86A292232502E02F3502726BB
:1008D000F4502822E86A2922000C29C033F028C0ED
:1008E00032F027C031F027502C02F4CF25F0F3CF9F
:1008F00024F028502D02F4CF27F0F3CF26F02C025D
:10090000F3502526F4502622E86A272231502D0282
:10091000F3502526F4502622E86A272229502C027B
:10092000F3502626F450272229502D02286AE86A1F
:100930002822F3502726F450282231502E02F3505B
:100940002626F4502722296AE86A282229223250D2
:100950002E02F3502726F4502822E86A2922335029
:100960002E02F3502826F4502922000C216AF9ECBB
:1009700085F021B6C0EF84F021A20AD021B403D0C3
:100980007F0E296E19D0800E296E16D0296A14D0D8
:1009900021B0FCD7870E2A60F1D77E0E2A64F6D7E5
:1009A000860E2A5C04E0D89029322A2AF9D721A49D
:1009B00003D0296C29AEEAD71200216AF9EC85F040
:1009C00021B6E7EF84F021A20ED021B405D07F0E2E
:1009D000296EFF0E286E1FD0800E296E286A1BD04C
:1009E000296A286A18D021B0FBD78F0E2A60EDD76C
:1009F0007E0E2A64F5D78E0E2A5C05E0D890293247
:100A000028322A2AF8D721A406D0286C291EE86AA1
:100A1000292229AEE5D71200216AF9EC85F021B62A
:100A200016EF85F021A20FD021B407D07F0E296EDA
:100A3000FF0E286E276E266E25D0800E296E01D0FF
:100A4000296A000EF6D721B0FBD7266A9F0E2A60CE
:100A5000EBD77E0E2A64F4D79E0E2A5C07E0D8906E
:100A600029322832273226322A2AF6D721A40AD060
:100A7000266C271E281E291EE86A272228222922E2
:100A800029AEDED712004CEC85F021B6000C21B067
:100A9000000C21A4000C010C216AF9EC85F011EC8A
:100AA00086F021B6120021AE08D021A004D021A8E2
:100AB00002D021801200219012002F502A5C0BE1FD
:100AC0002E50295C08E12D50285C05E12C50275C54
:100AD00002E121801200D8A002D0218E10D02A502D
:100AE0002FC02AF02F6E29502EC029F02E6E2850CC
:100AF0002DC028F02D6E27502CC027F02C6E2F50C3
:100B00002A5C10E0FF0F09E0219021B403D021AE50
:100B10002184120021AE219412002F2AD8902E3267
:100B20002D322C322C50275E2D50285A2E50295A07
:100B300029BEEAD7D8902736283629362A2EF8D764
:100B4000C8D77F0E2A6EFF0E296E286E276E120000
:100B50007F0E21BEFF0E2A6E02D07F0E2A6E800EFF
:100B6000296E286A276AF3D721AE04D0800E2A6E38
:100B7000296AF7D72A6A296AF4D72350221033103A
:100B80003210F8E025BEF0D723BE0CD0245025103B
:100B9000EBE0D89032363336223623362406D8A0FE
:100BA0002506F2D72550D4E12428D2E032AE11D068
:100BB0007F0E321402E133A00CD0332AE86A2222DD
:100BC000232207E3D880233222323332242A2428F6
:100BD000BFE02450C9E033C027F022C028F02334FE
:100BE000296E24302A6E29322A9E21BE2A8EA7EF32
:100BF00085F029362A3602E32184217E06E1218010
:100C00002A6A296A286A276A12002A2803E0D880FB
:100C100029321200D890293202E121821200218665
:100C200012002E362F3602E3218C217E06E1218828
:100C30002F6A2E6A2D6A2C6A12002F2803E0D880B2
:0E0C40002E321200D8902E32EAE1218A1200E4
:020C4E0011DBB8
:100C5000030EE126020EDB6A000E0901E76EE119C0
:100C6000E8AE02D0E13503D0E750D880E15501E28B
:100C7000E107000E0901E76EE219E8AE02D0E235A5
:100C800003D0E750D880E25501E2E20709010151A3
:100C9000000807E2010703E109019B9102D0090165
:100CA0009B810901A52B000EA623A723A8230901D8
:100CB000035119E0010EE66E58EC72F0E5520DECAE
:100CC0002EF0040EE66E090EE66E000EE66E060EBF
:100CD000E66E02EC98F0E552E552E552E5523AEC48
:100CE0002EF00901036B005171E00501F4516EE033
:100CF000DE6ADD6A8BDA04BE0568C0DA24C003F060
:100D0000D5DAABDA61E08E0E046E510E056E010E7F
:100D1000066EDECF07F0DDCF08F0096A08BE09686D
:100D2000E2DA07C027F008C028F009C029F06DEC0E
:100D300084F024C007F025C008F026C009F0045054
:100D40002424F36E05502520F46E065086DA026ED8
:100D5000036AC8C728F0C9C729F02D6E03C02EF05A
:100D600066ECA8F024C000F025C001F02450251046
:100D700026E1020EDB5002E04CEC72F00F0140B7AE
:100D8000FDD76FDA43DA04BE056827DAF62A000ECB
:100D9000F722F8220800F5CF47FF38DA04BE0568CD
:100DA0001CDA020EF626000EF722F8220800F5CF14
:100DB00048FF0F0148DAF36E020EF3CFDBFFDF2AA4
:100DC000010E98E3DB2A96D70901006B000E006E36
:100DD000030EE15C02E2E16AE55229D24ADA0A0E28
:100DE000E1266250026E036A050ED8900332023289
:100DF000E804FBE16150046E056A030ED8900436E6
:100E00000536E804FBE102500424006E035005207F
:100E1000016E080E00C0DBFF090E01C0DBFF0F0EE4
:100E200065140B01406F66CF41FB67CF42FB68CF73
:100E300043FB69CF44FB6ACF45FB6BCF46FB6CCFCE
:100E400047FB6DCF48FB609E0901010E006F3C0E11
:100E5000016F0B014351DE6EDD6A030E44CBDBFFF5
:100E60004451026E036A080E452544CB00F003C0CE
:100E700001F0000A05E0D89000360136E804FBE1F5
:100E8000040E00C0DBFF050E01C0DBFF09010251AB
:100E9000006E016A0050DF184DE10150DE52DD188E
:100EA00049E1035147E1750EE66EE40EE66E000E71
:100EB000E66E040EE66E090EE66E71EC74F0006EDE
:100EC000050EEBD92D0EE66EE66A730EE66EE40EA5
:100ED000E66E000E75D9080EDBCFE6FF090EDBCFFC
:100EE000E6FF6F0EE66EE40EE66E000E69D9DECF09
:100EF000E6FFDDCFE6FFCBD963D9020EDB6A080E31
:100F0000F36E020EDBCFF4FFF350F45C0FE2020E3F
:100F1000DB50EA6A410FE96E0B0EEA22EF50E66EF3
:100F2000E66AB5D94DD9020EDB2AE9D70901010ECF
:100F3000036F026B400E0B01425D03E342514A080E
:100F400002E2010EA9D0410E425D01E0A4D0000EE4
:100F5000DFCF28F0010EDBCF29F00C0E281801E1BD
:100F6000295066E02F0E281801E129505BE00D0E94
:100F7000281801E1295029E0460E281801E12950DE
:100F80001DE05C0E281801E1295014E00F0E28180E
:100F900001E129500BE0050E281801E07CD0295012
:100FA00001E079D03FD900C0C2F975D03BD900C06B
:100FB000C0F971D037D900C0C1F96DD009013C0E1C
:100FC000E16F7CD900C0ADF966D04B0E0701CB5D57
:100FD00004E1030EDBCF9FF95ED0030EDBCF26F0DA
:100FE000276A286A296AE80E2B6E7DD989ECA7F05A
:100FF00022C026F023C027F024C028F025C029F005
:10100000F40E2626010E2722000E28222922490E40
:101010002B6E060E2C6E2D6A2E6AF1ECA7F026C000
:101020009FF939D0030EDB50640DF4CFA0F933D013
:10103000D950040FE96EDACFEAFFEE50ED1017E158
:101040000901998D999F0901A951AA11AB11AC1100
:1010500022E1A5C9A9F9A6C9AAF9A7C9ABF9A8C9E6
:10106000ACF9A907000EAA5BAB5BAC5B0DD0090124
:10107000999D998F0901A951AA11AB11AC110BE0EF
:10108000A96BAA6BAB6BAC6B010EE66EE66AFEEC6D
:101090003EF0E552E552010E006E0A0EE15C02E2FE
:1010A000E16AE552C4D0E5D8020EE126FC0EDBCFA2
:1010B00028F0FD0EDBCF29F02D0E281826E129504F
:1010C00024E1E5D8E66E01D98CD80CE0B6D8F3CF90
:1010D000DEFFF4CFDDFFDBD8E66E000EE66EE66ADB
:1010E00080D802E1000E12D0A8D8F3CF02F909018E
:1010F000036B4CEC72F00F0140B7FDD7B2D8DFCFD5
:1011000047FF02C948FF9FD801D0000E006E020EB3
:10111000E15C02E2E16AE5528AD0D9CFE6FF020E35
:10112000E12605014F0EC86F320EC96FCA6BCB6B3B
:10113000CC6B0901006B016B026B036B0901E56964
:101140000901A56BA66BA76BA86B900E6F6E6EAEB8
:10115000FED7606A0F01196B1869016BFD0E006FF5
:10116000010E706ED20E716E020E726E200E736ED4
:101170000501F451000802E26F6A02D0600E6F6E42
:101180000701DC0ED56F0D0ED66F010ED76F07016C
:101190004E0EDB6F0C0EDC6F010EDD6F0B01A60E29
:1011A000496F100E4A6F010E4B6F0601EE81EE8300
:1011B000010E006E020EE15C02E2E16AE55237D0F8
:1011C000E66E060EDBCFE6FF070EDBCFE6FFA0ECF8
:1011D00074F0006E070E4DEF89F050D867D86CEFB1
:1011E00089F0E3ECA3F0006E050EE15E0050FA0E0C
:1011F000F3CFDBFFFB0EF4CFDBFFD950FA0FE96E24
:10120000FF0EDA20EA6EEE50ED1012008E0E006E28
:10121000510E016E010E026EDECF03F0DDCF04F041
:10122000056A120009013C0EE26F5EEF89F0E16E83
:101230000050E552E7CFD9FF120047D878EC89F08B
:10124000E552E5521200496B4A6B4B6B4C6B4D6B90
:10125000080E456F406F010E12003ED80800F55091
:101260001200406BE00E426FFB0E416F020E466FA4
:101270001200D9CFE6FFE1CFD9FF120034D803C066
:1012800027F004C028F005C029F06DEF84F06D0E42
:10129000E66EE40EE66E000E1200E15E0050060EF1
:1012A000F3CFDBFF070EF4CFDBFF12000050242446
:1012B000F36E01502520F46E02501200030EDB5035
:1012C000006E280E005E000E1200FA0EDBCFE6FF65
:1012D000FB0EDBCFE6FF12002620F86EF4CFF7FFFF
:1012E000F3CFF6FF1200030E2C6E2D6A2E6A120049
:1012F000FF0EE3CFEAFFE552FF0EE3CFE9FFE55231
:10130000E66AE66AD9CFE6FFDACFE6FFFC0EE12413
:10131000D96EFF0EE220DA6EE66AE66AE66A200E11
:10132000EF5C06E0090EEF5C03E0EF6603D03FD010
:10133000EE50F5D72D0EEF5C03E1FF0EE32A03D04C
:101340002B0EEF5C01E1EE502F0EEF6424D03A0E2D
:10135000EF6021D0D890F90EE336FA0EE336FD0E99
:10136000DECFE3FFFE0EDDCFE3FFD890F90EE336CC
:10137000FA0EE336D890F90EE336FA0EE336FD0E98
:10138000E350DE26FE0EE350DD22300EEE5CDE265C
:10139000000EDD22D9D7FF0EE3CFE8FFE85207E0C9
:1013A000F90EE31EE32AFA0ED8B4E306E31EE55273
:1013B000E552E552FF0EE3CFDAFFE552FF0EE3CF31
:1013C000D9FFE552E1CFE9FFE2CFEAFFED52ED525E
:1013D000EECFF3FFEFCFF4FF1200FF0EE3CFEAFFF3
:1013E000E552FF0EE3CFE9FFE552E66AE66AE66AF8
:1013F000E66AD9CFE6FFDACFE6FFFA0EE124D96E2E
:10140000FF0EE220DA6EE66AE66AE66AE66AE66AF5
:10141000200EEF5C06E0090EEF5C03E0EF6603D000
:101420006BD0EE50F5D72D0EEF5C03E1FF0EE32AF3
:1014300003D02B0EEF5C01E1EE502F0EEF6444D091
:101440003A0EEF6041D0D890F50EE336F60EE33653
:10145000F70EE336F80EE336FB0EDECFE3FFFC0EAD
:10146000DECFE3FFFD0EDECFE3FFFE0EDDCFE3FFB9
:10147000DD52DD52D890F50EE336F60EE336F70E68
:10148000E336F80EE336D890F50EE336F60EE33683
:10149000F70EE336F80EE336FB0EE350DE26FC0EC5
:1014A000E350DE22FD0EE350DE22FE0EE350DD228D
:1014B000DD52DD52300EEE5CDE26000EDE22DE2234
:1014C000DD22DD52DD52B9D7FF0EE3CFE8FFE8524F
:1014D00013E0F50EE31EF60EE31EF70EE31EF80E04
:1014E000E31EF50EE32A08E1F60EE32A05E1F70E06
:1014F000E32A02E1F80EE32AE552E552E552E5520D
:10150000E552D9CFE9FFDACFEAFFEECF26F0EECFF2
:1015100027F0EECF28F0EFCF29F0FF0EE3CFDAFF70
:10152000E552FF0EE3CFD9FFE552E552E552120036
:10153000D9CFE6FFDACFE6FFFA0EE3CFD9FFFB0EF5
:10154000E3CFDAFFFD0EE35209E72D0EDE6EFC0E4F
:10155000E31EE32AFD0ED8B4E306E31EE652E6528C
:10156000E652FD0EE124E76EFF0EE220E46EE65245
:10157000F70EE3CFE6FFF70EE3CFE6FF08EC8BF0C4
:10158000F90EE124E96EFF0EE220EA6EF8EC8AF033
:101590000AE1F5EC8AF009E1F8EC8AF008E1F5ECF3
:1015A0008AF007E108D003EC8BF0FEEC8AF003EC44
:1015B0008BF0FEEC8AF003EC8BF0DE6AF90EE1268C
:1015C000FF0EE222FF0EE3CFDAFFE552FF0EE3CF7C
:1015D000D9FFE552FC0EE124E96EFF0EE220EA6E2F
:1015E000EECFF3FFEFCFF4FF1200EF380F0B120036
:1015F000EF500F0B02E1EE52D8841200EF380F0BC0
:10160000300FDE6E1200EE500F0B300FDE6E120048
:10161000FC0EE3CFE9FFFD0EE3CFEAFF100EE66E0E
:10162000EE6AEE6AEF6AD890FD0EE336FE0EE33600
:10163000ED36ED36EF36FF0EE30609E029EC8BF0D0
:10164000EE5229EC8BF0EE5229EC8BF0EDD7E56EE3
:101650001200030EEF24E8B6EF6E300EEF24E8BE62
:10166000EF6E000CD9CFE6FFDACFE6FFF80EE3CF3E
:10167000D9FFF90EE3CFDAFFFD0EE35215E72D0E89
:10168000DE6EFA0EE31EFB0EE31EFC0EE31EFD0EE5
:10169000E31EFA0EE32A08E1FB0EE32A05E1FC0E45
:1016A000E32A02E1FD0EE32AE652E652E652E65252
:1016B000E652FB0EE124E76EFF0EE220E46EE652F6
:1016C000F30EE3CFE6FFF30EE3CFE6FFF30EE3CF37
:1016D000E6FFF30EE3CFE6FFCFEC8BF0F50EE1244F
:1016E000E96EFF0EE220EA6EBCEC8BF019E1BFEC74
:1016F0008BF018E1BCEC8BF017E1BFEC8BF016E13E
:10170000BCEC8BF015E1BFEC8BF014E1BCEC8BF082
:1017100013E1BFEC8BF012E1BCEC8BF011E112D0C5
:10172000C5EC8BF0CAEC8BF0C5EC8BF0CAEC8BF0FF
:10173000C5EC8BF0CAEC8BF0C5EC8BF0CAEC8BF0EF
:10174000C5EC8BF0CAEC8BF0DE6AF50EE126FF0EDD
:10175000E222FF0EE3CFDAFFE552FF0EE3CFD9FF1F
:10176000E552FA0EE124E96EFF0EE220EA6EEECFBA
:10177000F3FFEFCFF4FF1200EF380F0B1200EF5022
:101780000F0B02E1EE52D8841200EF380F0B300F2E
:10179000DE6E1200EE500F0B300FDE6E1200FA0EEE
:1017A000E3CFE9FFFB0EE3CFEAFF200EE66EEE6A21
:1017B000EE6AEE6AEE6AEF6AD890FB0EE336FC0E34
:1017C000E336FD0EE336FE0EE336ED36ED36ED364E
:1017D000ED36EF36FF0EE3060FE0FEEC8BF0EE5237
:1017E000FEEC8BF0EE52FEEC8BF0EE52FEEC8BF04A
:1017F000EE52FEEC8BF0E1D7E56E1200030EEF2403
:10180000E8B6EF6E300EEF24E8BEEF6E000CFE0E71
:10181000E3CFFEF4FF0EE3CFFFF41200FFC429F084
:10182000FEC428F0350E2D6E450E2E6E4FEC84F062
:10183000262AE86A2722279E27C0FFF426C0FEF446
:10184000FEC4F3FFFFC4F4FF1200D9CFE6FFDACFE6
:10185000E6FFF80EE3CFD9FFF90EE3CFDAFFE65249
:10186000E652E652E652E652FB0EE124E76EFF0E28
:10187000E220E46EE652F30EE3CFE6FFF30EE3CF91
:10188000E6FFF30EE3CFE6FFF30EE3CFE6FFCFEC88
:101890008BF0F50EE124E96EFF0EE220EA6E97EC84
:1018A0008CF019E19AEC8CF018E197EC8CF017E1D0
:1018B0009AEC8CF016E197EC8CF015E19AEC8CF038
:1018C00014E197EC8CF013E19AEC8CF012E197ECB8
:1018D0008CF011E112D0A0EC8CF0A5EC8CF0A0EC17
:1018E0008CF0A5EC8CF0A0EC8CF0A5EC8CF0A0ECCE
:1018F0008CF0A5EC8CF0A0EC8CF0A5EC8CF0DE6A02
:10190000F50EE126FF0EE222FF0EE3CFDAFFE552ED
:10191000FF0EE3CFD9FFE552FA0EE124E96EFF0E88
:10192000E220EA6EEECFF3FFEFCFF4FF1200EF38C4
:101930000F0B1200EF500F0B02E1EE52D884120091
:10194000EF380F0B300FDE6E1200EE500F0B300F22
:04195000DE6E120035
:0C1954000ADB030EE126020EDB6A000E27
:101960000901E76EE119E8AE02D0E13503D0E75096
:10197000D880E15501E2E107000E0901E76EE219A6
:10198000E8AE02D0E23503D0E750D880E25501E25C
:10199000E20709010051000807E2000703E109011D
:1019A0009B9102D009019B810901A52B000EA62362
:1019B000A723A8230901905141E009018E518F11FD
:1019C0003DE0090199A73AD00901012B3C0E015DC8
:1019D00035E3016B0901922B000E9323090190510D
:1019E000026E036A90C928F003C029F08EC92DF059
:1019F0008FC92EF04FEC84F026C000F027C001F014
:101A00000001265009010227000127500901032384
:101A1000000E04230523600E025DEA0E0359000E3A
:101A20000459000E05590AE30901982B600E0901BB
:101A3000025FEA0E035B000E045B055B09010651C1
:101A400001E19AD00501F45101E196D0DE6ADD6A28
:101A500064DA06BE07689FDA0050011001E18AD0FF
:101A6000380E046E510E056E010E066EDECF07F0C5
:101A7000DDCF08F0096A08BE0968050E2C6E2D6AD4
:101A80002E6A07C027F008C028F009C029F06DECC5
:101A900084F024C007F025C008F026C009F00450E7
:101AA0002424F36E05502520F46E06506DDA020EE4
:101AB00061DA0800F550026E036AC8C728F0C9C78A
:101AC00029F02D6E03C02EF066ECA8F024C000F0C3
:101AD00025C001F02450251047E1020EDB5002E042
:101AE0004CEC72F00F0140B7FDD7406B16DA06BE22
:101AF000076851DA070E0016000E0116050ED89081
:101B000000360136E804FBE100C042FF06DA06BEFB
:101B1000076841DA030ED89001320032E804FBE195
:101B200000C041FF0F01750E466F210E476FF5D9BA
:101B300006BE076824DA01C000F0016A00C048FF51
:101B4000ECD906BE07681BDA00500F01496F4A6BDB
:101B50004B6B4C6B4D6B040E456F080E406F010EC6
:101B6000F36E020EF3CFDBFFDF2A010E01E270D726
:101B7000DB2A6ED70901066B000E006E030EE15CD6
:101B800002E2E16AE552DCD1F0D9080EE1266250AA
:101B9000026E036A050ED89003320232E804FBE1BC
:101BA0006150046E056A030ED89004360536E804C9
